:020000040000FA
:040000006FD00400B9
:101000006F00507B000000000000000090200020D6
:10101000AA220020A9BDF9F56C23002000000000E1
:10102000000000006C230020902000200000000041
:101030000000000090200020000000009020002010
:101040000000000090200020902000209020002030
:101050009020002090200020242F00205E240020DB
:101060000000000090200020902000200424002098
:1010700090200020D22300209020002090200020EB
:101080009020002090200020902000209020002020
:101090009020002001A04111B7170040985F3AC688
:1010A000945F3247E39CE6FE3245410182800111A4
:1010B00013078008F337078093F787083EC20100C3
:1010C0000100B7170040930570052380B70413068D
:1010D00080FA2380C7040100010083C6B70493F699
:1010E000F60DA385D704238007049246F3A6068055
:1010F0000100010093760502D5CEF336078093F602
:10110000860836C4010001002380B7042380C70489
:1011100001000100B70614007D89558D88C70100C4
:1011200001000100010023800704A246F3A6068007
:101130000100010073370780137787083AC6010062
:1011400001002380B7042380C704010001000100CF
:1011500001003727004093061005A303D7802380A2
:101160000704B247F3A70780010001009307800836
:10117000F3B7078093F787083ECE01000100B71749
:101180000040130770052380E704130780FA2380CB
:10119000E7040100010003C7B70413670708A3852C
:1011A000E70423800704F247F3A70780010001004A
:1011B0000561828093760504BDC6F336078093F6F9
:1011C000860836C8010001002380B7042380C704C5
:1011D00001000100B7061400938606047D89558D31
:1011E00088C7010001000100010023800704C246F6
:1011F000F3A6068001000100733707801377870884
:101200003ACA010001002380B7042380C70401000B
:1012100001003727004093062005A303D7802380D1
:101220000704D24781B773370780137787083ACC12
:10123000010001002380B7042380C70401000100DE
:1012400098471367070C98C723800704E24719BF24
:101250000111814601468145114506CE97000000E7
:10126000E780005593078008F3B7078093F7870856
:101270003EC601000100B717004013077005238028
:10128000E704130780FA2380E7040100010003C785
:101290006704136717002383E70423800704B2471A
:1012A000F3A7078001000100F2400561828041112F
:1012B000814601468145114597000000E780404F77
:1012C00013078008F337078093F787083EC40100AF
:1012D0000100B7170040130670052380C70493066A
:1012E00080FA2380D70401000100FD552396B70240
:1012F00023800704A245F3A5058001000100733790
:101300000780137787083AC6010001002380C704CD
:101310002380D7040100010003C767041367170087
:101320002383E70423800704B247F3A70780010063
:10133000010001A0BD473305F50201007D1575FDD3
:101340008280411122C426C206C6AA8401446317C2
:101350009400B24022449244410182800504130566
:10136000803E420497000000E78000FD4180C5B741
:101370009305000273A04580824573901534924016
:101380002242B2424243D2436244F2440255925551
:101390002256B2564257D2576258F25806499649D9
:1013A000264AB64A464BD64B664CF64C065D965DD1
:1013B000265EB65E465FD65F09617300203041113C
:1013C000B7170040985F3AC6945F3247E39CE6FE49
:1013D000324541018280B71700401307000323887C
:1013E000E702854717170000232EF74273002030CD
:1013F000411122C406C637040020976000E0E78050
:1014000060DF1C408297D5BF3737004083474700D5
:101410009146BD8B6389D70099466394D700834773
:101420005740730020309736000083C6662C9387A0
:10143000160017360000230DF62A0347870097375A
:1014400000009387E71AB6972380E700B7E7040008
:10145000BC4F0946894517150000034565F482977E
:10146000C9B7B787004003C76700098B6309071036
:1014700003C777009306000313770703630DD708AC
:10148000173800000348586217360000130606613B
:101490000547B30606012380E60083C577001737AA
:1014A000000013072760429793F5F50F2300B7005C
:1014B00003C58700973500009385855EC295137537
:1014C000F50F2380A5000347070089451377F7032D
:1014D000630CB70C63E7E50A6306071A8545630CDE
:1014E000B7129737000083C7375C3307F60003470E
:1014F00007001377F70F19CB850793F7F70F0D4701
:101500006363F71A17370000A300F75AB787004044
:1015100009472383E700B787004083C77700E207C6
:10152000E18763DE07049737000083C7F757173753
:1015300000001307A7563E9785462300D7001737AC
:101540000000130727563E97930600032300D70099
:10155000173700001307C7543E97A146850723009D
:10156000D70093F7F70F0D476364F71417370000A0
:10157000A30CF752B787004009472383E7007300A5
:101580002030930610026300D70E930620026305F5
:10159000D70693060002E316D7F403C72702137792
:1015A000C70F13672700D5A803C767001377070481
:1015B00065CB03C7A702173800001308A82F1735FB
:1015C00000001305E526134707082385E70203C734
:1015D000A7021377370F136787002385E702814738
:1015E00013070004B305F5008C41B306F80091071A
:1015F0008CC2E399E7FEF5B503C7A70213470704BA
:101600002385E70203C7A7021377C70F13672700D5
:101610002385E702F9B503C767001377070449C3B9
:1016200003C76702173800001308881C173500002D
:101630001305C513134707082383E70203C767028F
:101640001377370F136787002383E7028147130758
:101650000004B305F5008C41B306F80091078CC275
:10166000E399E7FEBDBD03C7670213470704238361
:10167000E70203C767021377C70F136727002383A7
:10168000E70285B503C767001377070411CB03C7CB
:1016900027021377370F136787002381E70291B57D
:1016A000238006003DBD97370000A38F073EB9BDDC
:1016B00097370000A38A073E75BD230304801547B2
:1016C0002303E48001002302A480828083076480D6
:1016D000E3CE07FE23030480828083076480E3CE89
:1016E00007FE03454480828083076480E3CE07FEC3
:1016F0002302A4808280411126C44AC24EC006C67D
:101700001377F50BAD47AA892E899544630CF70032
:10171000194597000000E78080FA97000000E780F5
:1017200020FB8D444E8597000000E78040F9FD596D
:10173000FD1463983401B240A24412498249410128
:101740008280135509011375F50F97000000E7809B
:10175000E0F92209F1BF011126CC06CEB70408003A
:1017600097000000E780C0F6154597000000E7806D
:1017700000F597000000E78080F697000000E78002
:1017800000F62AC697000000E78080F43245937780
:10179000150089EB136515001375F50FF240E2444F
:1017A00005618280FD14E9F00145CDBF397126DC69
:1017B0004ADA4ED852D656D45AD25ED006DE62CE1F
:1017C00066CCB7E700E07D5783AA070022C603AACC
:1017D000470023A0E71823A2E718B7170040130714
:1017E00070052380E704130780FA2380E70483C78A
:1017F0004704930B75FFB684E20793FBFB0F854606
:10180000AA892E8B328937240040E187015763FA79
:1018100076016308D5008946130700026313D500DB
:101820000157D98F93F7F70FB71C00402382FC04B0
:1018300011472303E4801305F00F97000000E780B1
:1018400000E8094C97000000E78080E863657C159C
:10185000B7050700DA9537870700795563FEE50479
:10186000B3879500636AF704370B0800A94733EB89
:1018700065016395F90881E8814497000000E780DD
:1018800020E5268515A8DA85094597000000E78040
:10189000C0E605090345F9FFFD14050B970000009C
:1018A000E780C0E481C49377FB0FE5F79700000061
:1018B000E780A0EA69F17D55B7170040130770056E
:1018C0002380E704130780FA2380E70403C7470453
:1018D000418B2382E704F250B7E700E023A05711C1
:1018E00023A24711E25432445259C259325AA25AE1
:1018F000125B825B724CE24C21618280A547639B44
:10190000F90685691309F00FB3069900B3742B012A
:10191000B6941349F9FFB3749900856B3379690163
:10192000416B9387F9FFB3F7270199E363FC340117
:1019300093D94900C147E3E637FF3DBF0569C16957
:101940007D19D9B71305800D63886901130500025D
:101950006384790113051008CA8597000000E780A9
:10196000C0D997000000E78040DF31D54E99B3849D
:1019700034416DBFDA852D4597000000E780E0D740
:10198000CA94E30B99EE050997000000E78020D583
:10199000A30FA9FEFDB79387F9FF93F7F70F636DC8
:1019A000FC0C83C71C04130730086315F7063707C0
:1019B00008006361EB06B3079B00B706100063FBEA
:1019C000D704334BEB0089476399F9068980D549E1
:1019D000E38404EADA85094597000000E780E0D156
:1019E00011090327C9FF91472320E480030764807E
:1019F000E34E07FE23033481FD17EDFBFD14110BAD
:101A000081C49377FB0FE9FF97000000E780E0D4E3
:101A100061F155B5B717004003C75704B707080071
:101A20001377070219E3B78707007955E376FBE8D8
:101A300033079B00E3F9E7F841B58547E380F9F008
:101A4000DA852D4597000000E78020CB9389F4FFCD
:101A5000E38404E297000000E78060C893F7390050
:101A600091EB832604800327090093074900E3963E
:101A7000E6E03E89CE84D9BFB5476399F9001305E6
:101A8000900B97000000E78080C3FDB3B1471305BA
:101A9000B00AE388F9FE99476397F904B70508008F
:101AA000B365BB002D4597000000E78000C5814469
:101AB0008D4BA14997000000E78060C263967401D6
:101AC000832704802320F9008504E39534FF8327CE
:101AD000048013172B01635507002312F90069BB1B
:101AE0002322F90051BB9D47639FF90281451305ED
:101AF000B00497000000E78040C0BD4423200900E7
:101B000023220900FD5997000000E78040BD93F7AC
:101B10007400CA9703C70700FD14398D2380A700FE
:101B2000E39334FF91BBA1476397F9069700000048
:101B3000E780A0C28144630D0B008D479304C0036E
:101B40006308FB009304000563048B0193044004C5
:101B50001375C507E30295D2194597000000E78089
:101B600000B697000000E780A0B60545970000008A
:101B7000E780E0B4268597000000E78020B709459C
:101B800097000000E78080B697000000E780E0BC87
:101B9000E31405CE0DB39147639FF900130560066A
:101BA00097000000E780A0B197000000E78040B2F6
:101BB00013059009F9B5E38109CCF1547DB9BD66EF
:101BC0000147173600001306660B938606A6854567
:101BD0008347060093F7F70F91C382800507E3F967
:101BE000E6FE97370000238BB708DDB77D16620647
:101BF000618693178601E18763D4070001458280DF
:101C0000931726003307F500AE9718439C4363E70C
:101C1000E7007D16E37FF7FC7D55828005458280D5
:101C2000FD15E205E18513978501618793F7F50FAF
:101C300063480700FD15139725002A97584365D779
:101C4000138517006205618582803308B5021C4246
:101C500083A80600B335B502C29733B50701AE9825
:101C6000469585486367B5006394A50063E3070163
:101C700081480C43C6950CC388C21CC28280814730
:101C80001397870161876343B7008280139727000A
:101C90002A97232007008507E5B7814701479396D8
:101CA0008701E18663C5B6001335170082809396DD
:101CB0002700AA9694428507558FD5B793D75540EC
:101CC0008A07AA979C4305453315B5007D8D828010
:101CD00017F3FFDFE702A33D2A8497000000E780A7
:101CE00060F405C5931725003E940327C4FF814780
:101CF00011EB7D1516053E954205418517F3FFDF73
:101D00006700233D05838507E5B70145C5BF8147CA
:101D10001397870161876343C70082801397270069
:101D2000B386E50094422A97850714C3D5B77D167C
:101D300062066186014793178601E18763D5070034
:101D400013351700828093172600B306F500AE976F
:101D500094429C437D16B58F5D8FF1BF8A05AA958D
:101D600001476363B500828083A6C5FFF11593D751
:101D70001600D98F9CC11397F601E5B72A83014855
:101D8000014701456343D7008280B387050183A8DB
:101D90000700B30706019C43C697AA976384F8001F
:101DA00033B517010507B3080301620723A0F80044
:101DB00061871108C1BF2A8301478147014563C379
:101DC000D70082803388E50083280800330EE600C0
:101DD000032E0E003388A8403308C84163840801ED
:101DE00033B508018507B308E300E20723A0080123
:101DF000E1871107E9B717F3FFDFE702432B011172
:101E0000B286B2842E86AA850A8597000000E780F4
:101E1000C0FA2A84A6850A8597000000E78020E89A
:101E200033348000060413351500018D056117F366
:101E3000FFDF6700032A17F3FFDFE702C324411126
:101E4000AA89AE8A328BB68402C202C402C6014499
:101E5000131C8401135C8C4163499C02939B140006
:101E6000FD1B0549138CF4FFF15C33048901620406
:101E700061846340740792478E04CE9423AEF4FECF
:101E8000410117F3FFDF6700832313192400B30B0D
:101E90002B01014A93172A00D69783A50B0088438C
:101EA00078003400500097000000E78040DA050A0F
:101EB00093178A01E187F11BE35EFCFC92474E9980
:101EC00005042320F900A2473EC2B24702C63EC421
:101ED00041B7131A8901135A8A41131D240093171D
:101EE0008A01E18763CF970092470A044E941CC091
:101EF000A24705091379F90F3EC2B24702C63EC494
:101F0000ADB7B3079A0313152A0056950841780018
:101F100034005000050AEA97DA978C4397000000D6
:101F2000E780E0D26DBF0000197106C212C416C668
:101F30001AC81ECA22CC26CE2AD02ED232D436D6E9
:101F40003AD83EDA42DC46DECAC0CEC2D2C4D6C6D9
:101F5000DAC8DECAE2CCE6CEEAD0EED2F2D4F6D6C9
:101F6000FAD8FEDA971500009385458B8841E70083
:101F7000050092402242B2424243D2436244F244BC
:101F8000025592552256B2564257D2576258F258CD
:101F900006499649264AB64A464BD64B664CF64CFD
:101FA000065D965D265EB65E465FD65F096173008C
:101FB00020300000972100209381C1041751002098
:101FC0001301418417F5FFFF130505049705002051
:101FD00093854503171600201306C6FD63FAC50056
:101FE0008322050023A0550011059105E3EAC5FEF3
:101FF00017050200130505DE97150020938585FB64
:10200000171600201306066563FAC5008322050033
:1020100023A0550011059105E3EAC5FE1715002020
:102020001305456397450020938545116377B500F7
:10203000232005001105E36DB5FEFD42739002BC3F
:102040008D4273904280B722000093828288739001
:102050000230970200209382E2FA93E232007390FA
:102060005230975200009382E293739012346FB013
:10207000347973002030397101436EC619A039716B
:1020800041536AC866CA62CC5ECE19A03971015349
:102090005AD056D252D44ED64AD826DA22DC06DEA0
:1020A00033016140828241114AC026C222C406C661
:1020B0008282B24D4101024D924C224CB24B410101
:1020C000024B924A224AB2494101024992442244B7
:1020D000B240410182803D432A876373C3029377F4
:1020E000F700BDEFADE5937606FF3D8ABA960CC3C7
:1020F0004CC30CC74CC74107E36BD7FE11E282808B
:10210000B306C3408A069702000096966780A60031
:102110002307B700A306B7002306B700A305B7003F
:102120002305B700A304B7002304B700A303B70037
:102130002303B700A302B7002302B700A301B7002F
:102140002301B700A300B7002300B700828093F5F6
:10215000F50F93968500D58D93960501D58D61B7C2
:10216000939627009702000096968682E78086FA6B
:102170009680C1171D8F3E96E374C3F8A5B73367E9
:10218000B500FD530D8B79E7B7877F7F9387F7F70E
:1021900010419441B372F6003363F600BE92B3E28D
:1021A00062006397720C6318D6065041D441B37233
:1021B000F6003363F600BE92B3E262006398720ADF
:1021C000631BD60410459445B372F6003363F600E2
:1021D000BE92B3E262006391720A631ED60250455A
:1021E000D445B372F6003363F600BE92B3E26200E8
:1021F000639A72086311D60210499449B372F600CB
:102200003363F600BE92B3E2620063937208510535
:10221000D105E30FD6F61317060193970601631C49
:10222000F7001357060193D706013305F74093755E
:10223000F50F91E982804183C1833305F74093759F
:10224000F50F91E182801377F70F93F7F70F3305BE
:10225000F74082800346050083C605000505850515
:102260006313D60065FA3305D640828011059105C7
:10227000E312D6FE014582802105A105E31CD6FCB0
:10228000014582803105B105E316D6FC0145828007
:102290004105C105E310D6FC01458280B717004017
:1022A00003C777051377E70FA38BE704130700F83D
:1022B000A38DE7043D47238CE70413075003A38C49
:1022C000E70403C7A7051377D70F238DE7048280A0
:1022D000B717004003C7E7020D8941111377C70FF5
:1022E000498F93068008F3B6068093F6860836C6B3
:1022F00001000100930670052380D704930680FA3D
:102300002380D704010001002387E702238007040C
:10231000B247F3A70780010001004101828041110B
:102320002A83014E930E407E130F0019930F40062F
:1023300063E56E129308001913034006B378150382
:10234000854E0D4FA14F337365020D89133515006E
:1023500063EFBE121308F6FF7946729842081358CD
:1023600008013307C70213D61700BE07329761462C
:10237000B3F6C60213068070B386C6023697A1660E
:10238000F58F42075D8FB716004083C7F60293F7BB
:102390000708A303F1000346710083C7F60293F711
:1023A0000708E394C7FE83477100B716004093F710
:1023B000F70F6388071293078008F3B7078093F736
:1023C00087083EC401000100B7170040930670055E
:1023D0002380D704930680FA2380D70401000100EC
:1023E00023AA070383C6170393E60608A388D70228
:1023F00023800704A247F3A70780010001001166AC
:10240000B71700407D16D45BC85F93854703A98E3C
:10241000F18EF5FA93068008F3B6068093F68608E7
:1024200036C601000100930670052380D704930689
:1024300080FA2380D7040100010098C103C7170365
:1024400013670704A388E70223800704B247F3A7B2
:10245000078001000100410182807D133368E3039E
:102460009308E016630E08003368F3039308D01650
:10247000630808009378330093B818009388D8163F
:1024800033081E01131E0801135E0E0155B5639338
:10249000E5030548638608000148630303002A88B2
:1024A00071087298FD15131E0801C205135E0E0116
:1024B000C18179BD13F8150063F4BF007908D5B761
:1024C00013381800E5BF83C7F60293F70708A30384
:1024D000F1000346710083C7F60293F70708E394FF
:1024E000C7FE8347710093F7F70FF1DFE9B531714C
:1024F0004AD966CB06DF22DD26DB4ED752D556D32E
:102500005AD15ECF62CD6AC96EC7AA8C02D8971025
:102510000000E78020B12A8993078008F3B707807D
:1025200093F787083EDA01000100B7170040130750
:1025300070052380E704130780FA2380E704010075
:10254000010003C7F7021377770FA387E70203C7DA
:10255000F70213678700A387E70223800704D25797
:10256000F3A7078001000100054597000000E78000
:1025700060D6130780C13347E902116A93070AE85E
:1025800093065002BD69930BA004814A014B1304CA
:102590008008930470057D1AB347F9023307D70208
:1025A0003EC0FD873ECC938709A69309803E334702
:1025B000F7023AC27D873AC4334739038549B39954
:1025C000990193D93940B306D702B30B7703B3C649
:1025D000F602B3CBFB0236C6FD8636C893D6FB4166
:1025E00036CEB7460F00938606243349D902856656
:1025F000938606FAB3969601B389E90213076055EC
:102600003309D90293060010B389E9023349D9028C
:10261000B3C9F9029316390036CA37190040FD864E
:1026200036D0930D090493D7F9413ED2F336048096
:1026300093F6860836DC01000100930770052380BD
:10264000FD00930680FA2380DD000100010083462F
:10265000390593F6860FA309D9048346390593E615
:102660001600A309D90423800D00E256F3A60680C4
:1026700001000100130C80FA116DF336048093F60B
:10268000860836DE01000100930770052380FD00F7
:1026900023808D010100010083463905216693E600
:1026A0000602A309D90483560905B3E6A601231837
:1026B000D90483560905D18E2318D90423800D002F
:1026C000F256F3A60680010001008346390593F611
:1026D00006026381061A03463905218A6DDE081851
:1026E00097100000E7800098733604801376860800
:1026F000B2C20100010023809D0023808D010100F2
:102700000100B717004003C637051376F60DA389FD
:10271000C70403C6370513660602A389C704835698
:1027200009052166B3E6A6012318D90483560905D5
:10273000D18E2318D90423800D009646F3A6068077
:10274000010001008346390593F60602638B0614E7
:1027500083463905A18AEDFE97000020E780A0930B
:10276000AA8636D497000020E780E092A256E30ABA
:10277000D5FE835609054255B3E6A6012318D904B0
:1027800097100000E780C08F83463905A18AEDDEEF
:10279000035609058346290582473376CA00B306E6
:1027A000DA0293D5F641B296B388F640E24733B8E1
:1027B000C6002E983308F840A247B3B61601330876
:1027C000D84063C70701631DF800924763FA1701F9
:1027D000C247634FF80E63950701B24763EAF80EEC
:1027E000894663E9660FF2469315180013D3F80182
:1027F0005E8613951800B365B30042D646D497B0F1
:102800000100E780E07B3258050B137BFB0F634729
:102810000001631A0838A2586387083813081500A6
:10282000B336A800B69513D6F5013298B336C80072
:10283000AE9613581800FE06B3E606017336048000
:1028400013768608B2C60100010023809D00238014
:102850008D01010001000356C902B296C206C18271
:102860002316D90223800D00B646F3A60680010088
:10287000010021B5F336048093F68608B6C0010046
:10288000010023809D0023808D010100010083460B
:10289000390593E60602A309D90423800D00864674
:1028A0000DB5F336048093F68608B6C40100010026
:1028B00023809D0023808D0101000100834639059E
:1028C00093E60602A309D90423800D00A646BDB5F0
:1028D000E30B0BF0F336048093F68608B6C80100CC
:1028E0000100930680FA23809D002380DD00010013
:1028F00001008346390593F5FC0F93F6860FA30973
:10290000D90483463905CD8EA309D90423800D004F
:10291000C646F3A6068001000100130580FA0346AF
:102920003905930639051D8A631C96297336048080
:1029300013768608B2CC01000100130680FA2380CA
:102940009D002380CD000100010003C60600137620
:10295000F60D2380C60003C6060013660602238018
:10296000C600835609051166D18E2318D9048356F3
:1029700009052166D18E2318D90423800D00E6466F
:10298000F3A6068001000100130680FA834639058C
:1029900093F606026380062683463905130C390533
:1029A000A18AFDDA081897000000E780A06BF336D3
:1029B000048093F68608B6D001000100930680FAE1
:1029C00023809D002380DD000100010083460C0070
:1029D000116693F6F60D2300DC0083460C0093E6A7
:1029E00006022300DC0083560905D18E2318D90482
:1029F000835609052166D18E2318D90423800D0042
:102A00008656F3A6068001000100130680FA83466D
:102A1000390593F60602638A062083463905A18AA2
:102A2000EDFE97F0FF1FE78000672A8C97F0FF1FED
:102A3000E7806066E30C85FF835609051166425501
:102A4000D18E2318D90497000000E7806063834685
:102A5000390513063905A18AFDDAF336048093F6A9
:102A60008608B6D401000100930680FA23809D00F9
:102A70002380DD00010001008346060093F6F60D79
:102A80002300D60023800D00A656F3A60680010081
:102A900001008356090503462905D247B376DA00BB
:102AA0003306CA021305800C9355F6413696330D52
:102AB000F6408257333CD6002E9C3336A601330CA9
:102AC000FC40330CCC403308850392564E86B33518
:102AD000A5033305A503C29597B00100E780404EDA
:102AE00063468001631E0C16630C0D161306150059
:102AF0003335A6002E959356F5013696B335D6009C
:102B0000AA959396F50105828585D18E6346B0001E
:102B1000639D051A638B061A0356C9021582330595
:102B2000D6003336C500B2956348B00063910524E2
:102B30001306F00F637DA622894663F356159307AB
:102B40008008F3B7078093F78708BED6010001001D
:102B500037170040930770052300F704930780FAA6
:102B60002300F704010001008356C702896781171B
:102B7000D58FC207C1832316F70223000704B65777
:102B8000F3A7078001000100FA506A54DA544A5949
:102B9000BA592A5A9A5A0A5BFA4B6A4CDA4C4A4D8D
:102BA000BA4D296182801308F5FF3335A800FD1561
:102BB0002E951356F5013298B336C800AA9695B9EA
:102BC000F336048093F68608B6CA0100010023801C
:102BD0009D002380AD000100010083463905CD8EA4
:102BE000A309D90423800D00D646F3A60680010070
:102BF000010035B3F336048093F68608B6CE0100A3
:102C0000010023809D002380CD0001000100834648
:102C1000390593E60602A309D90423800D00F64680
:102C2000F3A606800100010095B3F336048093F605
:102C30008608B6D20100010023809D002380CD00CC
:102C4000010001008346390593E60602A309D90471
:102C500023800D009656F3A606800100010045BBB7
:102C60009306F5FF33B5A600FD152E959355F50196
:102C7000AE96B3B5B600AA951396F501858269B5EF
:102C8000F336048093F68608B6D801000100930657
:102C900080FA23809D002380DD000100010083561F
:102CA000C9020566011693F6F60FD18EC206C182DF
:102CB0002316D90223800D00C656F3A60680010014
:102CC0000100850A93FAFA0F95B233E6B60045C2C1
:102CD0000356C9023305D0403338A000B305B040D5
:102CE000B385054115826345B000D1E16371A60843
:102CF000894663F0560593078008F3B7078093F77A
:102D00008708BEDA01000100B717004013077005FD
:102D10002380E704130780FA2380E7040100010001
:102D200003D7C7027D8B2396E70223800704D6577B
:102D300081BDF336048093F68608B6DC01000100FD
:102D4000930680FA23809D002380DD0001000100AE
:102D50008356C9020566011693F6F60FD18EC20698
:102D6000C1822316D90223800D00E656B9B7930716
:102D70008008F3B7078093F78708BEDE01000100E3
:102D800037170040930770052300F704930780FA74
:102D90002300F704010001000356C7029397560071
:102DA000B297C207C1832316F70223000704F65720
:102DB000C1BB914763EEB70217D701001307C70BDA
:102DC0008A05BA959C41BA978287B717004003A736
:102DD000470B1345F5FF698F23AAE70A03A7070BE3
:102DE000698F23A8E70A03A7070A798D23A0A70AFA
:102DF0008280B717004083A6470B1347F5FFF98E73
:102E000023AAD70A83A6070B558D23A8A70A83A652
:102E1000070A758F23A0E70A8280B717004003A72F
:102E2000470B498F23AAE70A03A7070B1345F5FFB2
:102E300045BFB717004083A6470B1347F5FF758FB3
:102E400023AAE70A03A7070A598D4DB7B717004011
:102E500003A7470B498FEDB7914763EEB70217D72A
:102E600001001307A7028A05BA959C41BA97828789
:102E7000B717004003A7470D1345F5FF698F23AA35
:102E8000E70C03A7070D698F23A8E70C03A7070C1E
:102E9000798D23A0A70C8280B717004083A6470D29
:102EA0001347F5FFF98E23AAD70C83A6070D558D7E
:102EB00023A8A70C83A6070C758F23A0E70C82809C
:102EC000B717004003A7470D498F23AAE70C03A7B4
:102ED000070D1345F5FF45BFB717004083A6470D03
:102EE0001347F5FF758F23AAE70C03A7070C598D2D
:102EF0004DB7B717004003A7470D498FEDB779715C
:102F000022D43714004026D24AD0035924028354D5
:102F1000040206D64209C2044ECE52CC56CA1359F8
:102F20000901C1802DE11379F9F793F4F49F420967
:102F3000C20413590901C18093078008F3B70780C1
:102F400093F787083EC40100010093077005230032
:102F5000F404930780FA2300F40401000100231114
:102F600024032310940223000404A247F3A707803C
:102F700001000100B250225492540259F249624AAF
:102F8000D24A45618280B7F5070081463000B1051D
:102F9000194597000020E7806081A2471397270119
:102FA000E34A07FC1369090893E404409309800885
:102FB000F3B7098093F787083EC001000100930A28
:102FC000700523005405130A80FA2300440501000C
:102FD00001002311240323109402230004048247D8
:102FE000F3A7078001000100294597F0FF1FE78044
:102FF0006034F3B9098093F989084EC201000100D9
:1030000023005405230044050100010083570402F6
:1030100093E707202310F402230004049247B9B772
:10302000B71700408847420541819377050491EB2B
:103030009377F5013755E801130505803345F5020F
:1030400082809377050C130700046397E70093775A
:10305000F50137459C1CCDB72165130505D082804D
:1030600037E700E01C435443A183E206D58F1CC11F
:10307000FD572320F7182322F718828013178500A5
:10308000B7E700E023A0E710618123A2A7108280A8
:10309000B7F700E08847CC47828081473737004048
:1030A000A14663C4C700328582800345B740E38EE2
:1030B000A6FE3385F5000345050085072304A740D8
:1030C000CDB7970700209387E7EE9C431737002082
:1030D0001307C7063E95636EE500173700201307F8
:1030E00067526368A700170700202325A7EC3E85D9
:1030F0008280FD57EDBF8280411122C406C62A841A
:1031000097000000E78000F22947B307E502B240CC
:103110008D83B3D7870222449507B3D7E7023737A9
:103120000040C207C1832316F70041018280716508
:1031300041111305052006C697000000E78000FC3A
:10314000B7370040130770F82381E7000D47A381CC
:10315000E70013070004A380E70005472387E70083
:10316000B2404101828037370040834727001A056B
:1031700093F7F703C98F93F7F70F2301F7008280C6
:10318000B737004003C7170019C9D98DA380B7000E
:1031900003C70700136787002380E700828093C579
:1031A000F5FFF98DA380B7008280AE872A87B736F6
:1031B000004021463738004089E7170300006700C8
:1031C000C3F383C8B600E30916FF05078348F7FF7A
:1031D000FD17C20723041801C183F9BF411122C49E
:1031E00006C62A8497000000E780C0E32947B3079A
:1031F000E502B2408D83B3D7870222449507B3D747
:10320000E70237370040C207C1832316F740410168
:103210008280716541111305052006C697000000E4
:10322000E78000FCB7370040130770F82381E740C0
:103230000D47A381E74013070004A380E74005473B
:103240002387E740B24041018280CC41411106C64C
:10325000328503C6150083C5050022064D8E420641
:103260008D654186138875A2630C0611634BC804F3
:10327000138845A26300060D634AC800938535A2F2
:103280006301B6082390060029464DA0138855A275
:103290006305060D938565A2E316B6FE8D451D46B2
:1032A00063E6E5081146198E63F3C7003E86B7E76B
:1032B00004002390C600FC4797D50100938545BFC5
:1032C0009DA0138895A263030611634E060D138813
:1032D000A5A263000613938505A5E315B6FA9945E3
:1032E0001D4663E5E504198E63F3C7003E86B7E724
:1032F00004002390C600FC47970500209385C5D5A0
:103300001DA09D451D4663E3E5022146198E63F32A
:10331000C7003E86B7E70400FC472390C600970528
:1033200000209385A533BA9582970146B240328535
:1033300041018280AD451D46E3EAE5FE3146198E26
:1033400063F3C7003E86B7E704002390C600FC473E
:1033500097D50100938545B8F9B7B1451D46E3E718
:10336000E5FC3546198E63F3C7003E86B7E70400D7
:103370002390C600FC4797D501009385E5B665B755
:103380008D451D46E3E4E5FA1146198E63F3C70047
:103390003E86B7E704002390C600FC4797D501009E
:1033A0009385C5B149B78D451D46E3E1E5F8114662
:1033B000198E63F3C7003E86B7E704002390C6006A
:1033C000FC4797D501009385E5B3B1BFA5451D46E0
:1033D000E3EEE5F42946198E63F3C7003E86B7E7AE
:1033E00004002390C600FC4797D501009385C5AD26
:1033F0001DBFB5451D46E3EBE5F23946198E63F373
:10340000C7003E86B7E704002390C600FC4797D567
:1034100001009385E5A801BFB7E7040003A30713E4
:1034200097060020938646C24146A5451705002011
:10343000130585B802832D455DE703C505000947DF
:10344000631FE50803A84500411106C6034718009D
:1034500032850346080022074168518F930828FEF1
:103460006307170563E9E800051863030703239062
:103470000600294591A8130648FE630AC7041518DB
:10348000E31707FF15463E87637BF600154701A843
:10349000130600023E876374F60013070002B7E7C5
:1034A00004002390E600FC471316070111A83E868E
:1034B00091C30546B7E70400FC472390C6004206C7
:1034C000CC45418282970145B2404101828013067A
:1034D00000083E87E375F6FC13070008C9B7239080
:1034E0000600054582808280416779176304E50400
:1034F000411122C406C685472A84639FF500B7E7B9
:10350000040022852244B24003A3871397050020BC
:103510009385052F4101028389476399F500B7E739
:10352000040083A7070B8545829771D9B2402244D6
:10353000410182808280797122D452CC2E842A8AE1
:1035400097D501009385059E17D50100130505A0A9
:1035500006D63AC626D24AD0B68432894ECE97B025
:103560000100E78020F1A68517D501001305059F0E
:1035700097B00100E78000F0294597B00100E7808F
:1035800040F48347840093F70702E1E7834904008E
:103590008947054532476396F908544083C71600AA
:1035A00083C60600A207D58FC166138616FE638CFC
:1035B000C7028D16638FD7068D66938626902945A0
:1035C0006391D706B7E70400A285225403A34714EA
:1035D000B250F249A6864A86925402595285624AEE
:1035E0008547456102832D450DEF93070002354560
:1035F00063E99702B7E70400FC474844130600025A
:10360000CA858297814997070020938727209C438A
:10361000014581CB9C4391C74E852686CA858297FA
:103620000145B250225492540259F249624A45610E
:1036300082802D457DF79307700F3545E3E397FEB4
:10364000B7E70400FC4748441306700FCA85829709
:103650005DBF2145F9B7411122C437E40400832737
:10366000841326C2AA84416506C697050020938567
:1036700025197D1582978327C40A170500001305B5
:10368000E5E68588829795C0032304132244B2405F
:103690009244970600209386A6AD4146C54517057E
:1036A00000201305E59B41010283B240224492446D
:1036B00001454101828019C59707002023A8A7145E
:1036C00001458280454582801147636AA70A97D6E3
:1036D00001009386E6830A0536951841411106C616
:1036E0003697AE87B2850287130700026145639D56
:1036F000E700B7E70400FC471306000217050020A7
:10370000130545F682970145B24041018280054785
:103710006145E39BE7FEB7E70400FC470546170554
:103720000020130525F6F9BF1307700F6145E39DCF
:10373000E7FCB7E70400FC471306700F17050020ED
:10374000130585F4C1B7130700086145E39EE7FA46
:10375000B7E70400FC47130600081705002013050F
:1037600025024DB715476145E390E7FAB7E7040036
:10377000FC471546170500201305C50861B7094524
:103780008280411126C2B7E4040083A7C41322C477
:103790004AC006C62E8497050020938565062A89AF
:1037A0008297058905C5970700209387678B83D784
:1037B000A70BA28503A3440D2310F4002244B240BA
:1037C00092444A850249014641010283B2402244A3
:1037D000924402494945410182809707002023898C
:1037E00007029707002023A70702B717004003A787
:1037F000070CB706C0FFFD16758F23A0E70C03A7C3
:10380000070DB7064000558F23A8E70C03A7070C48
:103810003D9B23A0E70C03A7070D1367070123A80F
:10382000E70C8280B717004003A5470C83A7470C1D
:10383000598113451500C18B058999E3136525004E
:103840009707002083C7C7FC6380A7029707002063
:103850002380A7FC11C9970700209387A7FB03A328
:1038600007006303030002838280114517F3FFFF03
:10387000670023C8411193962500AA852D4506C6E9
:1038800097F0FF1FE78080F2B2400145410182803E
:10389000011122CC06CE3714004026CA4AC84EC6B3
:1038A00052C483447405034AB4058349840503491B
:1038B000940597F0FFFFE780A09E8347A40593F44B
:1038C000F40F137AFA0F93E71700230DF40493F91A
:1038D000F90F1379F90FB717004003C7A705058B38
:1038E0006DFF03D5C705A38D4705238C3705A38C32
:1038F0002705A38B9704F2406244D2444249B2495F
:10390000224A0561828041119397050122C406C6AF
:1039100026C2C1872E8463DC0700B7E40400FC5490
:10392000829719C1BC5482972165218D15A893F700
:10393000150013C515008DE793F725009DC7970067
:103940000000E78060EEB7E70400BC4F1306000AF2
:10395000894517050020034565EC8297134524002F
:10396000B24022449244410182809397250163D85A
:103970000702B7E4040083A7C41E829797000000E3
:10398000E780E0EEBC4C3756070013060630896529
:1039900017050020034585E88297096579B7939755
:1039A00015010145E3DE07FA17C50100130505639C
:1039B00097B00100E780E0C3B7E70400BC4F1306EF
:1039C0000064916517050020034545E58297116560
:1039D000A9BF2D71232A9110FD74E98C232C81102D
:1039E00023282111232631112A84AE893289930696
:1039F00000100A86A6852D45232E111097F0FF1F73
:103A0000E780C0DA13154401B7E70400FC47518191
:103A10000A0513962900CA850A958297A6858566A8
:103A20000146254597F0FF1FE78040D80A86A68506
:103A300093060010294597F0FF1FE78020D78320C9
:103A4000C111032481118324411103290111832908
:103A5000C11015618280B7F7070003C70701411144
:103A600006C622C426C24AC0A547631DF7009700B8
:103A70000000E78040F6B2402244924402490145EA
:103A80004101828013942500AA843289A286AA85E6
:103A90000146254597F0FF1FE78040D1A2864A8660
:103AA000A685294597F0FF1FE78040D0E9B71D7133
:103AB000A2CC37E404005C5C485886CE494697C5E2
:103AC00001009385254D829711E917C50100130563
:103AD000A54D97B00100E780C0B101A0B7F600E0A6
:103AE000795798CAFD57DCCA0567B7E700E023A0FD
:103AF000E7101306F00290C223A0E71801000100AE
:103B00003707002018471306000481459706002058
:103B100023A4E6D04157A38AE7403C440808829793
:103B2000970700209387476C3EC885671387074037
:103B3000231AE1001D673ACC370701051307071068
:103B40003ACE938757D11307B00F2310E102231207
:103B5000F102054797F7FFFF9387C7532301E1025F
:103B60003ED817070000130727D197070000938757
:103B700067D2B7F50700BAC23EDC1707000013078B
:103B8000C7ED97070000938787CE81463000E10597
:103B90001945BAC43EDE97F0FF1FE78020C1180820
:103BA0008147994630003E96034606008507050783
:103BB000A30BC700E398D7FEC24791C70357410143
:103BC00085676373F70001A0B7E7040083A7470A7E
:103BD00008088297AA8511C917C501001305053E7B
:103BE00097B00100E780008901A0F6406644256196
:103BF0008280411126C2B7E4040083A7040806C6E8
:103C000022C417050000130545D082971704002031
:103C10001304C4C02300A40097000000E7808002C2
:103C200097000000E780A0BB03450400224403A3E3
:103C30008405B24092441306003289654101028333
:103C4000797106D622D413078008F337078093F7DB
:103C500087083EC201000100B717004093057005B8
:103C60002380B704130680FA2380C70401000100F3
:103C700083C6F70293F6A60FA387D7022380070413
:103C80009246F3A606800100010073370780137780
:103C900087083AC4010001002380B7042380C704C9
:103CA0000100010003C7F70213672700A387E7029B
:103CB00023800704A247F3A7078001000100054500
:103CC00097E0FFFFE780006197000000E78020BADF
:103CD000014781468147054685451305407E97E0AB
:103CE000FFFFE780006437E404003C44680051466D
:103CF00081458297B707C0A83EC8B787E803938776
:103D000007D03ECA97E7FF1F9387676B3EC67C5874
:103D100068008297B250225445618280411197D544
:103D200001009385E59117C501001305252206C6FC
:103D300097A00100E780007417D50100130505A9BD
:103D400097A00100E7800073B2402945410117A305
:103D5000010067000377411197D501009385858F96
:103D600017C501001305851E06C697A00100E78050
:103D7000607017D50100130525A497A00100E78006
:103D8000606FB2402945410117A3010067006373CA
:103D9000411122C406C6834705002A849DC797D5D2
:103DA00001009385E59017C501001305251A97A01A
:103DB0000100E780206C4C4017D50100130545B584
:103DC00097A00100E780006B3DA058410DEF97D50B
:103DD00001009385E58D17C501001305251797A0F0
:103DE0000100E780206917D501001305E5B397A00E
:103DF0000100E78020682244B2402945410117A311
:103E000001006700036CA1679386D7036313D70291
:103E100097D501009385C58917C5010013050513C2
:103E200097A00100E780006517D501001305C5B014
:103E30007DBFED0797D501009385858717C50100E4
:103E40001305C510631BF70097A00100E78080628F
:103E500017D50100130585AF59BF97A00100E78072
:103E600060614C4017D50100130545B091BF411169
:103E700097C501009385457F17C501001305050D02
:103E800006C697A00100E780E05EB24029454101E7
:103E900017A301006700E362797122D426D24AD0C9
:103EA0002E842A898145B2844800714606D697E05F
:103EB000FFFFE780802297F7FF1F9387274CDC479F
:103EC00083D70700231421012313F100974000003A
:103ED000E780C07D9547A305F1009307401F3EC6CC
:103EE000FD572305A100230AF10097500000E78049
:103EF00020902686A285480097400000E780E07D5C
:103F0000B250225492540259456182809717002082
:103F1000239F077C971700202388076CB7E70400CE
:103F2000BC47411106C641468145170500201305CF
:103F3000251A829797200000E780005E97200000F6
:103F4000E7802039014597500000E780801B170764
:103F500000200347E7199307F00A6315F702930758
:103F6000F0F889451705002013058518170700206C
:103F70002300F71897070020A38C0716975000001E
:103F8000E780204897500000E780005A81453705B8
:103F900004009707002023AB071297070020239502
:103FA0000712970700202382071297070020239308
:103FB000070A9707002023910708970700202394FA
:103FC000071097070020239D071097300000E78017
:103FD000C0C1014597500000E780A04B97C5010084
:103FE0009385056B17C50100130545F697A00100E1
:103FF000E780404817D501001305859D97A0010073
:10400000E7804047B2402945410117A301006700FE
:10401000434B411122C406C626C293F715002E84D5
:10402000638F0710814617F6FF1F1306663285451A
:10403000170500200355050097C00000E78040B534
:1040400015C997C501009385656517C5010013055E
:10405000E5EF97A00100E780E04117C501001305D7
:10406000A50697A00100E780E040294597A0010040
:10407000E780204597C501009385456217C501007B
:104080001305C5EC97A00100E780C03E17C50100ED
:104090001305C50497A00100E780C03D294597A0FE
:1040A0000100E780004217F5FF1F1305252D5C4531
:1040B00005472390E70097300100E780C06597C56A
:1040C00001009385A55D17C50100130525E897A09C
:1040D0000100E780203A17C501001305650197A08C
:1040E0000100E7802039294597A00100E780603D65
:1040F000930710F817070020230CF7FE97070020FE
:1041000083D707F317070020A304F7FE1705002045
:10411000130505FEA183914517070020230BF7FC2B
:1041200097070020A38707FC97500000E780602DC9
:1041300013451400B240224492444101828093F717
:104140002500E1C317070020035707F845CB970662
:1041500000209386A6F7944297D70100938747895A
:1041600017060020034666F6814517050020130553
:1041700025F697700000E78000C1AA8441C197C569
:1041800001009385655817C50100130525DC97A02C
:104190000100E780202EA68517C501001305C5F68E
:1041A00097A00100E780002D294597A00100E78036
:1041B000403197070020239907F0930710F817075D
:1041C00000202307F7F29707002083D767E6170739
:1041D0000020A30FF7F0A18317070020230BF7F0AF
:1041E00091458D4717050020130585F0170700201E
:1041F000A301F7F097500000E780A02013452400AA
:1042000015BF93F74500D1C397C501009385C54FEE
:1042100017C50100130585D397A00100E78080250D
:1042200017C50100130505F097A00100E780802461
:10423000294597A00100E780C028930720F81707B9
:1042400000202307F7EA9707002083D7A7E0170786
:104250000020A30FF7E8A18317070020230BF7E83E
:10426000854717070020A306F7E897400000E7807E
:104270002058170500201305A5E791459750000029
:10428000E78020181345440075B593F78500A9C74A
:1042900097C501009385454717C50100130505CB58
:1042A00097A00100E780001D17C501001305C5E8B0
:1042B00097A00100E780001C294597A00100E78036
:1042C000402097070020239107E097700000E780C7
:1042D00060BB13458400B9BD93F70501D1C3854583
:1042E00017050020035505D797500100E780806D22
:1042F00097C501009385454117C50100130505C504
:1043000097A00100E780001717C50100130505E419
:1043100097A00100E7800016294597A00100E780DB
:10432000401A930730F8170700202303F7DC97079C
:10433000002083D727D217070020A30BF7DA170531
:1043400000201305E5DAA1838D451707002023021D
:10435000F7DA97500000E780C00A13450401D9BB83
:1043600093F70502D1C797C501009385E53917C5B5
:1043700001001305A5BD97A00100E780A00F17C598
:1043800001001305E5DE97A00100E780A00E294596
:1043900097A00100E780E012930740F8170700207C
:1043A0002308F7D49707002083D707C917070020F1
:1043B000A300F7D4A18317070020230CF7D2854769
:1043C00017070020A307F7D297070020239607C6F8
:1043D00097400000E780C04117050020130545D134
:1043E000914597500000E780C0011345040299B33E
:1043F00093F70504FDC397C501009385E53017C504
:1044000001001305A5B497A00100E780A00617C519
:104410000100130565D797A00100E780A005294595
:1044200097A00100E780E0099707002083C747CCE9
:104430001307700A6386E7061307800A638CE70890
:104440001307600A6393E704930760F817070020D7
:104450002300F7CA9707002083D7E7C61707002075
:10446000A308F7C8A183170700202304F7C88547CE
:1044700017070020A303F7C8B1451705002013054F
:1044800025C797500000E780C0F797400000E780FD
:1044900020361345040497070020239607C259B914
:1044A000930770F8170700202304F7C4970700202C
:1044B00083D767C117070020A30CF7C2A183170792
:1044C00000202308F7C2854717070020A304F7C27E
:1044D000994565B7930780F8F1B793F7050801454B
:1044E000E38A07C497C501009385052217C501001B
:1044F0001305C5A597A00100E780C0F717C5010007
:10450000130505CA97A00100E780C0F6294597A0CA
:104510000100E78000FB9307A0F81707002023099C
:10452000F7BC9707002083D7A7BB17070020A3017C
:10453000F7BCA18317070020230DF7BA854717079B
:104540000020A308F7BA97070020239B07B89740DD
:104550000000E780E02917050020130565B99145A3
:1045600097500000E780E0E913450408E1B64111E7
:1045700022C497C501009385E5142A8417C501005C
:104580001305C59C06C697A00100E780A0EE4C402D
:1045900017C501001305453597A00100E78080EDA0
:1045A000294597A00100E780C0F103470400930765
:1045B000F00F631FF70297C501009385A51017C57B
:1045C00001001305A59897A00100E780A0EA4C40E0
:1045D00017C501001305453297A00100E78080E967
:1045E0002244B2402945410117A30100670063ED51
:1045F000B240224441018280B1C1411122C417C599
:1046000001001305A5942E8497C5010093858506A6
:1046100006C697A00100E780E0E5A28517C5010066
:104620001305C53897A00100E780C0E42244B240DA
:104630002945410117A301006700A3E882804111C9
:1046400022C426C22E84AA8497C5010093854503FF
:1046500017C501001305858F06C697A00100E780E6
:1046600060E117C501001305253597A00100E7801B
:1046700060E0294597A00100E780A0E497C501000C
:1046800093850500970700202396979A17C5010088
:104690001305C58B854497070020239B87989707B0
:1046A000002023989798971700202392870497A0BB
:1046B0000100E78020DC9715002083D5450317C54E
:1046C00001001305E52F97A00100E780A0DA294536
:1046D00097A00100E780E0DE97170020238697F07F
:1046E00097200000E780E0BE228597500000E78019
:1046F00040A1054597500000E780A0D997F7FF1F1C
:104700009387C7C7DC4703D70700C167FD1763124C
:10471000F7022244B7E70400B240924403A387059E
:1047200017F5FF1F034505101306000A85454101D3
:104730000283B2402244924441018280011122CC82
:1047400037E404005C5C06CE26CA354697C50100F6
:104750009385050917D50100130585CD829711E9C9
:1047600017C501001305458497A00100E78060E8A4
:1047700001A097F7FF1F9387A70B3EC4B7F507006B
:10478000856793870780814617F6FF1F1306C609C2
:10479000E10519453EC697E0FF1FE78020017C44F4
:1047A000194697F5FF1F9385250817050020130567
:1047B000A58A8297340017F6FF1F1306E60697C5F1
:1047C00001009385E55917C501001305E55A976067
:1047D0000000E7804030AA8421C197C5010093857D
:1047E000A5F117B501001305657697A00100E780D4
:1047F00060C8A68517C50100130585FF97A00100B5
:10480000E78040C7294597A00100E78080CBF240B0
:104810006244D2440561828097E00000E780809284
:1048200017C501001305C5F397500000E780602409
:1048300097A00000E780C0E697500100E780404B5A
:1048400017F5FF1F130505B097500100E780E0330F
:1048500017C501001305C5F197500100E780C04B53
:10486000AA8497600000E780A08A97000100E78093
:10487000202397800100E78040BC97700000E7800C
:10488000E0E297600000E780A00097300100E78039
:1048900080E497C50100938525E617B5010013054F
:1048A000E56A99C897A00100E780C0BCA68517C536
:1048B0000100130525F699B797A00100E78080BB9A
:1048C00017C50100130545F797A00100E78080BADE
:1048D000294597A00100E780C0BE97300100E7801E
:1048E00060C097F00000E78020DF630F051085456A
:1048F0003705040097200000E780202F97C50100AE
:10490000938585DF17B501001305456497A0010065
:10491000E78040B617C50100130585F397A0010095
:10492000E78040B5294597A00100E78080B997F757
:10493000FF1F9387679483D707001717002023185A
:10494000F7DA8547171700202300F7CA97200000E1
:10495000E78000B797200000E780A0971715002098
:104960000355E5D897400000E780A079970700201D
:1049700083C75787ADEBA3030100832744171306B2
:104980007100854513055030829797C501009385C6
:10499000A5D617B501001305655B97A00100E78058
:1049A00060AD17C501001305E5EC97A00100E78095
:1049B00060AC294597A00100E780A0B097C5010031
:1049C000938585D317B501001305455897A00100BD
:1049D000E78040AA17C501001305C5EF97A00100A5
:1049E000E78040A905B597C501009385E5D017B5C7
:1049F00001001305A55597A00100E780A0A717C5E2
:104A000001001305A5EA55B797C501009385C5CEEA
:104A100017B501001305855397A00100E78080A515
:104A200017C501001305C5FA97A00100E78080A40F
:104A3000294597A00100E780C0A8014597500000D4
:104A4000E78020A5A5BF411122C437E404008327D5
:104A5000041A06C6829797400000E780A073832758
:104A6000040817F5FFFF1305055B829797F7FF1FF3
:104A7000238AA7DA17F5FF1F13054590974000001A
:104A8000E780A0092244B2404101170300006700FB
:104A900023CBB7E70400FC471171A2DDCAD986DF3A
:104AA000A6DBCED72E8432892E86AA8517F5FF1F66
:104AB00013050564829717F7FF1F13076763834782
:104AC0000700930680029387E70793F7F70FE3EC5D
:104AD000F610BA898A0717B7010013076750BA970B
:104AE0009C43BA9782878D4797C50100938505C37C
:104AF00017B5010013058545630FF40097A0010069
:104B0000E780409717C501001305058097A00100B5
:104B1000E7804096BDA497A00100E780A09517B557
:104B200001001305E57F97A00100E780A0942945C7
:104B300097A00100E780E098930720F8114697F5C9
:104B4000FF1F9385E55A4A8517F7FF1F2302F75A7F
:104B500097F7FF1FA38F075897F0FFFFE7800034F8
:104B60002A841DC997C50100938545BB17B501006F
:104B70001305C53D97A00100E780C08FA28517B53A
:104B800001001305A57D97A00100E780A08E2945AF
:104B900097A00100E780E09297C50100938505B8D2
:104BA00017B501001305853A97A00100E780808CB6
:104BB00017B501001305C57B97A00100E780808B26
:104BC000294597A00100E780C08F4165930730FA1F
:104BD000054697F5FF1F9385A5517D1517F7FF1F14
:104BE0002308F75097F0FFFFE780402B2A841DC968
:104BF00097C50100938585B217B5010013050535EA
:104C000097A00100E7800087A28517B50100130572
:104C1000E57497A00100E780E085294597A0010091
:104C2000E780208AB7E70400BC4F0566130606C874
:104C3000A14517F5FF1F0345E5BE8297FE506E5450
:104C4000DE544E59BE591161828091476303F402CC
:104C500097C50100938585AC17B501001305052F95
:104C600097A00100E780008117B501001305857347
:104C700071BDB7E70400FC4F914517F5FF1F0345D1
:104C800065BA829797C50100938545A917B50100BC
:104C90001305C52B97900100E780C07D17B5010073
:104CA0001305057297900100E780C07C294597A005
:104CB0000100E780008197400000E78060B39145E4
:104CC00035A485476303F40297C50100938505A5C4
:104CD00017B501001305852797900100E7808079BB
:104CE00017B501001305456F15B597F7FF1F2393FF
:104CF0002737B7E704000566BC4F130606C8C14551
:104D00000DBF8D476303F40297C50100938505A18C
:104D100017B501001305852397900100E780807582
:104D200017B501001305056DD5B3930740F811467B
:104D300097F5FF1F9385C53B4A8517F7FF1F23098A
:104D4000F73A97F7FF1FA386073A97F0FFFFE78030
:104D5000E0142A84E30405EE97C501009385059CC1
:104D600017B501001305851E97900100E78080703C
:104D7000A28517B501001305655E97900100E780D5
:104D8000606F294597900100E780A07345BD91476A
:104D9000E31CF4F6B7E70400FC4F9305000217F597
:104DA000FF1F034525A8829797C5010093850597A6
:104DB00017B501001305851997900100E780806BF6
:104DC00017B5010013058564F1BD894763E38702C8
:104DD00097C501009385859417B501001305051744
:104DE00097900100E780006917B50100130545633E
:104DF00031BB97F4FF1F83C4C42F97F7FF1F83C7EE
:104E0000372F97C5010093856591A20417B501005E
:104E10001305C513DD8C97900100E780A065A2857E
:104E200017B501001305056197900100E7808064C4
:104E3000C204294597900100E780A068C1849305CA
:104E4000D4FF93960401C1824A8693F5F50F17F5B6
:104E5000FF1F1305152A97200000E780C0DCE35FE1
:104E600090DC930750F817F7FF1F2303F72883C739
:104E70003900228697F5FF1F9385852785074A8588
:104E800017F7FF1FA307F72697F0FFFFE780000142
:104E90002A84E30505DA97C501009385258817B5AF
:104EA00001001305A50A97900100E780A05CA28588
:104EB00017C50100130585AEC9B5894763E38702AD
:104EC00097C501009385858517B501001305050871
:104ED00097900100E780005A17B501001305455768
:104EE00035B197400000E780A090A28517F5FF1F1D
:104EF0001305052097400000E780A05081B38D473F
:104F00006303F40297C501009385458117B501003D
:104F10001305C50397900100E780C05517B5010040
:104F20001305C554E5B6B76602000146B775020021
:104F3000054597E0FF1FE7806087930760F817F744
:104F4000FF1F2307F71A97F7FF1FA384071A93077A
:104F5000000617F7FF1F230FF718894717F7FF1FE2
:104F6000A30AF71897F7FF1F2387071897F7FF1F64
:104F7000A3830718C14717F7FF1F230FF7169307DF
:104F800020F917F7FF1FA309F716314697F7FF1F00
:104F9000A385A71697F5FF1F938585154A8597F773
:104FA000FF1F238C071497F0FFFFE78020EF2A8470
:104FB000E30605C897B501009385457617B501004E
:104FC0001305C5F897900100E780C04AA28517B580
:104FD00001001305254B55B3B1476303F40297B5A0
:104FE00001009385A57317B50100130525F6979069
:104FF0000100E780204817B501001305654A39B65E
:10500000B7E70400FC4F9305000417F5FF1F0345A5
:105010006581829797300000E780807DB145F9B5C2
:10502000914763E3870297B501009385256F17B514
:1050300001001305A5F197900100E780A04317B583
:1050400001001305A547D9B497F4FF1F83C4840A50
:1050500097F7FF1F83C7F709A204DD8C8E04B7778B
:1050600002006D14BE942286A68517B501001305B3
:10507000254697900100E780E03FB7E70400FC4732
:10508000228697F5FF1F9385F506280082979316D1
:105090000401C1823000A685094597D0FF1FE78033
:1050A000E0702A8409C917B50100130525449790BB
:1050B0000100E7800054930770F8194697F5FF1F29
:1050C000938505034A8517F7FF1F2303F70297F718
:1050D000FF1FA381870297F0FFFFE78020DC2A846F
:1050E000E30E05B497B501009385456317B501003C
:1050F0001305C5E597900100E780C037A28517B575
:1051000001001305A53F95B99947630BF41297B5B4
:1051100001009385A56017B50100130525E397905D
:105120000100E780203517B501001305A53EF9BA47
:10513000914763E3870297B501009385255E17B514
:1051400001001305A5E097900100E780A03217B594
:1051500001001305A53D5DBA97F4FF1F83C484F9D0
:1051600097F7FF1F83C7F7F8A204DD8C8E04B7778B
:1051700002006D14BE942286A68517B501001305A2
:10518000253C97900100E780E02EB7E70400FC473C
:10519000228697F5FF1F9385F5F5280082979316D1
:1051A0000401C1823000A6850D4597D0FF1FE7801E
:1051B000E05F2A8409C917B501001305253A9790C5
:1051C0000100E7800043930780F8194697F5FF1F19
:1051D000938505F24A8517F7FF1F230BF7F097F722
:1051E000FF1FA38987F097F0FFFFE78020CB2A8479
:1051F000E30605A497B501009385455217B5010054
:105200001305C5D497900100E780C026A28517B585
:1052100001001305E53595B699476303F40297B588
:1052200001009385A54F17B50100130525D297906E
:105230000100E780202417B501001305E534F9B01B
:10524000B7E70400FC4F9305000417E5FF1F034573
:10525000655D829797300000E7808059994579B164
:105260008D476303F40297B501009385254B17B56D
:1052700001001305A5CD97900100E780A01F17B589
:1052800001001305E53159B017B50100130545328A
:1052900097900100E780E0351305C01297D0FF1FFB
:1052A000E780200A014597E0FFFFE780A0DB0D457E
:1052B00097100000E780009F294597D0FF1FE780E7
:1052C000400897D0FF1FE780A0F88DBA9947630385
:1052D000F40297B501009385654417B501001305E5
:1052E000E5C697900100E780E01817B501001305A7
:1052F000E52C29B817F7FF1F0347D7DF97F7FF1FE4
:1053000083C747DF22075D8F9166BA96C206116692
:10531000C1821306F6EF8D476365D60297E7FF1F3C
:105320009387C7059C4B17F6FF1F034696DC9386B1
:10533000C7002DC203D6070069CA8907E39CD7FEC0
:1053400089471307A0F8114697F5FF1F938545DAA3
:105350004A8597F6FF1F238DE6D817F7FF1FA30A8C
:10536000F7D897F0FFFFE78060B32A84E308058C45
:1053700097B501009385853A17B50100130505BD62
:1053800097900100E780000FA28517B50100130573
:105390002524E5B203D60700630EE60A8907E39BDE
:1053A000F6FE8D4779BF91476304F40297B501007B
:1053B0009385C53617B50100130545B997900100CF
:1053C000E780400B17B50100130505226FF00FF4BD
:1053D000B7E70400FC4F9305000817E5FF1F0345DE
:1053E00065448297C9B897B501009385253317B5F1
:1053F00001001305A5B597900100E780A00717B538
:1054000001001305E51F6FF06FF02390E70017E52B
:10541000FF1F1305A5F697200100E780203297B5FE
:1054200001009385A52F17B50100130525B29790AC
:105430000100E780200417B501001305651D979052
:105440000100E7802003294597900100E78060076D
:105450008147C5BD2390070017E5FF1F130505F21F
:1054600097200100E780802D97B501009385052BDB
:1054700017B50100130585AD97900100E78080FF07
:1054800017B501001305451A5DBF411122C406C6B8
:10549000834705002A849DC797B501009385C523DE
:1054A00017B50100130585AA97900100E78080FCDD
:1054B0004C4017B501001305A55497900100E780F3
:1054C00060FBE1A05841B707CF009387777D631D4C
:1054D000F70697B501009385252017B50100130540
:1054E000E5A697900100E780E0F81C448356E400AD
:1054F0008355C40003C6070017B501001305C55145
:1055000097900100E78000F7294597900100E78018
:1055100040FB0357E4009707002083D7471D63092A
:10552000F7008355C400084497E0FFFFE78020C8D8
:105530000356E4008355C40008442244B2404101AC
:1055400017F3FFFF67002355B707CC009387777DDC
:105550006315F70497B501009385051817B5010089
:105560001305C59E97900100E780C0F01C44835648
:10557000E4008355C40003C6070017B501001305F6
:10558000A54997900100E780E0EE2244B24029450A
:105590004101179301006700C3F2B707CE0093875C
:1055A000777D6304F70297B501009385E51217B57F
:1055B00001001305A59997900100E780A0EB4C40EE
:1055C00017B501001305853ACDBDB2402244410113
:1055D0008280B7E70400FC4741112E8606C622C42C
:1055E00026C24AC02E842A89AA8517F5FF1F1305F3
:1055F00025B0829797B501009385051417B5010072
:105600001305C59497900100E780C0E697F5FF1F4A
:1056100083C505AE17B50100130505BA97900100C3
:10562000E78040E5294597900100E78080E997F4FD
:10563000FF1F9384E4AB83C70400414793870706A9
:1056400093F7F70F636AF75C17B70100130787A397
:105650008A07BA979C43BA9782879D476307F402EB
:1056600097B501009385450D17B501001305058E0B
:1056700097900100E78000E017B50100130545B4DD
:1056800097900100E78000DFADAC97F7FF1F83C75D
:1056900037A6DDCB17F7FF1F0347B7A597F7FF1F07
:1056A00083C727A522075D8F97F7FF1F83C787A4AE
:1056B000C2075D8F97F7FF1F83C7D7A3E207D98F74
:1056C00017F7FF1F2324F7A083C7640097B50100D5
:1056D0009385850617B501001305458717F7FF1F4A
:1056E0002305F79E97900100E780C0D897F7FF1F2A
:1056F0009387C79D8C4317F6FF1F0346069D17B57A
:1057000001001305A5AD97900100E780A0D62945BB
:1057100097900100E780E0DA97F7FF1FA38A079CC4
:105720002244B24092440249930700F817F7FF1F42
:105730002300F79C9D4517F5FF1F1305659B41014D
:10574000174300006700E3CB97600000E780008309
:1057500097F7FF1F238FA7989357850017F7FF1F11
:10576000A309F798935705012A8417F7FF1F23030E
:10577000F79893578501014517F7FF1FA30CF7967C
:1057800097600000E780408097F7FF1F2385A7966A
:1057900097B50100938545FA17A501001305057B10
:1057A00097900100E78000CD17F6FF1F0346A694EF
:1057B000A28517B501001305E5A3B1B7CD47630373
:1057C000F40297B50100938525F717A5010013058D
:1057D000E57797900100E780E0C917B50100130550
:1057E000E5A279BD37E404007C44414697F5FF1FEC
:1057F0009385159017F5FF1F1305858D829717F573
:10580000FF1F1305E58C97100000E78080C49710F8
:105810000000E78000AC97F7FF1F83C7878E17F75C
:10582000FF1F0347F78DA20703238405D98F17F7BE
:10583000FF1F231BF7881306000A89452244B24044
:105840009244024917E5FF1F0345C5FD410102834C
:105850008D476303F40297B501009385E5ED17A525
:1058600001001305A56E97900100E780A0C017B551
:105870000100130565A929B517F4FF1F03446487C8
:1058800097F7FF1F83C7D78697B501009385C5EAB1
:10589000220417A501001305656B5D8C979001002C
:1058A000E78040BDA28517B501001305A597979025
:1058B0000100E78020BC294597900100E78060C087
:1058C0000D4697F5FF1F9385A582228597E0FFFF80
:1058D000E780C05CAA8421C197B501009385C5E526
:1058E00017A501001305856697900100E78080B831
:1058F000A68517B501001305259497900100E78050
:1059000060B72244B24092440249294541011793AD
:105910000100670003BB97E7FF1F239D8772B7E76E
:105920000400116603A38705130606E8914539B7FD
:105930008D476303F40297B501009385E5DF17A552
:1059400001001305A56097900100E780A0B217B58C
:105950000100130525AA2DB317E4FF1F0344647942
:1059600097E7FF1F83C7D77897B501009385C5DCFC
:10597000220417A501001305655D5D8C9790010059
:10598000E78040AFA28517B501001305258C9790DD
:105990000100E78020AE294597900100E78060B2C2
:1059A0000D4697E5FF1F9385A574228597E0FFFFBD
:1059B000E780C04EAA841DC197B501009385C5D765
:1059C00017A501001305855897900100E78080AA6C
:1059D000A68517B501001305A58805B797E7FF1F32
:1059E000239C8764B7E70400116603A387051306A9
:1059F00006E89305000299B5894763E3870297B5E6
:105A00000100938565D317A50100130525549790D0
:105A10000100E78020A617B50100130565A08DB130
:105A200097E4FF1F83C4E46C97E7FF1F83C7576C9D
:105A300097B50100938545D0A20417A50100130571
:105A4000E550DD8C97900100E780C0A2A68517B5D0
:105A500001001305658297900100E780A0A1294508
:105A600097900100E780E0A5228697E5FF1F9385C8
:105A70002568268597E0FFFFE78040422A84630E71
:105A8000051A97B50100938525CB17A501001305CD
:105A9000E54B97900100E780E09DA28517A50100E6
:105AA0001305C57E99BD854763F98718834519009D
:105AB0002244B24092440249B335B00097E7FF1F39
:105AC0002384B75A17A501001305857D410117935B
:105AD00001006700239AA2852244B24092444A857D
:105AE000024941011703000067000322994763033D
:105AF000F40297B50100938525C417A5010013058D
:105B0000E54497900100E780E09617B50100130582
:105B1000E5AABDB617E4FF1F0344A45D97E7FF1F86
:105B200083C7175D97B50100938505C1220417A5AA
:105B300001001305A5415D8C97900100E7808093DB
:105B4000A28517A501001305257797900100E7802E
:105B50006092294597900100E780A096194697E545
:105B6000FF1F9385E558228597E0FFFFE78000330C
:105B7000AA841DC197B50100938505BC17A5010036
:105B80001305C53C97900100E780C08EA68517A538
:105B900001001305657395B397E7FF1F23928754A0
:105BA000B7E70400116603A38705130606E893050B
:105BB000000869B1854797B501009385E5B717A53A
:105BC00001001305A538630BF40097900100E780EE
:105BD000608A17A50100130565705DB497900100F8
:105BE000E780408917A501001305C5709790010053
:105BF000E7804088294597900100E780808C224407
:105C0000B2409244024997E7FF1F239F074A410190
:105C1000175300006700032797B501009385C5B1AE
:105C200017A501001305853297900100E780808455
:105C300017B501001305C59CA1B4B240224492449B
:105C4000024941018280411106C622C497E0FFFF4C
:105C5000E780C0249377F50FA1C32A8497B501008C
:105C6000938505AF17A501001305452E97900100F8
:105C7000E78040809375F40F17B50100130505D236
:105C800097800100E780007F2244B240294541010E
:105C9000179301006700E382B240224441018280F1
:105CA000411122C491462A8417E6FF1F130686522B
:105CB0009D652D4506C697D0FF1FE78020AFB7F73B
:105CC000070003C70701A5476313F70001A0930668
:105CD000001001469D65254597D0FF1FE78000AD68
:105CE00097E7FF1F2388874E2244B240914617E66C
:105CF000FF1F1306264E9D652945410117D3FF1F3F
:105D00006700C3AA5171CAD137E904008327C904C7
:105D1000A2D52E8686D7A6D32E84AA8517E5FF1F87
:105D20001305053D829797E7FF1F83C7673C13075D
:105D3000700A6387E710636CF7001307600A6384D7
:105D4000E704BE502E549E540E596D618280130795
:105D5000800A6388E7161307900AE394E7FE8D47ED
:105D60006309F41C97B50100938585D617A501003A
:105D70001305C51D97800100E780C06F17B50100AE
:105D8000130545D225A08D47630CF40297B5010099
:105D9000938505D417A501001305451B97800100C5
:105DA000E780406D17B50100130505C99780010014
:105DB000E780406C294597800100E780807051B7EB
:105DC000854717B501001305E5C817E7FF1F230D29
:105DD000F72897900100E780C081B7750200B76689
:105DE00002000146054597D0FF1FE780209C9307DE
:105DF00060F817E7FF1F230DF72E97E7FF1FA38A11
:105E0000072E9307002617E7FF1F2325F72EE577B8
:105E10009387072117E7FF1F2310F72EB14597E758
:105E2000FF1F238C072C97E7FF1FA388A72C17E5DC
:105E3000FF1F1305E52B97300000E780805C11B74A
:105E4000914763E3870297B50100938565C817A55D
:105E500001001305A50F97800100E780A06117B529
:105E60000100130525C199B797E4FF1F83C4842857
:105E700097E7FF1F83C7F727A204DD8C8327C90498
:105E80006D14228697E5FF1F9385D52628008297FB
:105E90008E0493160401B7750200C1823000A695E6
:105EA000094597D0FF1FE7806090930770F817E7C8
:105EB000FF1F230FF722994597E7FF1FA38CA72207
:105EC000BDB7914763E3870297B50100938545C04D
:105ED00017A501001305850797800100E780805909
:105EE00017B50100130585BAD1B597E4FF1F83C428
:105EF000642097E7FF1F83C7D71FA204DD8C832789
:105F0000C9046D14228697E5FF1F9385B51E2800EE
:105F100082978E0493160401B7750200C182300087
:105F2000A6950D4597D0FF1FE7804088930780F81E
:105F3000BDBF17B50100130525B897800100E780A4
:105F4000406B1305C01297C0FF1FE780803F0145DB
:105F500097D0FFFFE78000110D4597000000E78014
:105F600060D4294597C0FF1FE780A03D97C0FF1F61
:105F7000E780002EF9B341114AC097F6FF1F83D680
:105F80000677328917D6FF1F0356664122C426C200
:105F900006C62A84AE8497000000E780C05F35C142
:105FA0002DC0994763FF97048347140003470400FB
:105FB000A207D98F13978700A183D98FC2073167B2
:105FC000C1831307C755639EE70297D7FF1F83D787
:105FD000073DA301F400A1832302F40097F7FF1FFC
:105FE00083D7E77091C7A302F400A1832303F400D1
:105FF000A68517B501001305A5B197800100E780BC
:10600000604797F7FF1F83C7275EB9CF97D5FF1F5C
:1060100083D5E53817B50100130545B19780010018
:10602000E78040452686A28517D5FF1F03552537F3
:1060300097000000E78060C16301090497E7FF1F34
:1060400083C7471A9DCB95C897E7FF1F83C7C70132
:106050008DE722852244B2400249A685924441013F
:10606000173300006700E33917B50100130505ADCC
:1060700097800100E780E057C1B7B24022449244C4
:10608000024941018280834755008345450017B589
:1060900001001305A5A6A207DD8D17830100670087
:1060A000633D17B50100130565A417830100670060
:1060B00043548D4763FBB70A011126CA06CE22CC92
:1060C0000344350097E4FF1F83C4D41197B5010042
:1060D000938585A7B337800017E7FF1FA304F71048
:1060E00009C497B501009385E5A617B5010013050E
:1060F000E5A697800100E780E03797E7FF1F83C799
:10610000770E6386970097000000E780802697E768
:10611000FF1F83C7370D8DC785472306F100B7E7FB
:10612000040083A7471770008545130550308297F8
:1061300017B50100130585A397800100E780604B28
:106140009967938757EE2316F100680085479145BC
:10615000A30781002307F10097300000E780602A41
:10616000F2406244D244056182808280894763F7AD
:10617000B708011122CC06CE26CA834425008547E4
:106180002A84639DF404914763F5B70403454500F1
:106190008347340022055D8D97D7FF1F2391A720E9
:1061A00097000000E78000489967938767EE231403
:1061B000F1008347340023059100A305F1008347D4
:1061C0004400954528002306F10097300000E78041
:1061D0004023F2406244D24405618280FDF8996711
:1061E000938767EE2314F10097D7FF1F83D7271BF0
:1061F000A305F10023050100A183E1B7828001110D
:10620000996722CCD51717F4FF1F1304E43D23141C
:10621000F1008347040026CA97F4FF1F9384244D9E
:106220002305F10083D7040028009545A305F1005C
:10623000A18306CE2306F10097300000E780601CA2
:1062400003D604008345040017B5010013058593A8
:1062500097800100E7800022F2406244D244056149
:1062600082809D677971D9172316F10097F7FF1F78
:1062700083C7873706D62307F100A9C3B7E7040011
:10628000FC47414697E5FF1F938585E41305F10020
:1062900082976800CD4597300000E780801697F51B
:1062A000FF1F83C5653417B501001305A5909780BE
:1062B0000100E780201CB25045618280B7E70400EE
:1062C000BC47414681451305F1008297D9B7B767AE
:1062D00002045D71938757AA3EC08567938707A024
:1062E0002312F10097F7FF1F9387073083C707003A
:1062F000A2C4A30301002303F10097F7FF1F9387B4
:10630000073F83D7070037E4040086C62314F10053
:1063100097D7FF1F9387A70883D7070041466800D8
:106320002315F1007C4497E5FF1F938565DA82977A
:10633000F1450A8597000000E780E021231EA100B7
:106340007C448A850810794682973C441305E10312
:10635000094681458297101093050002014597D0A8
:10636000FFFFE780A036B640264461618280B7C750
:10637000A55A01119387C7333EC497E7FF1F83C710
:1063800077E63EC6B7F7070003C7070106CE22CC63
:10639000A5476313F70001A01164930504F0930669
:1063A00000100146254597C0FF1FE78020403000C0
:1063B000930504F0A146294597C0FF1FE780003FE1
:1063C00097E5FF1F83C515E217B501001305458F3B
:1063D00097800100E780000AF240624405618280F4
:1063E00001119165A1463000938505F02D4506CE3B
:1063F00097C0FF1FE780803B2247B7C7A55A938706
:10640000C7336314F702B24517A501001305857E53
:10641000B335B00097E7FF1FA386B7DC9780010074
:10642000E7804005F24005618280814517A50100A3
:106430001305857E97E7FF1FA38607DA9780010083
:10644000E780400397000000E780A0F2E1BFB7C7F4
:10645000A55A79719387F7353EC6B7E70400FC4724
:10646000AA8506D622D4414608088297B7F70700C6
:1064700003C70701A5476313F70001A01164930543
:1064800004E8930600100146254597C0FF1FE780EA
:10649000E0317000930504E8D146294597C0FF1FFD
:1064A000E780C03017B501001305458597800100CE
:1064B000E7802014B2502254456182807971916541
:1064C000D1467000938505E82D4506D697C0FF1F7D
:1064D000E780C02D3247B7C7A55A9387F73517A570
:1064E00001001305657B6310F702B7E70400FC4762
:1064F00017E5FF1F1305C5BD41460C08829717A578
:1065000001001305657797800100E780800EB25087
:1065100045618280B7F7070003C70701A5476313EA
:10652000F70001A091654111930600100146938583
:1065300005E8254506C697C0FF1FE7802027B24023
:1065400017A5010013054569410117830100670084
:10655000430AC16769768146FD1705061397060150
:1065600041836364B7003E8582803307D5000347CB
:106570000700B98F214713F81700858363050800CA
:10658000B18FC207C1837D171377F70F6DF78506AB
:10659000F1B741C5A547054763F2B7088347150022
:1065A000034705003168A207D98F13978700A1839D
:1065B000D98FC207C1831308C855054763900707E1
:1065C000411106C622C426C203442500914763F048
:1065D00087049307540063ECF502A301C5002182F0
:1065E0002302C5009304340091C6A302D500A18202
:1065F0002303D5002A84A68597000000E780A0F534
:1066000026942300A4002181A300A4000147B240E6
:10661000224492443A854101828005473A8582802E
:10662000B7C7A55A01119387E7343EC42AC6B7F706
:10663000070003C7070106CE22CC26CAA54763136D
:10664000F70001A091642A84938504EE930600105C
:106650000146254597C0FF1FE78040153000A14641
:10666000938504EE294597C0FF1FE7802014A2857B
:1066700017A501001305C56697800100E78080DF3C
:1066800097000000E780E0C4F2406244D244056114
:10669000828001119165A1463000938505EE2D455C
:1066A00006CE97C0FF1FE78060102247B7C7A55AE4
:1066B0009387E7346318F702B24517A50100130565
:1066C000A55797D7FF1F239CB7CCC205C1819780E0
:1066D0000100E78020DA97000000E78080BFF240E9
:1066E00005618280D147D14517A501001305C55624
:1066F00017D7FF1F2315F7CA97800100E78080D7BF
:1067000017D5FF1F0355A5C997000000E78080F14A
:10671000F9B7011126CA06CE22CC93F71500AE8434
:106720008DCBAD67371700409387A7AA1CC3B7E787
:106730000400BC4F13060019854517D5FF1F0345FC
:10674000E5C5829713C51400F2406244D244056146
:10675000828093F725006386071897A5010093852B
:10676000E55D2D46480097800100E78040C597F51C
:10677000FF1F83C5A5F7854793C4240063E5B704CD
:106780009DC9854517F5FF1F130545E697200000B5
:10679000E78060AA97E7FF1F83C7C7A489CF97F553
:1067A000FF1F83C5A5F417F5FF1F130525E49730D8
:1067B0000000E78000C51395040197F7FF1F2387AA
:1067C00007F2418151B717F4FF1F034424E297F702
:1067D000FF1F83C7B7E122045D8CAD67C2059387B5
:1067E000B755C181630DF40C63E18704A9679387F2
:1067F000A755630FF40C17F5FF1F130525DF97202E
:106800000000E78040A397E7FF1F83C7A79DD1CF74
:1068100097F5FF1F83C585ED17F5FF1F130505DDF0
:1068200097300000E780E0BD49A0B1679387C75566
:106830006302F404B5679387D755E31EF4FA17F59E
:10684000FF1F1305A5DA97300000E78080BB97F59E
:10685000FF1F83C5A5E9894763F9B704F915C20588
:10686000C18117F5FF1F130585D897200000E78029
:10687000809C25A8054617F5FF1F130525D797F01F
:10688000FFFFE780806F97F7FF1F83C7E7D591EF82
:10689000480097800100E78080DE93150501C181E3
:1068A000480097D0FFFFE7808090A28517A50100E0
:1068B0001305C54697800100E780C0BBEDBD17F505
:1068C000FF1F1305A5D297F0FFFFE780007CF1BF03
:1068D00017F5FF1F130585D197F0FFFFE780A07C18
:1068E000E9B793F745000145E38007E617A50100E6
:1068F0001305054497800100E780A0CF9730000082
:10690000E78040C413C5440081B5411122C437E477
:1069100004005C5C06C6354697A50100938545ECEE
:1069200017B501001305C5B0829711E917A501003D
:106930001305854197800100E780A0CB01A0832744
:10694000041C82972A84054597B00000E780E07E0A
:1069500097600100E780000497600100E78000D99C
:1069600097B00000E78060902285B2402244410148
:1069700082801567B71700401307575598C3D8434F
:106980009D66558FD8C3D843FD76758FD8C3D8433D
:106990001367F70FD8C335671307C7CC98C3828036
:1069A0004111054506C622C426C297C0FFFFE780F5
:1069B00040551305800497B0FF1FE780406F757541
:1069C00085457D1597C0FFFFE780E03E7D758545D5
:1069D0001305F53697C0FFFFE780404837140040A5
:1069E0008327840A8D451305002093E7072023247D
:1069F000F40A97C0FFFFE780003CB7E4040097D09B
:106A0000FFFFE7804081C85897800100E78060BEA3
:106A100017B501001305C5A197800100E78060BD8F
:106A20008327840C8545414593E707082324F40C0C
:106A300097C0FFFFE78080428D451305000897C08F
:106A4000FFFFE780A04197C0FFFFE780806E014510
:106A500097C0FFFFE780607185450545894717F7B7
:106A6000FF1F2307F7C897C0FFFFE780A071370714
:106A70000004B7E700E023A0E71097D0FFFFE7800E
:106A8000400397D0FFFFE780001797000000E780E2
:106A900000E897000000E780E09497000000E7809E
:106AA00080BF97E0FFFFE78040FA97000000E78093
:106AB000601097000000E780600B83A704081705AB
:106AC0000000130545C5829797D7FF1F2388A78C21
:106AD000BC4C130600648545829797000000E78050
:106AE00080E997C0FF1FE780A09001458280B7F73B
:106AF000070003C70701A547AE866316F700939703
:106B0000450191C301A0AA850146254517C3FF1F72
:106B10006700C3C94111B2862E86AA852D4506C6D7
:106B200097C0FF1FE78080C8B240014541018280C5
:106B30009307000463E8C7021D71A2CC2A840808E9
:106B400086CE32C697800100E7806087B246100883
:106B5000A285294597C0FF1FE78040C5F6406644DF
:106B6000256182803955828041110D658D4506C6AB
:106B700097C0FFFFE7802024B71700408D6623A64B
:106B8000D70A17F5FF1F1305E5B61387C70A9387C2
:106B9000870A1CC15CC5856689675CC958C114C574
:106BA00018C9B7E70400B24003A3871E410102835E
:106BB00097F7FF1F83C787B599EF411106C6971056
:106BC0000000E7806061B240854717F7FF1F230F81
:106BD000F7B241018280828011C589C517C3FFFFCA
:106BE0006700E35C8280411126C2AE848D4522C4D9
:106BF00006C62A8497C0FFFFE7804026B7170040EB
:106C000099C803A5C70C418D23A6A70CB240224406
:106C100092444101828003A5870C418D23A4A70CD7
:106C2000F5B78347050003471500A207D98FC207B0
:106C30006177C18713072720639AE7008345250002
:106C40003705040017030000670023FA828017F657
:106C5000FF1F1306E6AB8147B2861303F00FA94866
:106C60003308F6000348080013F7F70F6307A80C72
:106C7000630668008507E39517FF2947B387E60099
:106C80002380A70097F7FF1F938747A95DA84111AD
:106C900013D765001347170006C693F63500058B1A
:106CA000954791CA054699476387C60009469D479F
:106CB0006383C600A14713F645003336C00093F640
:106CC0008503050685C2A145638BB604E145638A49
:106CD000B604930580026388B6049305800363932A
:106CE000B600914697F5FF1F238FF5C897F5FF1F54
:106CF000238AC5C897F5FF1FA386D5C8BE8517A5EB
:106D000001001305E50D97700100E780A076B24001
:106D1000854717F7FF1FA308F7C641018280854604
:106D2000D1B78946C1B78D4675BF17A501001305B8
:106D3000A50D177301006700E37317F7FF1F130713
:106D4000E79DBA972380B700E147E302F5F4930784
:106D50007002E30CF5FC82802A87238005008147BE
:106D600017F5FF1F1305C59A1308F00F2946B30640
:106D7000F50083C606006396E60297F6FF1F93862A
:106D8000E699B69783C7070005452380F500994724
:106D9000636EF7029D4763FDE700E147630DF7006F
:106DA0008280638506018507E393C7FC0145C5B76B
:106DB000238005008280B737004003C7370083C7B0
:106DC000050093F70704D98F2380F500828079713D
:106DD00026D24AD097F4FF1F83C4C4CC17F9FF1FF3
:106DE000130989CB06D622D44ECE52CC56CA5AC8E5
:106DF000B307990083C7070093F7F70FA5C79387D9
:106E0000140093F7F70F0D476361F70C17F7FF1F97
:106E1000230AF7C897F7FF1F938787C8A69783C7EA
:106E200007001307100293F7F703638FE7286363E4
:106E3000F70A054463808720E389076E0947638961
:106E4000E71413070002E38EE758B7E700E03707BF
:106E5000400023A0E71801000100CA942380040029
:106E600023A0E710B787004003C76700058BE30F37
:106E7000077897F6FF1F83C606C30547E39AE676B1
:106E800029472381E70209472383E7022385E70295
:106E900097F7FF1FA38A07AE97F7FF1FA38507C0C9
:106EA000B7870040A381070017F7FF1FA30007AEB5
:106EB00005472383E700B250225492540259F24905
:106EC000624AD24A424B4561828097F7FF1F238B6B
:106ED00007BC89B7130730026386E70A63E6E71445
:106EE00013074002638AE70813070003E39FE7F4F0
:106EF00097F7FF1F938787BAA69703C70700A14795
:106F00001377F70FE31AF71C17FAFF1F130ACA814A
:106F100083476A0097F6FF1F238EF6A497F7FF1F9B
:106F200083C7F78091C7FD5797F6FF1F2384F6A408
:106F300097E5FF1F83C5557F97F7FF1FA38CB7A267
:106F400097E7FF1F83C7477E93F90708930600045E
:106F500093F707066393D7529307A009638DF51A39
:106F600063EAB7169307F005638AF54E9307500955
:106F70006388F52E014479ABFD5717F7FF1F230AED
:106F8000F79EE1B5FD5717F7FF1F2303F79E75BD69
:106F900017A501001305C5F897700100E78060652B
:106FA00097F7FF1F938787AFA69703C40700814910
:106FB00017FAFF1F130ACA8F1374F40F97AA010060
:106FC000938A8AF663C78904294597700100E78090
:106FD000404F854717F7FF1FA30AF78C17F7FF1FCE
:106FE0002307878C17F7FF1F2300F79A37E700E086
:106FF000B70640002320D718010001003786004063
:107000008347A60293F7370F2305F6022320D710F4
:107010002DBDB3073A0183C50700568585099770D2
:107020000100E780204579BF854717F7FF1F230F31
:10703000F78621BD17A50100130585EE97700100A5
:10704000E780205B97F7FF1F938747A5A69703C4A8
:107050000700814917EAFF1F130A4A791374F40FD6
:1070600097AA0100938A4AEC63C589042945977061
:107070000100E7800045854717E7FF1FA306F77665
:1070800017E7FF1F2303877617F7FF1F230EF78EDF
:1070900037E700E0B70640002320D71801000100C1
:1070A000378600408347660293F7370F2303F602C3
:1070B000B1BFB3073A0183C50700568585099770AC
:1070C0000100E780203B4DB7854717E7FF1F230DE1
:1070D000F770A5BB9307400A638DF5349307200B27
:1070E0006388F5369307100AE396F5E883072A00CC
:1070F000014463D1074297E7FF1F83C7176393F6E5
:107100003700638E061A0546638EC62209466399C8
:10711000C61A1D4775A217E5FF1F03450561C9473C
:1071200017EAFF1F034A7A6097E5FF1F83C50560D2
:1071300017E4FF1F0344945F6319F510CD476316EE
:10714000FA1093077008639CF5021307300FB71706
:107150000E006308E4001307900DB7B70400631432
:10716000E40817F7FF1F232DF780BE8517A5010040
:10717000130505DC97700100E780C02FE5BB93077E
:107180008008639DF50033048040B7774600137490
:10719000F40F938787CDB3D78702E1B793079008A1
:1071A000639AF5003304804091671374F40F93875A
:1071B000C766D5B79307A008639BF50033048040EA
:1071C000B7173D001374F40F93870790E9B793073F
:1071D000B008639AF5003304804091671374F40F8C
:1071E000938797D04DBF93F5F5078D47639BF500C7
:1071F00033048040B7975B001374F40F938707D86C
:1072000059BF8947639BF50033048040B7770B0073
:107210001374F40F9387071BBDBF8547639AF5006E
:1072200033048040DD671374F40F938767E3A5B7D9
:1072300089E9330480408D671374F40F938777DCFA
:1072400099BFF1679387072029BF97000000E78067
:1072500040A0A285528597000000E780809F19BB5F
:107260009305610017E5FF1F0345254C17E4FF1F39
:107270000344B44B97000000E78040AE93057100D3
:10728000228597000000E78060AD3C0017F7FF1FE4
:107290002322F780834761002304F10083477100B4
:1072A000A304F100894717E7FF1F2305F76C8357F5
:1072B000810017E7FF1F2319F7460944A1AC1547C2
:1072C00093F64700B336D00093F78703850685C34E
:1072D0002146638BC7066146638AC7061306800290
:1072E0006388C706130680036393C700914717E6B8
:1072F000FF1F2309D66897E6FF1FA385F66897E767
:10730000FF1F2382E76817E7FF1F03472742937693
:10731000070497E7FF1F83C777418DEE1377770C3C
:1073200093067008630CD7021377F7078D46631E28
:10733000D70AB307F040B7955B0093F7F70F938533
:1073400005D881A81947ADBF854755B7894745B7C7
:107350008D4771BF930670086311D7021307300F72
:10736000B7150E006389E7021307900DB7B5040047
:107370006383E7021307700845BF9306800C63110F
:10738000D702B307F040B775460093F7F70F938520
:1073900085CDB3D5F50297E7FF1F23A3B75EF9B3F9
:1073A0009306900C631AD700B307F040916593F7EA
:1073B000F70F9385C566F1BF9306A00C631BD7003A
:1073C000B307F040B7153D0093F7F70F938505908D
:1073D000C9B79306B00CE319D7F4B307F040916531
:1073E00093F7F70F938595D06DB78946631BD70048
:1073F000B307F040B7750B0093F7F70F9385051BA4
:1074000049BF8546631AD700B307F040DD6593F79F
:10741000F70F938565E3B5BF09EBB307F0408D65C2
:1074200093F7F70F938575DCADB7F165938505206C
:107430009DB783472A00C18B99C7854717E7FF1F70
:10744000230DF75205BE97E7FF1F238807521DB68D
:10745000854717E7FF1FA308F75229BE3C0017E72F
:10746000FF1F2329F7620947930700032314F10044
:1074700097E6FF1F2380E6502DBD639A0758A94762
:1074800063ECB74417A701001307C7928A05BA95A2
:107490009C41BA97828717E4FF1F03441429094AC5
:1074A000630C440F636C8A0885476309F40A9307E9
:1074B000F00F17E7FF1F0347E74B63F6E70017E7F7
:1074C000FF1F2309F74A17EAFF1F034AAA4A930737
:1074D00000041374FA0F63F447011304000497E7E0
:1074E000FF1F9387275B83AA0700228617E5FF1FEC
:1074F00013058523D685330A8A40A29A9770010026
:10750000E780E0EB97E7FF1F2386474797E7FF1FDA
:1075100023A2575997E7FF1F83C7D7451547639A9B
:10752000E762B7E700E03707400023A0E718010053
:107530000100B7860040238086028DA58D47630C2D
:10754000F40A9947E315F4F697A701009387078D8E
:1075500017E7FF1F2320F754A947A1BF17E7FF1F15
:107560000347675497E7FF1F9387C742494697A58C
:1075700001009385A5936306870097A50100938575
:10758000E58E3E8597700100E78060E317E7FF1FF7
:107590002322A750C94731BF97E6FF1F83C6A650D5
:1075A000054797E7FF1F9387E73E6394E6023E8512
:1075B0001306700297A501009385C58C9770010092
:1075C000E780E0DF17E7FF1F2326A74C9307700231
:1075D000CDB53E851306300497A501009385C5847B
:1075E00097700100E780A0DD17E7FF1F2324A74A5B
:1075F000930730047DBD97E5FF1F83C5051317A5CD
:1076000001001305259497700100E780A0E6854AE4
:1076100017EBFF1F034B2B4997E5FF1F83C5E510B1
:1076200017A501001305059263185B0B9770010005
:10763000E78040E497E7FF1F83C7270FB5CBE368D8
:10764000F4E617A401001304A48A638C670117A44D
:1076500001001304648A6386470117A40100130420
:10766000248B228597700100E78060011375F50F68
:1076700093071500860717E7FF1F230DF7308D4787
:1076800017E7FF1FA308F73097E7FF1F938787309F
:107690000147BE861376F70F89076365A60297E751
:1076A000FF1F23A9D73E97E7FF1F83C7A72E11B55A
:1076B000979701009387C77C17E7FF1F232CF73CA0
:1076C0009147C5BB3306E40003460600A3800700CC
:1076D00005072380C7007DBF97700100E78080D930
:1076E00097E7FF1F83C76704E1D7E362F4DC1794D1
:1076F00001001304E47C638C570117940100130408
:10770000A47C63864701179401001304647D2285DD
:1077100097700100E780A0F61375F50F9307150029
:10772000860717E7FF1F2307F7268D4717E7FF1F79
:10773000A302F72697E7FF1F9387C7250147BE8659
:107740001376F70F8907E37CA6F43306E4000346BB
:107750000600A380070005072380C700D5B797E57B
:10776000FF1F83C585FC179501001305657E977083
:107770000100E78020D097E7FF1F83C7772193E7B9
:10778000470017E7FF1FA305F72083472A0017E7E5
:10779000FF1FA30DF71E6FF0EFFD179501001305F6
:1077A000657C97700100E780C0E497E7FF1F93872F
:1077B000E71D83C7070017E7FF1F2307F7F617E446
:1077C000FF1F0344241B33348000A9B31795010025
:1077D0001305857A97700100E780A0E197E7FF1F06
:1077E00083C7171B93E7070117E7FF1FA302F71AC9
:1077F00083472A0017E7FF1F230AF7186FF08FF758
:10780000179501001305857897700100E78060DE09
:1078100003470A007D8B51EFB787004003C767021B
:107820001377C70B136727002383E70203C7A70259
:107830001377C70B136727002385E70203C7E70207
:107840001377C70B136727002387E70203C72703B4
:107850001377C70B136727002389E702854717E7CC
:10786000FF1F2303F7F817E7FF1F2301F70417E7AC
:10787000FF1F230FF70E17E7FF1F230CF70E97E7E5
:10788000FF1FA38307F697E7FF1FA381070297E770
:10789000FF1FA38F070C97E7FF1FA38C070C97E729
:1078A000FF1FA383070E97E7FF1FA38E071E6FF02E
:1078B0006FEC89476312F70297E7FF1F83C707E75B
:1078C0009146638CD70863E0F604638EE70C636926
:1078D000F70A05476380E70EFD5717E7FF1FA30B65
:1078E000F70837074000B7E700E023A0E7180100DA
:1078F0000100B78600401306F0FC2381C60223A0D6
:10790000E7106FF08FD4130720086382E7086362E3
:10791000F70213071008E391E7FC3787004083471D
:10792000670293F7C70B93E727002303F7026FF073
:107930006FE4130730086389E70213074008E39DEB
:10794000E7F8378700408347270393F7C70B93E790
:1079500027002309F7026FF0EFE1378700408347E4
:10796000270393F73707F5B7378700408347E702C8
:1079700093F7C70B93E727002307F7026FF08FDF1A
:10798000378700408347E70293F73707F5B7378714
:1079900000408347A70293F7C70B93E7270023050F
:1079A000F7026FF02FDD378700408347A70293F778
:1079B0003707F5B7378700408347670293F73707E4
:1079C000ADB7179501001305655D97700100E7805D
:1079D00040C297E7FF1F238907D4D5B3179501004D
:1079E0001305C55C97700100E780A0C097E7FF1FF3
:1079F000239C07D297E7FF1F9387C7F703C40700AD
:107A0000894763F3870009441374F40F21B6130701
:107A10000002E393E7EC6399090A638FF50093078B
:107A200020026381F508179501001305A55B977087
:107A30000100E78020A44DB5179501001305C55737
:107A400097700100E780E0BA0144179B0100130B17
:107A5000EB57A14AB3078A0083C507005A8505047E
:107A600097700100E78000A1E31654FF179501000D
:107A7000130585B497700100E780A0B717E4FF1FD6
:107A80000344C4CA11E497E7FF1F238207C859B40F
:107A90008947E313F4E4854717E7FF1F2309F7C677
:107AA0006FF04FCD17E6FF1F034636C897E5FF1F5F
:107AB00083C5A5C7179501001305C551977001002F
:107AC000E780409B6FF00FCB638FF50493071002A4
:107AD000E39BF5F497E5FF1F83C545C517950100A6
:107AE0001305455197700100E780C09897E7FF1F85
:107AF00023A247FB97E7FF1F938787E8944383D729
:107B0000470017E7FF1F034707E817E6FF1F232D6E
:107B1000D6C01D4497E6FF1F239AF6C097E7FF1FC4
:107B20002387E7C0C5BA97E5FF1F83C525C0179512
:107B300001001305A54D97700100E780A09397E71A
:107B4000FF1F238607BC97E7FF1F239F07BC6FF02B
:107B5000CFF62547E387E79C19476391E702B7868D
:107B6000004023808602B7E700E03707400023A0EB
:107B7000E71801000100130600FC41B31307100AC7
:107B80006391E702B786004023808602B7E700E0F2
:107B90003707400023A0E71801000100130680FC0E
:107BA000A9BB1307A009E38FE7FC1307400AE38B87
:107BB000E7FC13072002E386E7960547E383E79691
:107BC000B7E700E03707400023A0E718E3910996E4
:107BD00001000100B786004023808602130620FCC6
:107BE00029BB17E7FF1F0347F7D86308F71E63E7B2
:107BF000E7029547630EF70E99476308F704B786C7
:107C0000004023800602B7E700E03707400023A0CA
:107C1000E718010001001306A0FCC5B19307F005A9
:107C2000630AF700930750096306F70093071002F1
:107C3000E317F7FCB7E700E03707400023A0E71899
:107C400001000100B786004051BF97E9FF1F83C9BB
:107C500069D293070004CE8A63F43701930A0004C3
:107C600097E7FF1F938707E303AA070013F4FA0FB0
:107C70002286D28517E5FF1F130505AB976001002B
:107C8000E780E073B3878940529417E7FF1F23030F
:107C9000F7CE97E7FF1F23AF87DE638E0902B78712
:107CA000004023805703B7E600E03706400023A0DA
:107CB000C6180100010003C72702134707042381E8
:107CC000E70203C727021377C70F2381E70223A028
:107CD000C6106FF08F97B786004023800602B7E783
:107CE00000E03707400023A0E71801000100FDB5C0
:107CF000378700408347370097E6FF1F83C616C9C2
:107D000093F70708D58FA301F700B7064000B7E740
:107D100000E023A0D718010001001306A0FC2301F6
:107D2000C70223A0D7106FF04F9297E7FF1F9387EA
:107D3000E7D6A69783C7070093F7F70FD9CF97E742
:107D4000FF1F83C747D6D1EB17E7FF1F034797C233
:107D5000930700026313F70897E7FF1F9387C79CF9
:107D600003AB070097EAFF1F83CA4A9C17EAFF1F6D
:107D7000034ADA9B97E9FF1F83C9699BD28756871D
:107D8000CE865A8697E5FF1F83C565981795010033
:107D90001305452997600100E780C06D97E7FF1F35
:107DA00023A067BF97E7FF1F238E57BD97E7FF1FED
:107DB000A38A47BD97E7FF1F238737BD97E7FF1FBC
:107DC000A3868794B7E700E03707400023A0E718B1
:107DD00001000100B7860040D1B3B7E700E03707E4
:107DE000400023A0E71801000100B786004025B538
:107DF00029472381E70209472383E7022385E70216
:107E00002387E7022389E7026FF08F8803C76700A3
:107E1000118B6302078A83C75700918BB5CF17E791
:107E2000FF1F034747C885476313F70697E7FF1F00
:107E3000A38BE7B497E7FF1F2388079A97E7FF1FF5
:107E4000238607A697E7FF1F238407B297E7FF1F44
:107E5000238107B297E7FF1FA388079897E7FF1FC3
:107E6000A38607A497E7FF1FA38407B097E7FF1F28
:107E7000A38107B097E7FF1FA38807B097E7FF1F0D
:107E8000A38307C2B787004011476FF08F8217E7BF
:107E9000FF1FA30DF78679BF854717E7FF1F23054F
:107EA000F79417E7FF1F2303F7A017E7FF1F23012E
:107EB000F7AC17E7FF1F230EF7AA69BF854717E73F
:107EC000FF1F2303F79217E7FF1F2301F79E17E712
:107ED000FF1F230FF7A817E7FF1F230CF7A817E7CB
:107EE000FF1FA303079017E7FF1FA301079C17E7D6
:107EF000FF1FA30F07A697E7FF1FA38C07A682808B
:107F0000411106C697000000E78080FBB78700405C
:107F100023800700130740FC2386E7001307C004F3
:107F2000A386E70017E7FF1F130707802398E700E2
:107F300017E7FF1F13074783239AE70017E7FF1F81
:107F40001307C78E239CE70017E7FF1F1307479A05
:107F5000239EE70029472381E70209472383E7029D
:107F60002385E7022387E7022389E702A38107002D
:107F7000930600F8A380D700930690022380D700D1
:107F8000FD562383D7002381E700B706400037E77B
:107F900000E02320D71003C7170013671700A38042
:107FA000E700B24097E7FF1F2392079E41018280BE
:107FB000411106C697000000E78080F0B7870040B7
:107FC00023800700130700FC2386E7003147A386C0
:107FD000E70017D7FF1F130727752398E70017D768
:107FE000FF1F13076778239AE70017E7FF1F1307A0
:107FF000E783239CE70029472381E702094723837E
:10800000E7022385E702A3810700930600F8A38017
:10801000D700930690022380D700FD562383D70014
:108020002381E700B706400037E700E02320D710A0
:1080300003C7170013671700A380E700B24097E754
:10804000FF1F2395079441018280F16793870720E2
:1080500017E7FF1F2326F792854717E7FF1F231314
:10806000F792A14717E7FF1F230FF79097E7FF1F2E
:10807000A38B079097E7FF1F2388079097D7FF1FD1
:108080002387076897D7FF1FA3820768814717D503
:10809000FF1F1305E567FD5517D6FF1F130606687A
:1080A0002947B306F5002380B600B306F600238007
:1080B00006008507E397E7FE97E7FF1F238E079CDF
:1080C00097E7FF1FA38A079C97E7FF1F2387079C5B
:1080D00097E7FF1FA381078A97E7FF1FA38F0788F2
:1080E00097E7FF1F238A078897E7FF1F23850788E5
:1080F00097E7FF1F2384078897E7FF1FA38E078654
:1081000097E7FF1F238B078697E7FF1FA387079833
:10811000828017E7FF1F0347079985476316F7001B
:1081200017030000670003E917030000670083DD01
:10813000411122C406C617E7FF1F0347C7968547AC
:108140002E8613F4F50FAA856317F70417D5FF1FC2
:108150001305C57197600100E780602697D7FF1F60
:1081600023860774B787004023848702B7E600E0C0
:108170003706400023A0C6180100010003C7A7026C
:108180001377C70F2385E702B240224423A0C6100D
:1081900001454101828017D5FF1F1305E5609760F7
:1081A0000100E780C02197D7FF1F238F0762B787A1
:1081B000004023828702B7E600E03706400023A094
:1081C000C6180100010003C767021377C70F238396
:1081D000E7025DBF411106C697000000E78020E777
:1081E000B2404101170300006700E3F2411106C6E7
:1081F00097F0FFFFE780E0BD97D7FF1F83C7D75EEB
:1082000095C797D5FF1F83C5455E89C917D5FF1F41
:108210001305C55D97F0FFFFE780409C97D7FF1FD0
:10822000A384075C97D7FF1F23800776B2404101E4
:10823000828041C9D9C597D7FF1F83C72775D1C38E
:10824000011122CC4AC84EC656C25AC006CE26CA12
:1082500052C42E89AA890144930A0004371B0300E3
:1082600063772403B3078940C207C183BE8463F4E4
:10827000FA0093040004C204C180130A1BD497D7E8
:10828000FF1F83C767569DE37D1A631C0A00F240F7
:108290006244D2444249B249224A924A024B0561A1
:1082A000828097F0FFFFE780C0B2D1BF338589009D
:1082B0002694A685420497000000E780A0E741804D
:1082C00045B7828097E7FF1F9387878118429C43B9
:1082D00083D645000345070083C5C7000356460003
:1082E0006396A50083D5E700638DD502011106CE04
:1082F0002386A7002397D700B705CF00DC4B9385D3
:10830000757D05077D162EC2230001003AC4231691
:10831000C1002317D10099C30A858297F2400561F5
:1083200082808280DC4DDC4B81CFB7E70400904532
:1083300003A38705914517D5FF1F0345A57A02833F
:1083400082806D713C083EC6B707E500232291107C
:108350003EC8AA843C083285232611103ECA232435
:108360008110232021112E8997300000E780E05AE8
:108370002A8497950100938565CE17850100130522
:10838000E5BC97600100E780E00EA285179501002B
:10839000130545DD97600100E780C00D2945976012
:1083A0000100E7800012B705CB009385757D68005A
:1083B00097100000E7800064A285680097300000F5
:1083C000E7800048014781467000CA8526859720CE
:1083D0000000E780808705CD2A849795010093856A
:1083E000E5C717850100130565B697600100E780B2
:1083F0006008A28517950100130585D797600100D5
:10840000E7804007294597600100E780800B8320C3
:10841000C1100324811083244110032901105161EC
:10842000828097D7FF1F9387A76B18429C4379716F
:1084300022D406D60348070083C807012A8483D6BE
:108440004500035546006396080183D82701638DD4
:10845000D8022388070105072399D7003708CC00E5
:10846000DC4B1308787D3ACC1307F5FF42CA23088A
:108470000100231EE100231FD10099C7080832C65E
:108480002EC482973246A245228597000000E780DD
:1084900080EBB2502254456182806D713C083EC031
:1084A000B707E5003EC23C083EC423261110232432
:1084B0008110232291102317010023180100231992
:1084C0000100231A0100231B010097B7FF1F83D768
:1084D00067EF99E3C167FD172316F10097B7FF1FF8
:1084E00083D767EE91EB97D7FF1F9387675F9C4316
:1084F0009C43DC4783D7070017B4FF1F130484ECA9
:10850000584C2317F10083574400484B2318F100BF
:1085100031E197950100938565BB1785010013052F
:10852000E5A297600100E780E0F4179501001305CC
:1085300025BB97600100E780E0F3294597600100C3
:10854000E78020F88320C110032481108324411088
:108550005161828097B7FF1F83C737E789EBB7E781
:108560000400BC5782975C4C23AA0700E1BFFD17AB
:1085700097B6FF1FA38BF6E4035607018347040158
:108580004C470A85230BF10097300000E7806028F4
:1085900097D7FF1F9387C7549C4301478146884361
:1085A0000A866C0097100000E780206AAA8429C11F
:1085B00097950100938585B11785010013050599ED
:1085C00097600100E78000EBA68517950100130571
:1085D000E5B197600100E780E0E929459760010077
:1085E000E78020EE584CB7E70400BC57484B9DBFCE
:1085F00097B7FF1F83C777DDF5D7B7E70400BC4FF8
:108600001044854517D5FF1F0345C54D82971DBFF3
:108610005C4EDC4BB9CFB1CD411122C417850100AE
:108620001305C5922E8497950100938565A806C60B
:1086300097600100E78000E4A2851795010013050B
:10864000A5AD97600100E780E0E229459760010051
:10865000E78020E7B7E704002244B24003A3870580
:1086600017D5FF1F034505481306400691454101F4
:1086700002838280411122C417B4FF1F130444D225
:108680001C4C06C689C7DC4399C34C488297584C9A
:10869000B7E70400BC57484B82975C4CB240224479
:1086A00023AA07004101828017B7FF1F130747D194
:1086B000834707009306F00B850793F7F70F63E9ED
:1086C000F60097B6FF1F238DF6CE03450700828084
:1086D000930700F8FDB78357450063860710011123
:1086E0004AC817B9FF1F1309E9CD52C4032AC901AB
:1086F00006CE22CC03274A0126CA4EC656C2F157DF
:1087000035E31307D00DFD57636EC704B7E90400C6
:1087100083A709072A841305860042054181B28494
:10872000AE8A8297232AAA000325C9015C49A9E7DA
:10873000979501009385C59517850100130505815F
:1087400097600100E78000D317950100130505A588
:1087500097600100E78000D2294597600100E7801B
:1087600040D6DD57F2406244D2444249B249224ADF
:10877000924A3E850561828093874400B705CF0009
:108780002319F5009385757D310597100000E7806A
:1087900060260325C9018345640031059730000038
:1087A000E780000A0325C9012686D6853105973062
:1087B0000000E78000067146A2854A8597600100A7
:1087C000E780E0BF504419CA83A78905854517D5BE
:1087D000FF1F034525318297814769B79700000045
:1087E000E780E0CBD5BFFD573E858280411126C290
:1087F00097B4FF1F938404BDD84C22C437E404000F
:108800003C54484B06C68297DC4C0323C4052244E3
:10881000B240924423AA070017D5FF1F0345852CB9
:10882000854541010283411126C297D4FF1F9384DD
:10883000242B9C4006C622C44AC0D5C3DC43C5C312
:108840005CC12300B5002A84978501009385857F4C
:10885000177501001305856F97600100E78080C1DF
:10886000294597600100E780C0C59C4023A407000C
:1088700023A2070097B7FF1F938787B2DC4FDC4B1B
:1088800091C7295597000000E78000DF97B7FF1FC9
:10889000938747B3DC4FDC4B89C797000000E78024
:1088A00020F537E904008327C905894517D5FF1F3F
:1088B0000345452382978327C905914517D5FF1F97
:1088C0000345452282979C4003A3470163090300A7
:1088D00022852244B2409244024941010283B240BF
:1088E000224492440249410182800111328506CE20
:1088F00022CC26CA2E8497300000E7800002AA848A
:108900009785010093854577177501001305056468
:1089100097600100E78000B60307840003566400F7
:1089200083554400A686179501001305E5809760DE
:108930000100E78020B4294597600100E78060B816
:1089400097B7FF1F83C727A6639D97000145970030
:108950000000E78060D281450A8597000000E7802B
:10896000C0ECF2406244D244056182806D712324E0
:108970008110232611102322911093F745002E8495
:10898000638707143C083EC0B707E5003EC23C08B9
:108990003EC4231701002318010023190100231AE4
:1089A0000100231B010097B7FF1F83D7679F99E33F
:1089B000C167FD172316F10097B7FF1F83D7679E86
:1089C00091EB97D7FF1F9387A7119C439C43DC47EC
:1089D00083D7070017B7FF1F1307879C2317F100E2
:1089E000544F835747002318F100DC4AA1E79785CD
:1089F00001009385A56C1775010013052555976037
:108A00000100E78020A7178501001305656D9760B9
:108A10000100E78020A6294597600100E78060AA51
:108A2000134544008320C110032481108324411086
:108A30005161828097B7FF1F83C7F7962555D9C329
:108A4000FD1717B6FF1FA300F69603D6060183474E
:108A50000701CC460A85230BF10097300000E78020
:108A600040DB97D7FF1F9387A7079C4317B7FF1FCC
:108A700013070793978601009386866988430A86C1
:108A80006C0097100000E780401CAA8451D997859C
:108A900001009385A562177501001305254B9760AA
:108AA0000100E780209DA685178501001305056458
:108AB00097600100E780009C294597600100E780EE
:108AC00040A0268597000000E78000BB91BF93F788
:108AD00025009DC7B7E70400BC47414681452808EB
:108AE0008297255597000000E78000B92808930574
:108AF000F00F97000000E78040D3134524001DB716
:108B000093F71500014599DF97000000E780209951
:108B10001345140001BF5C4D411106C688C317D729
:108B2000FF1F232FF7FAB7E7040083A707081705ED
:108B300000001305E5E38297B24097D7FF1F238318
:108B4000A7FA01454101828001119307700F231696
:108B5000F10006CE97D7FF1F83C757FA8DE7B7E717
:108B6000040083A7870D17B6FF1F0346A6886C0075
:108B700017D5FF1F0355C5F882973335A00097D747
:108B8000FF1FA38DA7F6F2400561828041119397E4
:108B9000050122C406C626C2C1872E8463D40702FB
:108BA000B7E40400FC5417B5FF1F0345A584829762
:108BB00019C1BC5482972165218DB2402244924450
:108BC0004101828093F715008DC7B7E7040083A7A2
:108BD000471A17B6FF1F1306E68097D5FF1F938528
:108BE00025F117B5FF1F0345E58082971345140053
:108BF000E9B793F7250099CFB7E70400BC4F1306F8
:108C00000064894517A5FF1F0345C57E829713455C
:108C1000240065B793F785009DC7B7E7040003A854
:108C2000871A1307401F97A7FF1F83C7A77C81469A
:108C300013064006994517D5FF1F035565EC0298AA
:108C4000134584009DBF93F745000145BDD7B7E4A8
:108C5000040083A7041817D5FF1F035565EA829700
:108C6000BC4C13060064914517A5FF1F034585788A
:108C700082971345440091B797D7FF1F83D747E8E2
:108C80006398A70217D7FF1F231DB7E617D7FF1F4B
:108C9000231AC7E617D7FF1F2317D7E62E86178597
:108CA00001001305A566BE85175301006700837C8C
:108CB00017850100130505671763010067006393BB
:108CC00003574500011106CE22CC97D7FF1F83D74B
:108CD00027E3178501001305E5646310F706C167F4
:108CE000F91717D7FF1F232DF7E037E4040097D7B4
:108CF000FF1F23A907E07C4C894517A5FF1F0345EB
:108D0000656F82977C4C914517A5FF1F0345856EC3
:108D1000829797B7FF1F83C7F74C85CB8547A3077B
:108D2000F100832744171306F100854513055030E1
:108D30008297178501001305255397600100E7808E
:108D4000408BF24062440561828097D7FF1F83C742
:108D5000A789178501001305E555E5F38547A307A6
:108D6000F100832744171306F100854513055030A1
:108D700082971785010013056551C1B77D15954789
:108D800063E5A71A178701001307C74A0A053A9532
:108D90001C41011122CC06CEBA972E8482871785FA
:108DA00001001305A55897600100E780808415A293
:108DB00003C7250099476311F7022E85970000002D
:108DC000E78040F0834564001785010013050557CF
:108DD00097500100E780006A97B7FF1F2384074080
:108DE00017850100130545577DBF03C7250095472B
:108DF0006319F702C16717D7FF1F035767D0F91729
:108E000003D5A5006309F702B7E7040083A7C717D6
:108E10008297178501001305255597500100E780BB
:108E2000407D854717B7FF1F230EF73A17850100CE
:108E3000130505568DBF97D7FF1F2393A7CC83D764
:108E4000E50009661306069017D7FF1F231BF7CA14
:108E500083D7050117A5FF1F0345C55917D7FF1F66
:108E60002312F7CA83D72501A14517D7FF1F231C5B
:108E7000F7C8B7E70400BC4F82970356E400835558
:108E8000A400178501001305654F97500100E78086
:108E9000605E41BF178501001305455029B783C5A2
:108EA00025009147639BF50285471785010013054F
:108EB0006550A307F10097500100E7808073B7E782
:108EC000040083A747171306F100854513055030AA
:108ED0008297F24062440561828099476392F5026D
:108EE000228597000000E780E0DD83456400178558
:108EF00001001305A54497500100E780A057D1BF9A
:108F00009547639FF50083471400178501001305FB
:108F1000654AE39A07E8178501001305654B61B5BB
:108F2000178501001305454BF9B782806D71232425
:108F300081102326111023229110328401CD8947FC
:108F4000630AF5028320C110032481108324411099
:108F500051618280178501001305C548AE84975082
:108F60000100E7800069A285268597C0FFFFE780A2
:108F70008066C9BFB7E70400FC47280082971785C1
:108F800001001305E54697500100E780806683479E
:108F9000810039C41307000B6380E7021387A7051C
:108FA0001377F70F8D4663EDE602A285280097D070
:108FB000FFFFE78060D579B78547E3F587F88345FC
:108FC0009100177501001305A52DB335B00097B7B3
:108FD000FF1F238BB70897500100E780A0499DB77A
:108FE00003479100A207D98F35671307D7556385CB
:108FF000E7086368F7022D671307B7556387E7062D
:1090000031671307C755638AE70429671307A75514
:109010006394E702A285280097D0FFFFE780A008AD
:1090200015B739679306E765638DD70663E9F600E0
:109030001307E7556380E706A28528003DB73D6723
:109040009306F7556386D7061307F766E396E7FEA0
:1090500097D0FFFFE7802021F5B50146A2852800C3
:1090600097D0FFFFE78060F1F1BDA285280097D07F
:10907000FFFFE7808001F9B58947E3F587EC9305A9
:10908000E4FFC205C1811305A10097A0FFFFE7809F
:1090900000124DBDA285280097D0FFFFE780A001F8
:1090A00055B5A285280097D0FFFFE780600C59BD19
:1090B00097D0FFFFE780E01471B5411122C417A4D7
:1090C000FF1F13046434AA861786010013060618CE
:1090D0002285C14506C697500100E780C05203575C
:1090E000440097A7FF1F938727332393E700035775
:1090F00064002394E700B2402244410182800111C0
:1091000006CE22CC97000000E78060FB37E4040025
:109110008327841417A6FF1F1306062FD545014584
:109120008297832784179305F100130550308297A7
:109130008347F100A1C7A307010083274417130643
:10914000F10085451305503082978327441717A6F1
:10915000FF1F1306662CCD45130570308297854797
:10916000A307F100832744171306F1008545130573
:1091700050308297F2406244056182808327441711
:1091800017A6FF1F13064629CD4513057030D5B726
:1091900061712324811A37E40400832704082326FD
:1091A000111A2322911A2320211B232E311917056E
:1091B00000001305E59D829717A9FF1F1309892356
:1091C000994785442300A900231CF10097850100DD
:1091D0009385C5109307400617750100130505D741
:1091E000231CF1082308910097C9FF1F9389295078
:1091F00097500100E780002883D5090017850100FA
:109200001305850597500100E780C0262945975032
:109210000100E780002B03D5090085699700000055
:10922000E780E0E98327441710088545130550308F
:1092300082978327441717A6FF1F1306E61DCD4507
:109240001305703082978327441717A6FF1F130654
:10925000A61AB54513056030829783274417300856
:1092600089451305103182978327441730098945B2
:1092700013052031829783274415938509C80D452E
:10928000829783274415938509C811458297A305C2
:109290009100230691002308910002CD230C0100C8
:1092A00083278416300991451305704082978327E0
:1092B00084161306B1008545130500408297832765
:1092C0008416700085451305104082978327841605
:1092D000300885451305204082978327841610089F
:1092E0008545130550408297832704157D55829745
:1092F000832744137D5582977D5597A0FFFFE78014
:10930000C0358327440C829797A0FFFFE7800011A8
:109310008327841417A6FF1F1306060FD5450145A2
:10932000829789471306700F814528092306F100AB
:109330009790FFFFE78060DA8D47130600088145AC
:109340002808230CF1089790FFFFE78000D9914788
:10935000230CF100977701009387C7B0984383C728
:1093600047003AC8230AF10097D0FFFFE78060F674
:1093700070008545054597A0FFFFE780203530093F
:109380009305700F094597A0FFFFE7802034300850
:10939000930500080D4597A0FFFFE78020331008D4
:1093A0009545114597A0FFFFE7804032C16717C779
:1093B000FF1F1307E774F9171CC32322070017A523
:1093C000FF1F1305E50297A0FFFFE780002F83270B
:1093D000C41D17C5FF1F1305257182973C4803451F
:1093E0000900854582978320C11A0324811A8324AA
:1093F000411A0329011A8329C1195D618280C1675D
:1094000017C8FF1F0358C86FF9176301F8083DCD4F
:10941000B5CD011126CAB7E4040083A7841222CC7B
:109420002E862315B10006CE2A8401478146ED45DC
:10943000428582972AC611ED17850100130505EBB9
:1094400097500100E780E01AF2406244D24405617F
:109450008280FC440356A100A28582972C0017C588
:10946000FF1F0355E56997A0FFFFE780C03169DD65
:10947000178501001305C5E897500100E7806017C4
:1094800083A7C412ED45280082977DBF8280011119
:1094900006CE22CC2DC9854717A7FF1FA303F7F6D9
:1094A00097A7FF1F238007F637E40400832784175C
:1094B0009305F1001305503082978347F100A9CB43
:1094C000A3070100832744171306F1008545130500
:1094D000503082978327441717A6FF1F1306C6F143
:1094E000B5451305603082978547A307F1008327B0
:1094F00044171306F1008545130550308297F2405A
:1095000062440561828097A7FF1FA38C07EE49BFC5
:109510008327441717A6FF1F130606EEB54513054C
:109520006030E9BFC16717C5FF1F0355655DF917B7
:109530006307F500B7E7040003A3C717028382801F
:1095400001118547A307010017C7FF1F2308F75A1A
:10955000B7E7040083A7471706CE1306F100854539
:10956000130550308297F240056182801793FFFF08
:10957000E70203B22A8408452E89B28919C900C1BD
:10958000971500009385A586610597300100E78057
:10959000800181447D5A97100000E780E03963C75D
:1095A000A404814497100000E780003A63C8A40433
:1095B00097C7FF1F938747559C43DC47B307F94084
:1095C00091872302F400638309048327C900B3074A
:1095D000F4409587A302F4001C4C89C79C4799C3AB
:1095E000228582971793FFFF6700C3AD5C441397F2
:1095F00014008504BA972390470171BF1C48139744
:1096000014008504BA972390070069BF8327890057
:109610000547B307F4409587A302F400835704007D
:10962000638EE7028DC309476384E7040D47E39522
:10963000E7FA978701009387672E1CCC9787010074
:109640009387C72E11A8978701009387A7F41CCC96
:1096500097870100938707F55CC8BDBF9787010016
:10966000938747E01CCC978701009387A7E0EDB76D
:10967000978701009387472F1CCC9787010093871A
:10968000A72FD9BF95E51793FFFFE70203A2004676
:1096900018448347940075839D8B6317F7009710D8
:1096A0000000E78060B448C41793FFFF670023A25F
:1096B00082801793FFFFE702A39D13893500C164E1
:1096C00042094111AA890144F11413590901054ABB
:1096D0002EC697100000E7802026B2456348A400FC
:1096E000014541011793FFFF6700C39D83A7090050
:1096F00013171400BA9783D707006388B7006394E1
:10970000970063742A010504E1B70545D9BF179393
:10971000FFFFE7020397AA892E89328BB6843A8A23
:10972000BE8A97A00000E78020FB71C9268597209C
:109730000000E78020098D4763E7A7007D55179358
:10974000FFFF6700839783DB440097100000E780EA
:10975000A0242A8497100000E78040259307740016
:1097600031443305850263CDA70297100000E780DE
:10977000A02297100000E78020222A849710000082
:10978000E780C0229307740031443305850263C328
:10979000A70497100000E78020209307450029A820
:1097A00097100000E7808020330585021307F0172B
:1097B0009307C017E35FA7FA2D55E3C277F9630457
:1097C0000B02D6865286A6854A8597200100E7803F
:1097D00020BAB5B797100000E780401D3305850219
:1097E0009307C5FFD1BF832749001385C90083D5DF
:1097F000270097000000E78000EC61F581B769550C
:109800003DBF97C7FF1F2393A73097C7FF1F9387BD
:10981000A72F904381470C463307F5004207418349
:109820006393B70082805446139847008507C29619
:109830002390E600D5B797C7FF1F9387E72C9C437B
:1098400003C58700828017C5FF1F0355252C828022
:109850001793FFFFE7026385C1671387D7FF630B89
:10986000E502636AA700F1176300F502014517934B
:10987000FFFF6700C3851387E7FF6302E502FD175B
:109880001D8D13351500E5B797500000E780C02601
:109890007D15C5BF97500000E78040FBD5BF9750AE
:1098A0000000E78060F9EDB71783FFFFE702E37F71
:1098B0004111AA8401442EC697100000E780C00819
:1098C000B2456348A400014541011793FFFF6700BB
:1098D00003809C48131514003E9583570500E385CB
:1098E000B7FE0504C9BF03485500814693F7F60F3C
:1098F00063E5070181473E8582805845939756006E
:10990000BA9703D727006316B70003D70700E3040D
:10991000C7FE8506E1BF8346450001479377F70FF1
:1099200063E4D700814711A81C45131657000507AB
:10993000B29703D60700E313B6FE3E8582801783F5
:10994000FFFFE702E37493170501C18797CAFF1F62
:10995000938A8A1B635BF00883A70A00C0479C4771
:1099600003570400198D420541816368F5000144E5
:1099700022851783FFFF6700E37412052A94CDBF89
:10998000DC4713944900014A3E94834744006341F5
:10999000FA02014A834754006349FA028509C20961
:1099A00093D9090183A70A009847E3EBE9FCC1B703
:1099B0001C4413195A00A6853E994A859700000059
:1099C000E780C0EE05E1050AC9B75C4413195A00E7
:1099D000A6853E994A8597000000E78020ED19E1B1
:1099E000050A4DBFE30C09FA61B7AA8481495DBF3E
:1099F0001783FFFFE702636B1C452A8481E7930707
:109A0000C5001CC51C44231204001CC09307F00FA2
:109A100063EDB70093F5F50F228597200000E780EE
:109A200020E21783FFFF6700836A93940501C167F3
:109A3000C18063F9F500A685228597200000E780A4
:109A400040E5C5B7C18193F5F50F22859720000049
:109A5000E78000DFA685228597200000E78040E0B0
:109A6000C9B797C7FF1F9387270A884382801C4581
:109A700099C797C7FF1F23A9A708014582807D5575
:109A8000828097C7FF1F9387270898438347450025
:109A9000484792073E9582801783FFFFE702E36005
:109AA000617100451C183EC6B70780013EC81C18EE
:109AB0003ECA8357440002CE02D002CC231EF100DE
:109AC000834784002A8902D22301F1023C083ED454
:109AD00002D697000000E78000FB8357050023169D
:109AE000F10297500000E78060C42307A1025C40A8
:109AF00003556400F18313F717008347F102520501
:109B00005181F99BD98FA307F10297100100E780DB
:109B1000807539CDAA840355050097A00000E78021
:109B200080BC83D704002AD26800231CF10083D7AD
:109B30002400231DF1001C4803D647008C439720C6
:109B40000000E78000CD8347B400CA861786010075
:109B50001306C68A8117A305F4006C0048109720ED
:109B60000100E780E0805D611783FFFF67002356F7
:109B70002155D5BF1C45B1CF03C5A7008946135752
:109B80006500630BD7028D46630ED70285466300DE
:109B9000D702130740063305E50203C7B700418B20
:109BA00015CB83C7B700BD8B3355F5408280137545
:109BB000F5031307803EC5B709671375F50313074F
:109BC0000771D1BF372709001375F5031307077C09
:109BD000D9B7014582801783FFFFE702034D03A930
:109BE0008500630C09048347B900AE8493F7070E20
:109BF00085C303459900930520030D810505B30531
:109C0000B5028844610597300100E780E0A935A0DE
:109C10002E8597000000E78020F62A8419CD970052
:109C20000000E780605C8325C900B307B54063FA94
:109C300087002E94B305A440E9F51783FFFF670062
:109C4000034985457DBF1783FFFFE70203462A844A
:109C500003D50500011132C636C43AC22EC002CA6D
:109C600002CC02CE97A00000E780E0A782452ACA76
:109C700022852ECC97000000E780E0E00357050026
:109C8000231EE10097500000E78040AAA24632461A
:109C90009247230FA10036874C08B28622850146E1
:109CA00097000000E780E0A605611783FFFF6700CB
:109CB00003421783FFFFE702433F61711C183EC652
:109CC000B70780013EC81C183ECA3C0800453ED478
:109CD000AA8402CC02CE02D002D202D697000000A3
:109CE000E78060DA8357050035592316F102975053
:109CF0000000E780A0A32307A10209C48357440002
:109D000081EB21594A855D611783FFFF6700233C82
:109D1000035564005205518197100100E780A0545B
:109D20002A8965D18347B40093F7070E99C71305B5
:109D3000840197300100E780609983574400231E17
:109D4000F100834784002301F1025C4003550900C0
:109D5000D98313F7070883471102231CA10093F747
:109D6000F707D98FA300F10283572900231DF100C3
:109D70005C40F18313F717008347F102F99BD98FF9
:109D8000A307F10297A00000E780E0952AD235D919
:109D9000834794006800139757008347B400FD8BF6
:109DA000D98FA305F4001C4803D647008C439720A5
:109DB0000000E78000A6A687177701001307076455
:109DC000740005464C10268597000000E7806094DB
:109DD0002A890DD98347B400A685FD8BA305F4001D
:109DE00097000000E78060DF31BF1783FFFFE702C5
:109DF000C32B832485FE2A84411126859700000009
:109E0000E78080D7834734FF93F7070E8DCB2AC6B0
:109E1000268597000000E78060C809CD834734FF9E
:109E2000B245FD8BA309F4FE91C522859730010050
:109E3000E780808741011783FFFF670043297DD9B1
:109E40008327C4FF2685829775F5834734FF93F7F0
:109E5000070E91C7228597300100E78020870325F0
:109E600084FE97000000E78000E5E9B71783FFFF55
:109E7000E702A3209C4141112A8903C707008947B3
:109E80002E84935667006380F6040D466388C604EB
:109E90009307F0076304F7022E8597200000E78000
:109EA000C0A7AA848149C16B130C490097C7FF1F43
:109EB000938787C59C43984763E4E904410117836E
:109EC000FFFF6700431F03D745008547E3F8E7FE20
:109ED0002E8597200000E780A0A9E1B703D74500B1
:109EE000E3FEE7FC2E8597200000E78000A3AA840C
:109EF000228597200000E78060A4C204C98C5DB76A
:109F0000DC470355A900139A49003E9A93170501AF
:109F1000C187635DF00083570A006397A70263E778
:109F200074038327CA00034D5A002DA0A16721673F
:109F3000A98F1307F7EFE374F7FE63970900970003
:109F40000000E780209161FD85098DB783278A0095
:109F5000034D4A00835DA90003576900216A138BF2
:109F6000C7003AC6814A33CA4D01631E5D0197C7D7
:109F7000FF1F9387E7B99C43E1DBA2866286814598
:109F800026858297D1B7A1679387F7EF930C4BFF94
:109F900063F24703B2455A8597F0FFFFE780A0714F
:109FA0000DC103278B00104709CE10436382C40202
:109FB0003107D5BFEE85668597000000E780008FEA
:109FC00071F993861A0093FAF60F130B0B0271BF07
:109FD000835644005C43E3E9F6F622853AC69710BF
:109FE0000000E780807DA1679387D7042A8A035DFC
:109FF0004400324763E897008347D90093E707F8A6
:10A00000A306F9001C4766852286E2858297C16710
:10A010000844FD17337AFA00529508C02312A401B0
:10A0200025B797C7FF1F938727AE9843814715C36E
:10A030001447814763FFD500939745004C47BE9571
:10A0400019C903C7550081476375E600DC4516064C
:10A05000B2973E85828003C745008147E37BE6FED9
:10A0600016069C45F5B71783FFFFE7026302AA892E
:10A070002E8A814497CAFF1F938A0AA983A70A00E0
:10A08000984763E6E4001783FFFF6700A303DC47FC
:10A090001394440001493E9413BB140083474400C9
:10A0A000634BF900014913BB140083475400634F0D
:10A0B000F9008504E1B70844931759005287DA86FE
:10A0C0000146A2853E9582990509C9BF4844931768
:10A0D00059005287DA860546A2853E958299050980
:10A0E000E9B71783FFFFE70243FC814517F5FFFF40
:10A0F0001305054897C7FF1F239A07A09700000084
:10A10000E780A0F61783FFFF670063FC97C7FF1F78
:10A110009387879F9C4395C31783FFFFE702E3F86C
:10A12000814517F5FFFF1305A54497000000E78060
:10A13000C0F31783FFFF670083F982801783FFFF57
:10A14000E70203F537E40400832784124111231545
:10A15000E100AE893289368A3A8681460147ED456B
:10A16000AA8482972AC621C90356A100D2859740A6
:10A170000100E780C0248327C413CE8526858297FB
:10A18000058905C98327440D2314210101462C00AC
:10A19000268582972A8401C9B7E7040083A7C712DE
:10A1A000ED4528008297228541011783FFFF670054
:10A1B00063F14944D5B76554FDB75C41FD175CC1F7
:10A1C00082801783FFFFE70243EEB7E70400FC5FDE
:10A1D000829795473305F50281450D811783FFFF6F
:10A1E0006700E3EE1783FFFFE70223ECB7E7040005
:10A1F000FC5F829795473305F5020D811783FFFFBA
:10A200006700E3EC1783FFFFE70223EAB7E70400E8
:10A2100083A7870B0355050082971783FFFF67000D
:10A2200003EB1783FFFFE70243E80355050032877E
:10A23000AE861796FF1F0356462497C5FF1F9385CA
:10A24000658D97000000E780A0EF1783FFFF670090
:10A2500003E81783FFFFE70243E5B7E7040083A79E
:10A26000C71782971783FFFF670063E61783FFFF17
:10A27000E702A3E3B7E7040083A7871397C5FF1F8F
:10A2800093854589829701451783FFFF670023E483
:10A290001783FFFFE70263E1B7E7040083A7C71F47
:10A2A00081451795FF1F0355451982971783FFFFB7
:10A2B0006700E3E11783FFFFE70223DFB7E704004E
:10A2C00083A7871397C5FF1F9385C585829701458F
:10A2D0001783FFFF6700A3DF1783FFFFE702E3DCBD
:10A2E000B7E7040083A7C71F81451795FF1F0355D4
:10A2F000C51A82971783FFFF670063DD1783FFFF8F
:10A30000E702A3DA2E8597800000E780E0AF978010
:10A310000000E780E0EC1783FFFF670043DB178353
:10A32000FFFFE70283D897800000E780E0F61783FD
:10A33000FFFF6700C3D95C49E1175CC95CC583575F
:10A340002501A1072319F50083570501A10723184B
:10A35000F5008280F1473305F50297B7FF1F938719
:10A36000677E9C433E9582808D476315F60803D730
:10A370004600854763F0E7081783FFFFE702E3D253
:10A38000368536842E8997100000E780005929C948
:10A390008357440093140501C18063E39704228529
:10A3A00097100000E7806057FD1423129400930774
:10A3B000A0026300F5029307B0026307F50293075A
:10A3C0009002631FF500228597000100E780C08599
:10A3D00001A80146CA85228597A00000E78060B0E9
:10A3E0001783FFFF6700A3CE228597100000E78048
:10A3F000C003FDB7828097B6FF1F9386E6749C4228
:10A40000014599CF9843D44217B6FF1F232EE67219
:10A410006396D70097B6FF1F23AAE6721385C7FE7F
:10A4200082801783FFFFE70243C897000000E780A0
:10A43000A04B714433058502914597900000E78059
:10A4400020E911E565551783FFFF670043C897B7FB
:10A45000FF1F23A7A76E97000000E780E0483305A1
:10A460008502914597900000E78080E661DD97B70F
:10A47000FF1F23A9A76C97000000E780E04697B76D
:10A48000FF1F2399A76A97000000E780E04597B770
:10A49000FF1F2392A76A97770100938767FB17B77F
:10A4A000FF1F232DF76897070000938707E917B769
:10A4B000FF1F2323F768014579B71783FFFFE702E2
:10A4C000C3BEAA8517B5FF1F1305C5669710000008
:10A4D000E780C05B1783FFFF670063BF1783FFFF41
:10A4E000E702A3BC97000000E78060FD9710000022
:10A4F000E780405B97B7FF1F938707659C4391CF29
:10A500001387C7FE19CB83D5C7FF17B5FF1F1305E8
:10A51000256497200100E78020191783FFFF67005B
:10A5200003BB1783FFFFE70243B897000000E780F3
:10A53000C0EC09CD834785002A8493F7070499EB83
:10A540000355E50097000000E78080F91783FFFFBF
:10A550006700E3B78347C5009304450117B9FF1FA0
:10A560001309895E85E3832709005CC997B7FF1F3C
:10A5700023AC975C83274900F1FB97B7FF1F23A704
:10A58000975CE9B7FD172306F50061059780000089
:10A59000E780C0D68307840063CB07048347840029
:10A5A00093E707F82304F400B7E704009C5F829761
:10A5B0004205A94741813375F5028347840093F72B
:10A5C00007FCC98F2304F4008347D4003E951C4048
:10A5D0002318A40089CF984319CB8347C400504067
:10A5E000814585073305F50242054181029783279E
:10A5F00009005CC897B7FF1F23A897548327490019
:10A6000089E797B7FF1F23A397548347C4009DDFB3
:10A610008355040117B5FF1F1305855397200100CB
:10A62000E780800825B71783FFFFE70203A897B7E5
:10A63000FF1F938727779C4701448583858B85E39C
:10A64000AE84B2853A8697100000E780804B2A845A
:10A6500019C597100000E780C041829408CC22857C
:10A660001783FFFF6700A3A61783FFFFE70243A23C
:10A6700041112E8932C6AA8997000000E780C031B7
:10A68000324713060502CA86970500009385C5CC9C
:10A6900017B5FF1F1305054A97000000E780E0F893
:10A6A0002A8425C99304C50097000000E780E04193
:10A6B0001946AA85268597100000E78080158545F4
:10A6C000268597100000E7806011177501001305BB
:10A6D000E5D54E9583450500268597100000E78057
:10A6E00020165C4831468145A1075CC85CC483578D
:10A6F0002401E1172319F40083570401E1172318FB
:10A70000F4001C4C3E859780FFFFE780009DA3046A
:10A710002501228541011783FFFF6700A39A178354
:10A72000FFFFE70283984111AA842EC632C4971016
:10A730000000E7806036004DB24522468347840022
:10A740000CC050C093F7F70393E707042304F40009
:10A7500023180400268597100000E7808031834786
:10A760009400A9462317A40013D737000507330721
:10A77000D7029D8B85072306F400A306E40083C758
:10A780000401D8488507230FF7FE17B7FF1F1307EB
:10A79000A73B5843232A04009307440129E317B732
:10A7A000FF1F2325F73A17B7FF1F232FF73817B4DA
:10A7B000FF1F1304E439228597200100E78000E1A0
:10A7C0001C44858B5D8D19E581452285972001000C
:10A7D000E78080ED41011783FFFF6700438F1CC3B3
:10A7E00017B7FF1F2324F736D9B71783FFFFE702F8
:10A7F000C38B97050000938565B70145970000005E
:10A80000E78000B001451783FFFF6700438C178383
:10A81000FFFFE702838997000000E78080B017837D
:10A82000FFFF6700C38A8347C500A5E31783FFFFC7
:10A83000E702A3872A840355E50097000000E7801C
:10A8400000C821C18347840093F7F7FB2304F40079
:10A850001C4091C7DC4381C74C400145829797005B
:10A860000000E78080B917B5FF1F1305652E9720FC
:10A870000100E780A0E50355E40097000000E780B1
:10A8800020C61783FFFF6700838482801783FFFF42
:10A89000E702A38197B7FF1F9387072B9705000057
:10A8A000938565C817B5FF1F1305852A23A00700E8
:10A8B00023A2070097200100E780E0CE1783FFFF67
:10A8C0006700E3801C4D91CFDC4381CF1773FFFFFE
:10A8D000E702A37D8345070082971773FFFF670098
:10A8E000037F828097B7FF1F9387C7289C4303C5C8
:10A8F0000700828097B7FF1F9387C7279C4303C534
:10A900001700828097B7FF1F9387C7269C4303C514
:10A910002700828097B7FF1F9387C7259C4303C5F5
:10A920004700828097B7FF1F9387C7249C4303C5C6
:10A930003700828097B7FF1F9387C7239C4303C5C7
:10A940005700828097B7FF1F9387C7229C4303C598
:10A950006700828097B7FF1F9387C7219C4303C579
:10A960007700828097B7FF1F9387C7209C4303C55A
:10A970008700828097B7FF1F9387C71F9C4303C53B
:10A980009700828097B7FF1F9387C71E9C4303C51C
:10A99000A700828097B7FF1F9387C71D9C4303C5FD
:10A9A000B70011E11D45828097B7FF1F9387871C71
:10A9B0009C4303C5C700828097B7FF1F9387871BFF
:10A9C0009C4303C5D700828097B7FF1F9387871AE0
:10A9D0009C4303C5E700828097B7FF1F93878719C1
:10A9E0009C4303D50701828097B7FF1F9387871881
:10A9F0009C4303C52701828097B7FF1F9387871762
:10AA00009C4303D54701828097B7FF1F9387871622
:10AA10009C4303D56701828097B7FF1F93878715F3
:10AA20009C4303D58701828097B7FF1F93878714C4
:10AA30009C4303C5A701828097B7FF1F93878713A5
:10AA40009C4303C5B701828097B7FF1F9387871286
:10AA50009C4303C5C701828097B7FF1F9387871167
:10AA60009C4303C5D701828097B7FF1F9387871048
:10AA70009C438857828097B7FF1F9387A70F9C43FB
:10AA800003D5C702828097B7FF1F9387A70E9C4309
:10AA900003D5E70219E11305800C828097B7FF1FE9
:10AAA0009387470D9C4303C50703828097B7FF1F19
:10AAB0009387470C9C43C85B828097B7FF1F93879F
:10AAC000E70A8843828097B7FF1F9387670A884306
:10AAD000828019E17D558280F5DE984265DFFDD9DF
:10AAE00017B7FF1F1307072C1847AA877155058B47
:10AAF000631D072403C507001547E37DA7FC03C7B3
:10AB000037001305F0057D171377F70FE364E5FCB5
:10AB100003C35700E30003FC83C86700E38C08FA13
:10AB200003C77700494579171377F70FE364E5FA10
:10AB300003C7A70011481305F7FF1375F50FE36B63
:10AB4000A8F803CE97000D481305FEFF1375F50F07
:10AB5000E362A8F803C8B700630908006518137812
:10AB6000F80F1305600DE36705F703C5C7007948C3
:10AB700079151375F50FE36FA8F403C8D7000D45D9
:10AB80007D181378F80FE36705F503D80701930ED6
:10AB900040175118420813580801E3ED0EF303C89B
:10ABA000E7007D181378F80FE36605F303C8270163
:10ABB0007D181378F80FE36F05F103C88700C54EC1
:10ABC00075181378F80FE3E70EF103D86701856E67
:10ABD000938EBEE06D18420813580801E3EC0EEFA7
:10ABE00003D847016D18420813580801E3E40EEF3B
:10ABF00003D887017918420813580801E36C05ED62
:10AC000003C8A7017D181378F80FE36505ED03C5A8
:10AC1000B7011D487D151375F50FE36DA8EA03C54F
:10AC2000D701714879151375F50FE365A8EA03D5C7
:10AC3000E7011308E00F7D1542054181E36CA8E8A8
:10AC400003C50702494879151375F50FE364A8E8B1
:10AC5000C85301C937C834005915130858BFE36BEE
:10AC6000A8E603A8870237C53400130555BF591855
:10AC7000E36205E717B5FF1F232CC5EE03C60501E8
:10AC800017B5FF1F2328F5EE0545E375C5E403D886
:10AC90002501D04933760603E31E06E203C61501FB
:10ACA000E30A06E217B6FF1F2322B6EC83C527008E
:10ACB00001466387A50003C61700F1453306B602B7
:10ACC00083C707039305C00272971A071307C705C6
:10ACD00016031A9796084697B387B70241553E97D1
:10ACE0003297420741836362E8061773FFFFE7026A
:10ACF000C33B368597800000E780A068970001007D
:10AD0000E78020482A8497A00000E780805A2A9490
:10AD100097F00000E78060262A9497900000E78073
:10AD2000A0812A9497F0FFFFE780E06F2A94974074
:10AD30000000E78060932A9497700000E780A09C51
:10AD400022951773FFFF6700833882801773FFFF18
:10AD5000E702A3354111A307A10097A00000E780F7
:10AD6000A0C59305F100170500001305E5B597F0A0
:10AD7000FFFFE780802F014541011773FFFF670048
:10AD800003351773FFFFE702C32F17B4FF1F130428
:10AD900064010328840079599368180097B4FF1F51
:10ADA00023A614011378180063100802BA84BE8920
:10ADB000368B328A2E89AA8A97F0FFFFE780E0A7B8
:10ADC0007D15269519E531594A851773FFFF6700F0
:10ADD000C32E97F0FFFFE78040A67D152695A1675B
:10ADE000E353F5FE97B7FF1F9387C73298433E8C16
:10ADF000814B01CB014597F00000E7802044933B55
:10AE000015004A85DA865686D28597900000E7803D
:10AE1000C04D2A8911CD1C44F99B17B7FF1F23276A
:10AE2000F7F883270C00CDD3E3800BFA829769BF34
:10AE3000268597B7FF1F23A907F697F0FFFFE78046
:10AE4000809C4146CE8517B5FF1F130525FF97301F
:10AE50000100E780C05697D00000E78040990325A5
:10AE6000040B97D00000E780009D054597D00000B7
:10AE7000E78000A4054597000000E78060EDA9B7D2
:10AE800097B7FF1F938707F29C47858BEDC7177312
:10AE9000FFFFE702832117B5FF1F130565F897B77A
:10AEA000FF1F23A107F097B7FF1F23AF07EE97B748
:10AEB000FF1F23AD07EE97200100E7802081975008
:10AEC0000000E780E0F597100100E780A04C9710A4
:10AED0000100E780A05297B7FF1F938727EB9C43A1
:10AEE00091C7054597800000E780402097B7FF1F76
:10AEF000938787D39C4399C741657D159770000060
:10AF0000E78040A297F00000E780E03D97D0000086
:10AF1000E780808F97B7FF1F9387C7FD9C431397E8
:10AF200017016356070097F00000E78000AD97B760
:10AF3000FF1F23A507F097B7FF1F23A307F097B7BD
:10AF4000FF1F23A107F097B7FF1F23AF07EE97005E
:10AF50000000E780008C97000000E780007297F007
:10AF6000FFFFE780401897F00000E78040D6177396
:10AF7000FFFF6700C315828097B7FF1F938787E2A3
:10AF8000884382801773FFFFE70223129780000037
:10AF9000E780607597800000E780C0771773FFFF38
:10AFA0006700E3121773FFFFE702830E2A849304FE
:10AFB000140201112E85B289A685214636C63A892A
:10AFC00097300100E780403D0DE9B24638082686FB
:10AFD000CE851305940497500000E7806041214618
:10AFE0002C084A8597300100E780003B1335150097
:10AFF00005611773FFFF6700E30C0145D5BF1773A9
:10B00000FFFFE702830A9305450617B5FF1F1305E7
:10B01000A5B697100100E78020691773FFFF67004E
:10B02000030B1773FFFFE702430841112EC697F089
:10B03000FFFFE780601BB24588C141011773FFFF26
:10B040006700E3081773FFFFE7028304AA842E84D6
:10B0500097800000E780006CAA89854522859700CB
:10B060000000E780E07D83C7E4011389940899E339
:10B0700013890403CE85228597000000E780407C79
:10B08000214693051902228597000000E780607829
:10B0900097B7FF1F938707D18C4322859710000035
:10B0A000E780C082214693858402228597000000B4
:10B0B000E78020761773FFFF6700C3001773FFFF59
:10B0C000E70223FC397197F00000E780E0B49305B4
:10B0D000400661E997800000E78000606302051484
:10B0E00097B7FF1F83C707AB13B7170097B6FF1FAC
:10B0F0002382E6AA014499CFC16417B9FF1F13093F
:10B1000069CA9309400EFD1497000000E780C086CD
:10B110006342A40A97F0FFFFE780000D4169B72959
:10B120000900096AFD7A2A8B81447D199389F97B8C
:10B13000130A0A71938A8AC797000000E780C083C8
:10B1400063D7A4041304400EB387840217B7FF1F0C
:10B15000130747C50324070B3E948357C40163823A
:10B16000270B18403307EB4063EAE90083474400AC
:10B170008507B3874703D6976365F708014681457E
:10B18000094597F0FFFFE780604EAA8B29E59740BD
:10B190000000E780808385476317F50689659385FE
:10B1A000057117B5FF1F1305259D97100100E78056
:10B1B000A04F95A0B30734030327090BBA9703D711
:10B1C000C7016308970003C75700A38207002382C3
:10B1D000E700050415BF9305C50022859700000010
:10B1E000E78080E65E852286976501009385452588
:10B1F00097F0FFFFE780E0525E8597100000E78040
:10B20000608A850415BF97B7FF1F9387A7B99C472E
:10B210008D83858BC1F721611773FFFF6700E3E919
:10B2200001468545094502D002D202D402D697F0E4
:10B23000FFFFE780A043AA8479DD97F00000E78054
:10B24000E09C1389C4002A8481454A859700000048
:10B25000E780005F0C4041464A8597000000E78088
:10B26000405B832944006385090C4E8502D802DACD
:10B2700002DC02DE97300100E78060402ACE141025
:10B2800005462C0808184ECC97500000E780E00ACD
:10B290001375F50F51ED8355840093E525004A851C
:10B2A00097000000E780E05E11460C104A85970089
:10B2B0000000E78000560146976501009385C51898
:10B2C000268597F0FFFFE780C045268597000000A0
:10B2D000E780407D5C40A1D3014685450D4597F050
:10B2E000FFFFE780A038AA841DD548401389C40019
:10B2F00097300100E780A0382AC64A8597000000F1
:10B30000E780404C3246636FC5004C404A85970049
:10B310000000E780005001468145268597F0FFFF39
:10B32000E7802040268597000000E780A077E5B5FC
:10B3300083558400ADB71773FFFFE70203D797B7B4
:10B34000FF1F938727A69C471DC193E7870017B56A
:10B35000FF1F1305658217B7FF1F2329F7A4971056
:10B360000100E78040321773FFFF670043D6DD9B83
:10B3700017B7FF1F232CF7A297300000E780E06487
:10B380007DF117A5FF1F1305257F97100100E780AA
:10B39000E033D1BF1773FFFFE702A3CE4169AA894B
:10B3A0002E8AB28A368BBA8B814417BCFF1F130CCE
:10B3B0006C9F930C400E7D1997F0FFFFE780C05BF8
:10B3C00063C4A40001443DA03384940383270C0B81
:10B3D0003E948357C401638627055A87D6865286D2
:10B3E000CE851305040397000000E780E0BB01C988
:10B3F00023800B0022851773FFFF670003CC834770
:10B40000F40185C35A87D6865286CE8513059408E3
:10B4100097000000E78040B909C585472380FB00FD
:10B42000D1BF850451BF835745006380071E177342
:10B43000FFFFE702E3C501112A8497000000E780BF
:10B44000C04D09C985476309F50605611773FFFFFC
:10B45000670043C797E00000E780007C7DF58357D5
:10B4600044004947ED9BE392E7FEC14522859700E2
:10B470000000E7804033AA84228597000000E7801F
:10B48000204F0357440002CE91472A89631AF700E0
:10B49000228597000000E780A0513C082ACC3ECED0
:10B4A00097E00000E78080765C55C5D374084A8633
:10B4B000A6850545829751BF03574400D147E3F65F
:10B4C000E7F8032A0400C169014997BAFF1F938A6C
:10B4D0006A8D130B400EFD1997F0FFFFE780C049FE
:10B4E000634FA90E2285032A040097000000E7801D
:10B4F000C042A1452A89228597000000E780A02A42
:10B50000AA84228597000000E780804A14402A869A
:10B51000AA8978082685CA8597000000E780C0E7D9
:10B52000AA8405D503C7F40189476315F70083474B
:10B53000C10181DF5546D285138564009730010033
:10B54000E780E0E7014597800000E780C01901C56A
:10B5500083D7C401A5E797B7FF1F9387A7849C47AC
:10B5600093551900858913D73700058B01CF89833F
:10B57000858B6399B70001452EC697000000E780D0
:10B58000C0DBB2454E8597800000E780601F034610
:10B59000C1012A8493751900268597900000E780E1
:10B5A000E03935C1268597800000E780E0182685C0
:10B5B00011C0014597800000E780004C97300000E3
:10B5C000E780A0408547E312F5E883C754001307DE
:10B5D000F00FE38CE7E68507A382F400BDB5B30462
:10B5E000690383A70A0BBE9483D7C401638B370119
:10B5F0005546D2851385640097300100E780C0D995
:10B6000055DD0509D1BD5DD86DB782801773FFFF89
:10B61000E70203A897800000E780000C05C1C16421
:10B62000014417A9FF1F1309E9779309400EFD1480
:10B6300097F0FFFFE7804034634EA40017A5FF1F7B
:10B640001305855397100100E780E0031773FFFF90
:10B65000670043A7330534038327090B3E958357BF
:10B66000C501638897002312050097800000E780DA
:10B67000A00C050475BF97A7FF1F9387A7729C476F
:10B680008D83858B8DE31773FFFFE70203A217A558
:10B69000FF1F1305654E97100100E7802003177305
:10B6A000FFFF6700C3A282801773FFFFE702E39FDB
:10B6B000970500009385C5A017A5FF1F1305C54B6F
:10B6C00097100100E78020EE1773FFFF670023A0AB
:10B6D0001773FFFFE702639D8841B7E70400BC5B77
:10B6E000050542054181829709C585472300F5007C
:10B6F00005051773FFFF6700839D83C7F5FF2E8540
:10B700008507A38FF5FE828083C7F5FFFD1793F7AA
:10B71000F70FA38FF5FE99EF1773FFFFE702E3988A
:10B72000B7E70400BC571385F5FF82971773FFFF37
:10B730006700E39982801C41035745008D8FBA95BD
:10B740001CC12312B5003E85828093D78500A205D7
:10B750001441DD8D835745001387E6FF18C1890723
:10B760002312F50013D685004111238FB6FEA38F57
:10B77000C6FE4101828018419307F7FF1CC1835721
:10B78000450085072312F500A30FB7FE828083577B
:10B7900045008D8F2312F5001C41BE950CC12E85EE
:10B7A0008280AA8703D7470008410D8FAA9523926C
:10B7B000E7008CC38280184108453305A74082808A
:10B7C00083574500035765001D8F1C41084533858D
:10B7D000A7403305A74082801773FFFFE702E38C81
:10B7E00041112EC62A8497000000E780A0FDB245D3
:10B7F0006373B50001A0835744000840BE9523122F
:10B80000B4003E9541011773FFFF6700438C177327
:10B81000FFFFE702838941112E84B28532C697006B
:10B820000000E780A0FB3246A28597300100E78048
:10B8300000B941011773FFFF670063891773FFFFAA
:10B84000E702A3862E84854597000000E78000F973
:10B85000230085001773FFFF670063871773FFFFDF
:10B86000E702A38441112317B10089459700000026
:10B87000E780C0F68347E1002300F5008347F1002D
:10B88000A300F50041011773FFFF6700438417739E
:10B89000FFFFE702838193D78500A2054111DD8D6B
:10B8A0002317B100894597000000E78020F3834704
:10B8B000E1002300F5008347F100A300F5004101FA
:10B8C0001773FFFF6700A3801763FFFFE702E37DA5
:10B8D0001397850193D78501C166938606F0D98FAA
:10B8E00013D78500758FD98FA2053707FF00F98D13
:10B8F0004111DD8D2EC6914597000000E78000EED6
:10B900006C00114697300100E78060AB410117637E
:10B91000FFFF6700C37B1763FFFFE70203791C414A
:10B92000854503C4070097000000E78080E6228574
:10B930001763FFFF6700A3791763FFFFE702E37652
:10B940001C414111894503C7070083C7170023071E
:10B95000E100A307F10097000000E78080E30355B2
:10B96000E10041011763FFFF670063761763FFFF84
:10B97000E702A3731C414111894503C7070083C730
:10B9800017002307E100A307F10097000000E780FC
:10B9900040E08357E100410113D58700A2075D8D88
:10B9A000420541811763FFFF670063721763FFFF62
:10B9B000E702A36F0C4141112A84114668009730B9
:10B9C0000100E780C09F9145228597000000E78035
:10B9D00040DCB247C166938606F01397870113D502
:10B9E0008701598D13D78700758F598DA2073707A7
:10B9F000FF00F98F5D8D41011763FFFF6700236D25
:10BA00001C45BE950CC18280AE87944391E6584197
:10BA100001EF0CC15CC1828003C757001367170098
:10BA2000A382E700B687D5B70CC3EDB7AA87084154
:10BA300019CD1841D44398C36313D500D8C32A87BE
:10BA4000034657009376160081E623200700828084
:10BA5000944381CA8C4203A847008CC363930601B8
:10BA6000CCC3799A14C3A302C7003687D1BF1C4543
:10BA7000DC471D8DB777DBB6938777DB0985330508
:10BA8000F502420541818280F147B385F5024845C0
:10BA90002E9582808347450085072302F50082802A
:10BAA0001763FFFFE70263602A8409E41763FFFF5F
:10BAB0006700E36183474400F5DBFD1793F7F70F59
:10BAC0002302F400E5F71C4403D727000507239160
:10BAD000E700DC4399C3228582974C4889CD834790
:10BAE0005400898B99E71C4422859C479C439C47C2
:10BAF0008297232A04000040232004007DB71763A7
:10BB0000FFFFE702835A8357250041112EC681EBC0
:10BB10000144228541011763FFFF6700435B035720
:10BB200005008147F146E305F7FEB385D70240459E
:10BB300085072E948345440008C4F5F5B247AA84CE
:10BB400081E7232A040009A81C456C0022859C4338
:10BB50009C43829748C84DDD85472312F400B247C5
:10BB600023200400231804002319F4005C485CC45B
:10BB700083D72400FD172391F40061BF1763FFFFF3
:10BB8000E702A35297A7FF1F938707018843232645
:10BB9000050023240500410597100100E78000B34C
:10BBA0001763FFFF6700A3521763FFFFE702E34F2E
:10BBB00017A4FF1F130444FE1C40411199CF9C475A
:10BBC0002300B5002AC65CC197000000E78040FB57
:10BBD0001C40DC4399C33245829741011763FFFF44
:10BBE0006700E34E0347450029E3584DAA877D557A
:10BBF0001DCF1763FFFFE702434B1CC3DC4797A62B
:10BC0000FF1F23ABE6F8F156130507012390D70079
:10BC1000970500009385050297100100E780A09822
:10BC200001451763FFFF6700834A7D55828082804C
:10BC30001763FFFFE7026347011161468145280052
:10BC40009760FFFFE780604997A7FF1F9387C7F4BE
:10BC50009C4328009305F00FDC473EC69700000088
:10BC6000E780C0F405611763FFFF6700434697A7AD
:10BC7000FF1F938767F29C43D847A1679387C7024A
:10BC8000631EF70A397106DE22DC26DA80004AD804
:10BC90004ED652D456D23285B28497000000E78047
:10BCA000C0C7AA89268597000000E78020C923180D
:10BCB000A4FC268597000000E78040C82319A4FC57
:10BCC000268597000000E78060C783D744000A8A72
:10BCD000231AA4FC858393F7F70F230EF4FC860741
:10BCE000BD0793F7073F3301F1408A8A0149834733
:10BCF000C4FD6367F902CE85130584FC232C54FD33
:10BD000097000000E78080EA5281130104FCF250A2
:10BD10006254D2544259B259225A925A21618280B5
:10BD2000268597000000E78060C193171900D69719
:10BD300005092390A7001379F90F55BF828097A7B3
:10BD4000FF1F938767E59C43D847A1679387A702A6
:10BD5000631AF70A397106DE22DC26DA80004AD837
:10BD60004ED652D456D23285B28497000000E78076
:10BD7000C0BAAA89268597000000E78020BCFD573D
:10BD80002318A4FC26852319F4FC97000000E78003
:10BD9000E0BA83D744000A8A231AA4FC858393F768
:10BDA000F70F230EF4FC8607BD0793F7073F330117
:10BDB000F1408A8A01498347C4FD6367F902CE8551
:10BDC000130584FC232C54FD97000000E78000DE5F
:10BDD0005281130104FCF2506254D2544259B259B8
:10BDE000225A925A21618280268597000000E780BE
:10BDF000E0B493171900D69705092390A70013798B
:10BE0000F90F55BF828097A7FF1F9387E7D89C4300
:10BE1000D847A16789076310F70A397106DE22DC6B
:10BE200026DA80004AD84ED652D456D2328532898C
:10BE300097000000E78060AEAA894A85970000005D
:10BE4000E780C0AF835749000A8A2318A4FC858382
:10BE500093F7F70F230CF4FC8607BD0793F7073F12
:10BE60003301F1408A8A8144834784FD63E7F40209
:10BE7000CE85130584FC232A54FD97000000E7803B
:10BE8000E0D25281130104FCF2506254D254425960
:10BE9000B259225A925A216182804A859700000045
:10BEA000E780C0A993971400D69785042390A70034
:10BEB00093F4F40F55BF828097A7FF1F9387C7CDD8
:10BEC0009C43D847A1679387E704631EF70A39713B
:10BED00006DE22DC26DA80004AD84ED652D456D26C
:10BEE0003285B28497000000E78020A3AA892685C6
:10BEF00097000000E78080A42318A4FC2685970003
:10BF00000000E780A0A3231AA4FC26859700000068
:10BF1000E780C0A283D744000A8A2319A4FC858342
:10BF200093F7F70F230EF4FC8607BD0793F7073F3F
:10BF30003301F1408A8A01498347C4FD6367F902EE
:10BF4000CE85130584FC232C54FD97000000E78068
:10BF5000E0C55281130104FCF2506254D25442599C
:10BF6000B259225A925A2161828026859700000098
:10BF7000E780C09C93171900D69705092390A70066
:10BF80001379F90F55BF828097A7FF1F9387C7C00A
:10BF90009C43D847A1679387C704631AF70A39718E
:10BFA00006DE22DC26DA80004AD84ED652D456D29B
:10BFB0003285B28497000000E7802096AA89268502
:10BFC00097000000E7808097FD572318A4FC268582
:10BFD000231AF4FC97000000E780409683D74400C2
:10BFE0000A8A2319A4FC858393F7F70F230EF4FC28
:10BFF0008607BD0793F7073F3301F1408A8A01495D
:10C000008347C4FD6367F902CE85130584FC232CA6
:10C0100054FD97000000E78060B95281130104FCD1
:10C02000F2506254D2544259B259225A925A216162
:10C030008280268597000000E780409093171900C2
:10C04000D69705092390A7001379F90F55BF828071
:10C0500097A7FF1F938747B49C43D847A167DD0785
:10C060006317F7041763FFFFE70223047971328532
:10C07000328497000000E780408A2AC62285970014
:10C080000000E780A08B2311A10222859700000009
:10C09000E780A088B2452300A1022808970000008D
:10C0A000E780C0B045611763FFFF670043028280ED
:10C0B00097A7FF1F938747AE9C43D847A1679387F5
:10C0C00087046317F7041763FFFFE70203FE797124
:10C0D0003285328497000000E78020842AC62285BA
:10C0E00097000000E78080852311A1022285970038
:10C0F0000000E7808082B2452300A1022808970053
:10C100000000E780A0AA45611763FFFF670023FCDA
:10C11000828097A7FF1F938727A89C43D847A167D2
:10C120009387A7046312F7021763FFFFE702E3F7A1
:10C1300001112800814597000000E78020A70561D4
:10C140001763FFFF6700A3F8828097A7FF1F9387FD
:10C15000A7A49C43D847A167938757026319F702A6
:10C160001763FFFFE70263F40111328597F0FFFFC9
:10C17000E780A07A2308A1008145280097000000ED
:10C18000E780C0A205611763FFFF670043F4828068
:10C1900097A7FF1F938747A09C43D847A167938722
:10C1A000E702631BF7041763FFFFE70203F00111C7
:10C1B0003285328497F0FFFFE7804078AA84228599
:10C1C00097F0FFFFE7808077854709E9228597F0A0
:10C1D000FFFFE78080744205B337A0002800814547
:10C1E000231891003ECA97000000E780209C05615B
:10C1F0001763FFFF6700A3ED828097A7FF1F938758
:10C20000A7999C43D84799476313F7081763FFFF23
:10C21000E702A3E979713285328497F0FFFFE78066
:10C22000C06F2AC6228597F0FFFFE7802071231098
:10C23000A102228597F0FFFFE780206E2301A10273
:10C24000228597F0FFFFE780406DA301A1022285C0
:10C2500097F0FFFFE780606C2302A102228597F030
:10C26000FFFFE780806B2313A102228597F0FFFF79
:10C27000E780A06AB2452314A102280897000000B5
:10C28000E780C09245611763FFFF670043E4828047
:10C2900097A7FF1F938747909C43D847A167938731
:10C2A000C7036313F7081763FFFFE70203E0797121
:10C2B0003285328497F0FFFFE78020662AC6228508
:10C2C00097F0FFFFE78080672310A102228597F097
:10C2D000FFFFE780A0662311A102228597F0FFFFF0
:10C2E000E780A0632302A102228597F0FFFFE78089
:10C2F000C062A302A102228597F0FFFFE780E06100
:10C300002303A102228597F0FFFFE7800061B24579
:10C31000A303A102280897000000E7802089456157
:10C320001763FFFF6700A3DA82801763FFFFE7024E
:10C33000C3D701112A8497F0FFFFE780005EAA842B
:10C34000228597F0FFFFE780605F228597F0FFFF6F
:10C35000E780C05E035744008D4763F7E7002285FE
:10C3600097F0FFFFE780805D228597F0FFFFE78071
:10C37000E05C2800A68597000000E7802083056127
:10C380001763FFFF6700A3D497A7FF1F9387C7809A
:10C390009C43D847A167FD07631FF7001763FFFFA2
:10C3A000E702A3D0328597000000E78040F81763CA
:10C3B000FFFF6700C3D182809797FF1F9387C77DD8
:10C3C0009C43D847A167E5076315F7081763FFFF8C
:10C3D000E702A3CD79713285328497F0FFFFE780C1
:10C3E000C0532AC6228597F0FFFFE780205522859B
:10C3F00097F0FFFFE78080542310A102228597F079
:10C40000FFFFE780A053520551812311A10222852D
:10C410002302010297F0FFFFE7802050A302A10250
:10C42000228597F0FFFFE780404F2303A10222857A
:10C4300097F0FFFFE780604EB245A303A1022808F2
:10C4400097F0FFFFE780807645611763FFFF670085
:10C4500003C882809797FF1F938707749C43D84730
:10C46000A1679387E703631FF7001763FFFFE702E6
:10C47000C3C3328597000000E78060EB1763FFFFBE
:10C480006700E3C482809797FF1F9387E7709C4300
:10C49000D847A16793874704631EF7021763FFFF1E
:10C4A000E702A3C079713285328497F0FFFFE780FD
:10C4B000C0462AC6228597F0FFFFE7802048B24594
:10C4C000280897F0FFFFE780606E45611763FFFF64
:10C4D0006700E3BF82809797FF1F9387E76B9C43BA
:10C4E000D847A167938787026310F7041763FFFF9C
:10C4F000E702A3BB79713285328497F0FFFFE780B2
:10C50000C0412AC6228597F0FFFFE7800041B2456F
:10C510002300A102280897F0FFFFE780206945610A
:10C520001763FFFF6700A3BA82801763FFFFE7026C
:10C53000C3B7011197F0FFFFE780203EAA852800CE
:10C5400097F0FFFFE780806605611763FFFF6700D4
:10C5500003B89797FF1F938727649C43D847A16729
:10C56000D107631FF7001763FFFFE70203B43285AB
:10C5700097000000E780A0FB1763FFFF670023B56B
:10C5800082809797FF1F938727619C43D847A167B5
:10C59000C507631FF7001763FFFFE70203B132858A
:10C5A00097000000E780A0F81763FFFF670023B241
:10C5B00082809797FF1F9387275E9C43D847A16788
:10C5C000B907631FF7001763FFFFE70203AE328569
:10C5D00097000000E780A0F51763FFFF670023AF17
:10C5E00082809797FF1F9387275B9C43D847A1675B
:10C5F000AD07631FF7001763FFFFE70203AB328548
:10C6000097000000E780A0F21763FFFF670023ACEC
:10C6100082809797FF1F938727589C43D847894765
:10C620006318F7021763FFFFE70223A801113285A1
:10C6300032C897F0FFFFE780402EAA85280097F0C8
:10C64000FFFFE780A05605611763FFFF670023A87F
:10C6500082809797FF1F938727549C43D847A167F1
:10C660008D076311F7041763FFFFE70203A40111AD
:10C670003285328497F0FFFFE780202A130661009D
:10C68000AA844C00228597300000E780C023280050
:10C69000A68597F0FFFFE780605105611763FFFFF4
:10C6A0006700E3A282809797FF1F9387274F9C43E1
:10C6B00081CFDC4391CB1763FFFFE702039F829793
:10C6C0001763FFFF6700A3A082801763FFFFE702E5
:10C6D000C39D79713C08AE843ED2A165B7070A00BC
:10C6E0002A843ED448103C08DD053ED636C432C606
:10C6F0003AC297D0FFFFE780E02F12474810BA8573
:10C7000097F0FFFFE780C01332464810B28597F0DC
:10C71000FFFFE780E014A2464810B68597F0FFFFC0
:10C72000E7800012501001478146A685228597D0E8
:10C73000FFFFE780805145611763FFFF6700239982
:10C740001763FFFFE702639601117C000329C5010F
:10C75000AE843ECAA165B70707002A843ECC4808CC
:10C760007C00C5053ECE97D0FFFFE780A02883451B
:10C77000D900480897F0FFFFE780800C5008014778
:10C780008146A685228597D0FFFFE780004C056192
:10C790001763FFFF6700A3931763FFFFE702E390B0
:10C7A00083C7950093F7F707A384F500970000006F
:10C7B000E78040F91763FFFF670063911763FFFF8E
:10C7C000E702A38E79713C08AE843ED2A165B7071B
:10C7D00009002A843ED448103C08938545043ED67F
:10C7E00032C636C497D0FFFFE780C020A24648106B
:10C7F000B68597F0FFFFE780A00432464810B28567
:10C8000097F0FFFFE780C005501001478146A685DD
:10C81000228597D0FFFFE780404345611763FFFF04
:10C820006700E38A1763FFFFE702238883C7950049
:10C8300041112A8493F7F707A384F50032852EC6A9
:10C8400097F0FFFFE780800F85672AC46370F502C9
:10C8500097700000E78020E92246B24509ED1147B4
:10C860008146228597000000E78060E6410117635A
:10C87000FFFF6700C38501478346F501DDB71763F6
:10C88000FFFFE702E38001113C003ECAB7070A0040
:10C890003ECC3C003ECE83C79500AA89328593F7F3
:10C8A000F707A384F5002E8497F0FFFFE7800009C7
:10C8B0008567637DF504A165AA849385850448088E
:10C8C00097D0FFFFE7800013268597700000E78070
:10C8D00080E12A8929E19145480897F0FFFFE78028
:10C8E00020F6A685480897F0FFFFE78060F7CA8525
:10C8F000480897F0FFFFE780A0F401478146500801
:10C90000A2854E8597D0FFFFE7802034056117533D
:10C91000FFFF6700237B8145480897F0FFFFE78012
:10C9200020F20349090275BF1753FFFFE702437660
:10C9300079711C103ECAB7070F003ECC404D1C1049
:10C94000AA84AE894808994532C636893ECE97D02A
:10C95000FFFFE780200A32464808B28597F0FFFFC4
:10C96000E78000EE630C0902A545480897F0FFFF39
:10C97000E780C0E62546CA8597200100E78020A40D
:10C98000500801478146CE85268597D0FFFFE78076
:10C99000C02B45611753FFFF6700C3728355C40264
:10C9A000480897F0FFFFE780A0EB0355E4028145BC
:10C9B00005C5854785456301F502C167FD179305E8
:10C9C000F00F630BF5007D1597700000E780208E57
:10C9D0009305150093F5F50F480897F0FFFFE780E2
:10C9E00020E683450403480897F0FFFFE78040E511
:10C9F00083451403480897F0FFFFE78060E4835500
:10CA00002403480897F0FFFFE78080E5835544033F
:10CA1000480897F0FFFFE780A0E49DB71753FFFF9A
:10CA2000E702A36883C795008146014693F7F7079D
:10CA3000A384F50097000000E78040EF1753FFFF45
:10CA40006700E3681753FFFFE702236679713E84AE
:10CA50001C103ECA2E89B7070F00A1653ECCFD050C
:10CA60001C10AA84480842C03AC23ECE36C432C620
:10CA700097D0FFFFE78000F832464808B28597F06C
:10CA8000FFFFE780E0DBA2464808B68597F0FFFF8E
:10CA9000E78000DD12474808BA8597F0FFFFE7807E
:10CAA00020DC0248630C08029145480897F0FFFF1C
:10CAB000E780C0D21146A28597200100E780209030
:10CAC000500801478146CA85268597D0FFFFE78039
:10CAD000C01745611753FFFF6700635F894548082A
:10CAE00097F0FFFFE78080CF834704002300F50025
:10CAF00083471400A300F500E1B71753FFFFE702D7
:10CB0000235983C7950001112A8A93F7F707A38455
:10CB1000F5003285AE8432C697F0FFFFE78000E271
:10CB200032462A89328597F0FFFFE78000DF85676C
:10CB30006373F902AA894A8597700000E780A0BA5A
:10CB40002A8419ED114781464A86A68552859700A9
:10CB50000000E780C0B705611753FFFF67008356E9
:10CB60009387E9FF93F7F70F0547E366F7FE8347DF
:10CB7000F50195EB8947E380F9FE8346F401528580
:10CB800001474A86A68597000000E78040B4A16768
:10CB9000D90748083ECC230A010002CE97000000C6
:10CBA000E780A0B04DBF639EE7008947639EF90010
:10CBB00093071020231FF50097700000E780C0B78F
:10CBC0006DBF0947E39BE7FA8D47E398F9FA2285A1
:10CBD00097700000E78080DF9797FF1F9387071B00
:10CBE0009C4399E79797FF1F938707049C4399C736
:10CBF00003D5040097800000E780A0CE231F040027
:10CC000022855DBF1753FFFFE702234A01113C0055
:10CC10003ECAB7070B003ECC3C003ECE83C7950012
:10CC20002A89328593F7F707A384F500AE8497F03D
:10CC3000FFFFE780A0D093170501C187635AF00674
:10CC4000A1652A849385E502480897D0FFFFE78015
:10CC500060DAA285480897F0FFFFE78060C09797E9
:10CC6000FF1F938767FC9C43A9EB01449375F40F66
:10CC7000480897F0FFFFE780A0BC9355844093F5E8
:10CC8000F50F480897F0FFFFE78080BB93550441FC
:10CC900093F5F50F480897F0FFFFE78060BA01476A
:10CCA00081465008A6854A8597D0FFFFE780E0F9C6
:10CCB00005611753FFFF67008341416585460546BF
:10CCC000A2857D1597500000E78060BD59DD5105B4
:10CCD00097000100E780808F1304400633448502EB
:10CCE00071B71753FFFFE702433C0111B707060076
:10CCF0003EC683C7950021642A8993F7F707A3846A
:10CD0000F500AE8428009305A4040AC40AC897D08D
:10CD1000FFFFE78020CE300001478146A6854A8587
:10CD200097D0FFFFE78060F297E0FFFFE780801574
:10CD300013049404480822CC230A010002CE970071
:10CD40000000E780809605611753FFFF67002338D6
:10CD50001753FFFFE702C333C1642A89014497993F
:10CD6000FF1F93892904130A8002FD1497E0FFFF37
:10CD7000E78080C16347A40001451753FFFF6700A8
:10CD80006334B307440303A7C90ABA9703D707005C
:10CD90006306970083D72700638427010504F9B74A
:10CDA0000545E1BF1753FFFFE702832E2A8A2E892C
:10CDB00099C123A0050081498144979AFF1F938A56
:10CDC0002ADE614B97E0FFFFE78040C263C7A40003
:10CDD0004E851753FFFF6700E32E3384640383A758
:10CDE0000A003E948357040099E763040900232056
:10CDF00089008504C1BF4146D285130544009710C0
:10CE00000100E780605975F5A289E5B71753FFFF68
:10CE1000E702032839717C083ED4B7070A003ED6E2
:10CE20007C083ED883C795002A8A328593F7F70796
:10CE3000A384F5002E8932C697F0FFFFE78000B08B
:10CE400085676373F5083246AA84328597F0FFFF41
:10CE5000E780A0AC8547AA8963E8A706A16593850A
:10CE60008504281097D0FFFFE780C0B8268597700B
:10CE70000000E78040872A8429ED9145281097F02B
:10CE8000FFFFE780E09BA685281097F0FFFFE78073
:10CE9000209DCE85281097F0FFFFE780609A01471C
:10CEA00081463010CA85528597D0FFFFE780E0D9D0
:10CEB000A1679387770448183EDC230A010202DE4B
:10CEC00097F0FFFFE780607E21611753FFFF670047
:10CED000631F8145281097F0FFFFE7806096A685C5
:10CEE000281097F0FFFFE780A0979797FF1F938781
:10CEF00027229C4381CB22856389090097D00000BB
:10CF0000E78040248345040271B797D00000E78092
:10CF1000C022CDBF1753FFFFE702831783C79500D9
:10CF20004111AA8993F7F707A384F5003285AE84EF
:10CF3000328A97F0FFFFE78060A08567637FF50284
:10CF40002A8997600000E780007A2A84914631C5DB
:10CF50008347F50105476387E70291C70D4763667D
:10CF6000F704AD461DA89305050303250A004146B5
:10CF700097100100E78040420DE941011753FFFF80
:10CF8000670043149305950803250A00414697104E
:10CF90000100E7806040814669F54A86A6854E8596
:10CFA00097000000E780C081C9BF83250A001305F0
:10CFB000940897700000E780A02919C1C146F1BF0D
:10CFC0009797FF1F938787DC9C4399E79797FF1FED
:10CFD000938787C59C4399C7228597800000E78087
:10CFE000208A69FD8547A30FF400228597B00000D1
:10CFF000E7806084228597600000E780E0734E85BB
:10D0000081464A86A68597F0FFFFE780607BA1678F
:10D010009387570448003EC42302010002C697F0DC
:10D02000FFFFE780806891BF1753FFFFE7026305AA
:10D0300083C795004111AA8993F7F707A384F500E8
:10D0400032852E89B28A97F0FFFFE780208F8567AF
:10D050006374F50EAA8497600000E780C0682A8494
:10D060000DED416B014A979BFF1F938BABD3130CC4
:10D07000400E7D1B19A833048A0383A70B0B3E9433
:10D080008357C40163836705050A97E0FFFFE780C4
:10D09000A08EE342AAFE95460DA08357C501639674
:10D0A00097029305050303A50A0041469710010066
:10D0B000E780802E994611E181462686CA854E85F5
:10D0C00097F0FFFFE780C06F85A883A50A001305CE
:10D0D000040397700000E780A017C14679FD228500
:10D0E000231E940097A00000E780E07422859760DB
:10D0F0000000E78060649797FF1F938767019C4358
:10D10000A9C323000402228597D00000E78040F0E5
:10D110004E8581462686CA8597F0FFFFE780406AE4
:10D12000A1679387070448003EC42302010002C69A
:10D1300097F0FFFFE780605741011753FFFF67003B
:10D14000C3F789472300F402E1B7397106DE22DC18
:10D150004AD8800052D456D25AD026DA4ED65ECE65
:10D160002E8A32892A8B97D0FFFFE780E07D060563
:10D17000710541998A8A3301A140232224FC23149A
:10D1800004FC97D0FFFFE780207C83479A000605C8
:10D19000350593F7F7072315A4FCA304FA004A8585
:10D1A000232624FC97E0FFFFE780407993170501D1
:10D1B000C1876340F0025681130104FCF2506254AF
:10D1C000D2544259B259225A925A025BF24B21610F
:10D1D0008280AA844A8597E0FFFFE7802076AA89AB
:10D1E0004A8597E0FFFFE7806075A1659385C502DA
:10D1F0002A89130544FC97C0FFFFE780A07F26859E
:10D2000097C0FFFFE780E073854511C94A86CE8548
:10D2100097C0FFFFE780606DAA8B21E98945130560
:10D2200044FC97E0FFFFE780A061A685130544FC5E
:10D2300097E0FFFFE780C062CE85130544FC97E0CE
:10D24000FFFFE780E061CA85130544FC97E0FFFF1C
:10D25000E780006101478146130644FCD2855A8568
:10D2600097D0FFFFE780609EB9B78145130544FC66
:10D2700097E0FFFFE780C05CA685130544FC97E0BC
:10D28000FFFFE780E05DCE85130544FC97E0FFFFDC
:10D29000E780005DCA85130544FC97E0FFFFE78047
:10D2A000205C814497D0FFFFE780006AE3D4A4FAB2
:10D2B00083A70B0113971400BA9783D5070099C56C
:10D2C000130544FC97E0FFFFE78080598504D9BF30
:10D2D000797106D622D44AD000184ECE52CC56CA06
:10D2E00026D25AC8AE893289AA8A97D0FFFFE78032
:10D2F000A0650605690541990A8A3301A140232AE0
:10D3000024FC231C04FC97D0FFFFE780E06383C765
:10D31000990006052D0593F7F707231DA4FCA384A8
:10D32000F9004A85232E24FC97E0FFFFE780006187
:10D3300093170501C187634FF0005281130104FD6B
:10D34000B250225492540259F249624AD24A424B94
:10D3500045618280AA844A8597E0FFFFE780005EEE
:10D36000A1659385A5022A89130544FD97C0FFFF97
:10D37000E7804068268597C0FFFFE780805C854591
:10D3800009C9CA8597C0FFFFE78020592A8B29E188
:10D390008945130544FD97E0FFFFE780604AA685B5
:10D3A000130544FD97E0FFFFE780804BCA85130516
:10D3B00044FD97E0FFFFE780A04A0147814613063E
:10D3C00044FDCE85568597D0FFFFE7800088B5B72E
:10D3D0008145130544FD97E0FFFFE7806046A68581
:10D3E000130544FD97E0FFFFE7808047CA851305DA
:10D3F00044FD97E0FFFFE780A046814497D0FFFF00
:10D40000E7808054E3DBA4FA83270B011397140011
:10D41000BA9783D5070099C5130544FD97E0FFFF30
:10D42000E78000448504D9BF1753FFFFE702E3C735
:10D4300083474500404DD5EFFD575DC483469400BA
:10D4400009476363D70A0346B400854663EEC608FE
:10D450008306E40063CA06085C45F9562390D700AA
:10D460009787FF1F83C7077499E3A304E400978796
:10D47000FF1F9387677B9C4381E78947A306F400DE
:10D480009797FF1F9387C7C89C4381E78947230667
:10D49000F4009705000093854506AA84130504014E
:10D4A00097F00000E7802010FD57231AF40281470F
:10D4B0001CDC01489787FF1F23A2876E9787FF1FF9
:10D4C0009387076E232E040304C0804397D0FFFF89
:10D4D000E780C05161463306C502814522859750D9
:10D4E000FFFFE78080BF81473E851753FFFF67003E
:10D4F00003BEFD57D5BF1753FFFFE70203BB2A84C6
:10D500000355450297600000E780E01D19E5231EE2
:10D5100004001753FFFF670083BB8357E401F5DB6B
:10D52000930504FF174501001305C52B97E0000084
:10D53000E780E014F9BF1753FFFFE70203B72E8916
:10D54000A16541119385E5032A8436C432C6BE84A1
:10D550003AC297C0FFFFE780E04912472285BA85AB
:10D5600097E0FFFFE780C02D32462285B28597E025
:10D57000FFFFE780E02EA2462285B68597E0FFFFF9
:10D58000E780002E630309029145228597E0FFFFA3
:10D59000E780C0241146A68597100100E78020E2AD
:10D5A00041011753FFFF670083B28945228597E049
:10D5B000FFFFE780A02283C704002300F50083C794
:10D5C0001400A300F500E9BF1753FFFFE702E3AD26
:10D5D00083C79500444D054793F7F707A384F500EB
:10D5E0001C42411183C707006367F7062E842A890E
:10D5F000B1C003C7D400630FF7021787FF1F1307DB
:10D60000A762184305C3A386F40097A00000E78033
:10D61000404A83C7D40099E741657D1597400000D3
:10D62000E780403083D72403918B89C797E00000BF
:10D63000E780C0134A85A28597F0FFFFE78080103E
:10D64000A167C10748003EC42302010002C697F04B
:10D65000FFFFE780800541011753FFFF670023A705
:10D660001753FFFFE70263A403D745008D47AA8441
:10D6700041112E8432892E8563E3E70297E0FFFF94
:10D68000E780C02BAA8523000900268597C0FFFFED
:10D69000E780A02841011753FFFF670043A397E0ED
:10D6A000FFFFE780A0292AC6228597E0FFFFE780D9
:10D6B000E028B24585472A862300F900268597C0D1
:10D6C000FFFFE7808022F9B7397106DE22DC26DA17
:10D6D00080004ED652D456D24AD85AD05ECEAE89A9
:10D6E000B284AA8A97D0FFFFE780002506051305BC
:10D6F000250241990A8A3301A140232224FC2314E4
:10D7000004FC97D0FFFFE780202383C7990006051C
:10D710004D0593F7F7072315A4FCA384F90026858C
:10D72000232624FC97E0FFFFE780402193170501A3
:10D73000C1876340F0025281130104FCF25062542D
:10D74000D2544259B259225A925A025BF24B216189
:10D750008280AA8B03AB040097C0FFFFE780601EA6
:10D7600051E583D7440001498544F11793B7170069
:10D77000A301F4FC834734FCA165C9C79385E50484
:10D78000130544FC97C0FFFFE780C026A68513055C
:10D7900044FC97E0FFFFE780A00ADE85130544FC08
:10D7A00097E0FFFFE780C00B834734FC114691E30D
:10D7B0000946DA85130544FC97E0FFFFE780600522
:10D7C0008144630A0900416B7D1B97D0FFFFE7800E
:10D7D000A01663CCA40201478146130644FCCE8503
:10D7E000568597C0FFFFE7804046B1B7A685130670
:10D7F00034FC97000000E780E0E6933415002A89A6
:10D8000086048DBF9385C504A5BF8327C9001397E0
:10D810001400BA9783D5070063886501130544FC9B
:10D8200097E0FFFFE780C003850445B71753FFFF6C
:10D83000E702238579711C103EC4B7070F003EC66E
:10D840001C103EC883C79500AA8A328593F7F70754
:10D85000A384F500AE89328497E0FFFFE780000ED5
:10D8600093170501C187635AF0062A8A228597E03B
:10D87000FFFFE780A00C2A895285032B040097C084
:10D88000FFFFE780000C39ED8357440081440544D5
:10D89000F11793B71700A303F10083457100DA87EE
:10D8A0002287CA865286280097000000E780E0C8D9
:10D8B000014781463000CE85568597C0FFFFE7803F
:10D8C000C038A1679387D70348083ECC230A81005C
:10D8D00026CE97F0FFFFE78040DD45611743FFFF4D
:10D8E0006700A37DA2851306710097000000E78002
:10D8F00060D7AA84094455D13544E30055FB4A85D5
:10D9000097F0FFFFE78000450D4441D9014497D0CF
:10D91000FFFFE7806002634DA400C16B0144FD1B63
:10D9200097D0FFFFE7804001634EA4001544B5B7D0
:10D93000DC4413171400BA9783D7070063832703C7
:10D940000504F1B7D84493171400BA9703D707001A
:10D95000631B770123902701268597A00000E780AD
:10D9600080DB01441DBF050465BF1743FFFFE702CD
:10D97000237283C7950041112A8A93F7F707A3847E
:10D98000F50032852E89328497E0FFFFE78000FBA7
:10D9900093170501C1876353F006AA89228597E092
:10D9A000FFFFE780A0F92311A1004E85832A040020
:10D9B00097C0FFFFE780E0F839E5835744008544CE
:10D9C0000144F11793B71700A300F10003481100B9
:10D9D00003572100D6875285CE862686CA8597F0C2
:10D9E000FFFFE7806006A167F10748003EC42302FD
:10D9F000910022C697F0FFFFE78020CB410117433B
:10DA0000FFFF6700236CA28513061100970000003A
:10DA1000E78040C52A84894455D98357210011677E
:10DA20008544BA97C2071167C1831307F7EFE36F05
:10DA3000F7F89787FF1F938767359C4381CB854510
:10DA40001305210097500000E780207583552100C1
:10DA50002285814497C0FFFFE78040E525D9231048
:10DA60000500228597A00000E78040CD85B71743C9
:10DA7000FFFFE702036183C7950041112A8B93F7EB
:10DA8000F707A384F50032852E8A328497E0FFFFE2
:10DA9000E780C0EA93170501C1876351F006AA8A9F
:10DAA000228597E0FFFFE78060E92A895685832B6E
:10DAB000040097C0FFFFE780C0E831E583574400CA
:10DAC00081440544F11793B71700A301F1000348FF
:10DAD0003100DE875A854A87D6862286D28597F01E
:10DAE000FFFFE78060F6A167ED0748003EC4230210
:10DAF000810026C697F0FFFFE78020BB4101174356
:10DB0000FFFF6700835BA2851306310097000000CA
:10DB1000E78040B5AA8409445DD99167CA97C207D6
:10DB20001167C1831307F7EF0544E362F7FACA856B
:10DB300097C0FFFFE78080D7014451F9814997D012
:10DB4000FFFFE78060E063DBA90098489397190026
:10DB5000BA9703D7070005EF2390270197D0FFFF5F
:10DB6000E78080DE1544E384A9F6268597A00000AF
:10DB7000E780C0BC9787FF1F938747219C430144E0
:10DB8000B9D74A8597500000E780C05889B7850902
:10DB90007DB71743FFFFE702A34F79713E847C08EE
:10DBA0003EC82E8AB7071400A1653ECAE5057C0869
:10DBB000AA89080836C4428932C6BA8AC6843ECCCD
:10DBC00097C0FFFFE78000E3CA85080897E0FFFFE2
:10DBD000E78000C732460808B28597E0FFFFE7807C
:10DBE00020C8A246630A09049D45080897E0FFFF84
:10DBF000E780C0BE1D4681459740FFFFE780E04DAE
:10DC000063890A089145080897E0FFFFE78000BD97
:10DC10001146A68597000100E780607A1008014749
:10DC20008146D2854E8597C0FFFFE780000245619F
:10DC30001743FFFF67000349B685080897E0FFFF19
:10DC4000E78000C21C400808D8439355C701858966
:10DC500012075183B205D98D97E0FFFFE78040C0DE
:10DC60001C40080883C5870097E0FFFFE78040BDA0
:10DC70001C40080883C5A70097E0FFFFE78040BC71
:10DC80001C40080883C5970097E0FFFFE78040BB72
:10DC900085BF8945080897E0FFFFE78020B483C768
:10DCA00004002300F50083C71400A300F500BDB7EE
:10DCB0001743FFFFE702C33D83C795004111AA89BF
:10DCC00093F7F707A384F5003285AE84328497E09A
:10DCD000FFFFE780A0C693170501C187635DF004CD
:10DCE0002A89032A040097C0FFFFE78080C519E94D
:10DCF000835744000548F11793B71700A307F100B5
:10DD0000814631A81306F100A28597000000E78044
:10DD100060951DC51C459DC783D647000148034734
:10DD2000F10093078500D2884A86A6854E85970024
:10DD30000000E78040E641011743FFFF670083389A
:10DD400009487DBF1D486DBF1743FFFFE7024334FD
:10DD500065715C083EC4B7077B013EC65C083EC8DF
:10DD600083C795002A8A328593F7F707A384F500C5
:10DD7000AE8997E0FFFFE78040BA8357E100E1C733
:10DD80008945280097C0FFFFE780C0C6814528006D
:10DD900097E0FFFFE780C0AA97C0FFFFE780A0CC15
:10DDA0009787FF1F9387C7369C431784FF1F034441
:10DDB00064DFAA843334800099C3136424009787F6
:10DDC000FF1F938767E69C4399C3136444009787BA
:10DDD000FF1F9387A7FB9C4399C31364840083D5DB
:10DDE00004002800014997E0FFFFE78060A783D582
:10DDF0002400280097E0FFFFE78080A683D5440039
:10DE0000280097E0FFFFE780A0A597D0FFFFE780FD
:10DE1000A0AE93150501C181280097E0FFFFE780C0
:10DE200020A4A285280097E0FFFFE78060A39C4420
:10DE30006360F902014781463000CE85528597C064
:10DE4000FFFFE78080E059611743FFFF67008327EA
:10DE5000DC441314490028003E9497E0FFFFE7805C
:10DE60006096834744000347540089070607BA9722
:10DE70008607E36AF5FC835524002800814A97E071
:10DE8000FFFFE780E09D83454400280097E0FFFF07
:10DE9000E780009B83455400280097E0FFFFE78060
:10DEA000209A8347440063C9FA00814A834754009B
:10DEB00063C1FA020509A5BF1C4413975A00280044
:10DEC000BA9783D50700850A97E0FFFFE78040995E
:10DED000C9BF032BC40093975A0028003E9B83556B
:10DEE0002B00850A97E0FFFFE780809783550B00A2
:10DEF000280097E0FFFFE780A0964DBF1743FFFF84
:10DF0000E702A31A5C4993E717005CC997A00000D9
:10DF1000E78020B61743FFFF6700631B1743FFFF2F
:10DF2000E702A3182E84814597F0FFFFE780C0E742
:10DF300005C583570500FD172310F50009C4835755
:10DF400025002310F40097000000E78060FB0145E6
:10DF50001743FFFF6700A31731457DD82310040046
:10DF6000C5BF1743FFFFE702A31283C79500411106
:10DF70002A8A93F7F707A384F50032852E89328425
:10DF800097E0FFFFE780809B93170501C1876356E9
:10DF9000F006AA89C145228597E0FFFFE780A080AF
:10DFA0002A8B4E85832A040097C0FFFFE780609983
:10DFB00031E983574400231101000544F11793B759
:10DFC0001700A300F100814403481100035721000A
:10DFD000D6875285CE862286CA8597F0FFFFE780D6
:10DFE000A0A6A1679387170248003EC423028100C0
:10DFF00026C697E0FFFFE780406B41011743FFFF14
:10E000006700430C13061100A28597F0FFFFE7801D
:10E010006065AA8409E523110100094475B79305D9
:10E0200021005A8597000000E78080EF8357210088
:10E030002A84D9DB9787FF1F938747D59C4381CBE1
:10E0400085451305210097500000E7800015835592
:10E0500021002685314497C0FFFFE78020852DD51C
:10E0600023100500268597900000E780206D01446D
:10E07000A1BF1743FFFFE702430341112E896C0044
:10E08000AA8402C697F0FFFFE78000D20DC10357B4
:10E09000050005072310E50097000000E78040E633
:10E0A00081473E8541011743FFFF67004302324726
:10E0B000954765DBCA85268597300000E780400DCF
:10E0C000C147E34005FE3244854741462310F40032
:10E0D00083570900A685130544002311F400970017
:10E0E0000100E780C02D228545BF1743FFFFE702EF
:10E0F00023FA83C795004111AA8A93F7F707A384EF
:10E10000F5003285AE89328497E0FFFFE780008317
:10E1100093170501C1876356F0062A8AC1452285F7
:10E1200097D0FFFFE7802068AA845285032B040064
:10E1300097C0FFFFE780E08031E983574400231157
:10E1400001008544F11793B71700A300F1000144C3
:10E150000348110003572100DA875685D2862686A8
:10E16000CE8597F0FFFFE780208EA1679387070297
:10E1700048003EC42302910022C697E0FFFFE780DB
:10E18000C05241011743FFFF6700C3F3A285130686
:10E19000110097F0FFFFE780E04C2A8409E5231186
:10E1A0000100894475B7268593052100970000007A
:10E1B000E78060ECAA8449FD83552100228597B051
:10E1C000FFFFE780A06E49F5014997C0FFFFE78098
:10E1D000A077635DA900184893171900BA9703D771
:10E1E00007000DEF035721002390E70097C0FFFFC2
:10E1F000E7808075630625039787FF1F938707B91C
:10E200009C4399C70355210097500000E78080F098
:10E21000228597900000E78060521DBF050975B701
:10E2200095443DB705C19307F00F630FF500C5474F
:10E23000630CF5009307F5FF05453315F50042051E
:10E24000418182800145828041657D158280B9E9E6
:10E250001743FFFFE70263E5034506033284970097
:10E260000000E78060FC9305803EB305B502C2055F
:10E27000C18181CD0357E402854763F8E7001305A8
:10E28000040197E00000E78020428357E4024167E1
:10E290007D176385E700FD172317F4021743FFFF7F
:10E2A0006700E3E282801743FFFFE70283DD00425D
:10E2B00083C79500444D0349140093F7F707A384DF
:10E2C000F50083470400220911673369F900A1674B
:10E2D000B347F90041112A8BAE8A63ECE70E8347FE
:10E2E00024001307C00EB91793F7F70F6373F710E5
:10E2F00003473400C14763EEE70E8347440013072A
:10E30000E00793C707086371F70C834984008347CC
:10E310007400A209B3E9F900856763F7F90A034AB3
:10E320006400834754004E85220A336AFA009750EE
:10E330000000E780403B61C123962403834B3400F7
:10E34000137AFA00239A340323887403239944032D
:10E3500093890401631C090023A604022398040284
:10E360004E8597E00000E78060363DA00349240019
:10E370004A8597000000E78020EB2397A40283479B
:10E3800044004E85A388F402E38D0BFCE30B09FCEB
:10E3900097E00000E780202F97900000E78000734F
:10E3A00081460146D6855A8597E0FFFFE7800058F1
:10E3B000A167938797033EC423020100480002C669
:10E3C00097E0FFFFE780602E41011743FFFF6700E2
:10E3D000C3CE8544A2862686D6855A8597E0FFFF60
:10E3E000E780C054A167938797033EC4230291003E
:10E3F000F1B7BD44C5B79144F1BF1743FFFFE70232
:10E4000023C901111C08404D3EC2B7070F003EC48E
:10E410001C083EC62A89AE8997C0FFFFE780A0DAB4
:10E42000585C1C5C6346B70E6394E50063E2A70E7C
:10E430003385A740B3B7A700B305B7401306803EA6
:10E4400081469D8D97000100E78080B793140501F8
:10E45000C180A1659385C503480097B0FFFFE780A1
:10E4600060598145480097D0FFFFE780603D8355A4
:10E470000404480097D0FFFFE780803E83552404C2
:10E48000480097D0FFFFE780A03D814589CCC16758
:10E49000FD179305F00F6388F40026859750000060
:10E4A000E780E0E0AA85480097D0FFFFE780403989
:10E4B00003554404814501CDC167FD179305F00F55
:10E4C0006307F50097500000E78060DEAA854800EA
:10E4D00097D0FFFFE780C03683456404480097D09B
:10E4E000FFFFE780E03583457404480097D0FFFFC5
:10E4F000E7800035500001478146CE854A8597B0B8
:10E50000FFFFE780807405611743FFFF670083BB4F
:10E51000814481B71743FFFFE70223B983C7950002
:10E5200093F7F707A384F50097000000E78020ED3C
:10E530001743FFFF6700A3B91743FFFFE70243B587
:10E5400083C795004111404D93F7F707A384F50069
:10E550002A8A3285B284AE8997D0FFFFE780003ED9
:10E560002A8B268597D0FFFFE780403D2A892685A4
:10E5700097D0FFFFE780603A93170B0163CA070249
:10E58000E177CA97C207C183116763E3E702930784
:10E590000910C207C1831307B00F637BF7009317FD
:10E5A0000901C187AA8A634AF000C54763FE570183
:10E5B00041011743FFFF6700E3B097B0FFFFE7801B
:10E5C000C028E31725FFD5B763080B0263060902CD
:10E5D000814463890A02B7077F0023106405231171
:10E5E00024057CC0568597000000E780E0C39304B3
:10E5F000803EB304950239A0B7077F0023200404AE
:10E600007CC081440355240497E00000E780A0A368
:10E61000A1C497C0FFFFE78000BB269593D7F441C4
:10E6200033379500AE97BA9708DC5CDCCE8552850F
:10E6300097000000E780A0DC99E023220404A16792
:10E640009387B70348003EC42302010002C697E047
:10E65000FFFFE7808005A9BF814701481CDC232E0E
:10E660000403E9B71743FFFFE70223A497C0FFFFA6
:10E67000E780C037E1473305F50291459750000028
:10E68000E78000C5E55711C59777FF1F23AAA7505C
:10E6900081473E851743FFFF670063A385471777D0
:10E6A000FF1F2301F75082801743FFFFE702E39F1C
:10E6B0009777FF1F9387874E80433DC0835704049D
:10E6C0006390A70683572404639CB7043689B284F9
:10E6D00097C0FFFFE78020AF5C5C63C3B70463951E
:10E6E000B7001C5C63EEA7028347640463F3F40085
:10E6F000A6872303F4048347740463F39700A68773
:10E70000A303F4048357440441677D176385E7003E
:10E7100085072312F4043C4481C7CA852685829765
:10E720001743FFFF6700A39A9777FF1F9387074759
:10E730009C43014599C303C5870082801743FFFFAF
:10E74000E702A3960111B70707003EC683C79500ED
:10E75000584D0AC493F7F7070AC8A384F5002A891D
:10E76000AE8411CB1C4283C707002304F7009790A7
:10E770000000E7800034216493055402280097B01C
:10E78000FFFFE780202797000000E78020FAAA8596
:10E79000280097D0FFFFE780A00A3000014781469C
:10E7A000A6854A8597B0FFFFE780204A13044402FC
:10E7B000480822CC230A010002CE97E0FFFFE78041
:10E7C000C0EE05611743FFFF670063901743FFFF2B
:10E7D000E702A38D01117C003ECAB70707003ECCBB
:10E7E0007C003ECE83C795002E84AA8493F7F7075A
:10E7F000A384F500A16593855502480897B0FFFFF3
:10E80000E780401F97000000E78040F2AA85480893
:10E8100097D0FFFFE780C002500801478146A285DC
:10E82000268597B0FFFFE780404205611743FFFF51
:10E830006700E3899777FF1F938747369C43094515
:10E8400099C303C5970082809777FF1F9387073589
:10E850009C43094599C303C5D70082809777FF1F62
:10E860009387C7339C43014599C303C5A7008280A2
:10E870001743FFFFE702C3810111B70708003EC637
:10E8800083C79500404D0AC493F7F7070AC8A384CD
:10E89000F5002A89AE8429C41442854703C70600BF
:10E8A00063E0E70A83479400094681496380C70211
:10E8B000B307F740A304E400B339F00083C71600A0
:10E8C0002305F40097900000E780A01E035724035F
:10E8D000058B19C76386090097D00000E78000E91F
:10E8E000216493058402280097B0FFFFE780801021
:10E8F00097000000E78040F4AA85280097D0FFFF2A
:10E90000E78000F497000000E78080F5AA852800E2
:10E9100097D0FFFFE780C0F2014781463000A6850F
:10E920004A8597B0FFFFE78040321304740248081D
:10E9300022CC230A010002CE97E0FFFFE780E0D659
:10E9400005611733FFFF6700E3771733FFFFE70227
:10E95000C37501117C003ECAB70708003ECC7C009D
:10E960003ECE83C795002E84AA8493F7F707A3842D
:10E97000F500A16593858502480897B0FFFFE78001
:10E98000600797000000E78020EBAA85480897D031
:10E99000FFFFE780E0EA97000000E78060ECAA85CF
:10E9A000480897D0FFFFE780A0E95008014781465B
:10E9B000A285268597B0FFFFE780202905611733E0
:10E9C000FFFF6700C3709777FF1F9387271D9C4346
:10E9D000014599C303C5B70082801733FFFFE702E3
:10E9E000C36C0111B70707003EC683C79500404DB1
:10E9F0000AC493F7F7070AC8A384F5002A89AE84EE
:10EA000005C81C42054783C707006368F70603472C
:10EA1000B400630FF700A305F40097900000E780AF
:10EA200040098347B400B9CF97D0FFFFE78040BECD
:10EA300021649305B400280097B0FFFFE78080FBB6
:10EA400097000000E78060F8AA85280097D0FFFFB4
:10EA5000E78000DF014781463000A6854A8597B0F0
:10EA6000FFFFE780801E2904480822CC230A01000A
:10EA700002CE97E0FFFFE78040C305611733FFFF39
:10EA80006700E36497D0FFFFE78020BF55B71733D7
:10EA9000FFFFE702836101117C003ECAB707070050
:10EAA0003ECC7C003ECE83C795002E84AA8493F78B
:10EAB000F707A384F500A165AD05480897B0FFFFEF
:10EAC000E78040F397000000E78020F0AA8548081F
:10EAD00097D0FFFFE780C0D6500801478146A28546
:10EAE000268597B0FFFFE780401605611733FFFFCB
:10EAF0006700E35D9777FF1F9387470A9C430945AB
:10EB000099C303C5C70082801733FFFFE702E359AB
:10EB100001117C00AE843ECAA165B70707002A84B4
:10EB20003ECCD1057C0048083ECE97B0FFFFE78081
:10EB300060EC97000000E78020FCAA85480897D089
:10EB4000FFFFE780E0CF500801478146A685228578
:10EB500097B0FFFFE780600F05611733FFFF670085
:10EB600003571733FFFFE702435483C7950093F71A
:10EB7000F707A384F50097000000E78020F917331A
:10EB8000FFFF6700C3541733FFFFE702635083C7DB
:10EB900095000329C501411193F7F707A384F500F8
:10EBA0001C4283C90700854763E637079777FF1F35
:10EBB000938707569C432E84AA8485CF9700000034
:10EBC000E78080F389476306F502630409028347FF
:10EBD000C900638037032306390197900000E7805E
:10EBE00040ED83572903898B89C797D00000E780C0
:10EBF000E0B72685A28597000000E78020F1A16795
:10EC0000CD0748003EC42302010002C697E0FFFF83
:10EC1000E780A0A941011733FFFF6700A34A977758
:10EC2000FF1F9387A7F79C431D4599C303C5E700C2
:10EC300082801733FFFFE70243470111B707070040
:10EC40003EC683C79500584D0AC493F7F7070AC814
:10EC5000A384F5002A89AE8415C71C4283C7070028
:10EC600093968701E18663C4060685466381D706CD
:10EC70008346E7006388F6002307F70097900000BB
:10EC8000E78020E321649305E400280097B0FFFFAC
:10EC9000E78040D697000000E780A0F8AA8528000A
:10ECA00097D0FFFFE780C0B9014781463000A685B5
:10ECB0004A8597B0FFFFE78040F93504480822CC29
:10ECC000230A010002CE97E0FFFFE780009E056166
:10ECD0001733FFFF6700A33F1733FFFFE702E33C53
:10ECE00001117C003ECAB70707003ECC7C003ECE37
:10ECF00083C795002E84AA8493F7F707A384F500B1
:10ED0000A165B905480897B0FFFFE780A0CE97003E
:10ED10000000E78000F1AA85480897D0FFFFE78050
:10ED200020B2500801478146A285268597B0FFFF93
:10ED3000E780A0F105611733FFFF67004339173300
:10ED4000FFFFE702E334AA8401441779FF1F130988
:10ED500029E5E14997C0FFFFE78040C96344A4006B
:10ED6000014519A833053403832709003E958357CD
:10ED700025006397970011051733FFFF6700833461
:10ED80000504C9BF032E8500630A0E121773FF1F07
:10ED90001303C3FF03230300631503002943639098
:10EDA000061203234E01631503001D4363990710E8
:10EDB0001733FFFFE702E32CC689428A3E89BA8AED
:10EDC000B684328BAE8B2A84B5E103554E0019E52B
:10EDD00001431A851733FFFF6700232EA167A98F10
:10EDE000116763FBE70097000000E78080F581452D
:10EDF00097F0FFFFE780C0120844B70700E05841D2
:10EE0000F98F18455CC1B707001FF98F1CC55C4915
:10EE100091C7610597E00000E780408BE38A09FA1B
:10EE2000228597900000E78060C65DB7328597C065
:10EE30000000E78040430D4349DD1C44116703D5C2
:10EE40004700A167A98F63FBE70097000000E780F8
:10EE500040EF814597F0FFFFE780800C032384009B
:10EE600093164B01D1828347B30003566300858814
:10EE7000FD8BA305F300FD777D8E558EFD76FD1687
:10EE8000B204F18E83274301C58E2312730123132D
:10EE9000D3002304530123052301A3044301BDDF51
:10EEA000228597B0FFFFE78020CDAA850844B5D121
:10EEB000610597D00000E780207F8DB71D431A853C
:10EEC00082801733FFFFE702A31C0569AA84AE897D
:10EED000328A0144FD5A7D1997C0FFFFE780C0A523
:10EEE0006347A40001451733FFFF6700A31DD84403
:10EEF00093171400BA9703D70700631F37032390B3
:10EF0000570163070A00268597900000E780A080DC
:10EF10009C449DC383D76700B3F72701639E3701E5
:10EF2000D2880148814701478146014681452685AF
:10EF300097000000E78040E5050479BF1733FFFF25
:10EF4000E702031579711C103EC4B7070F003EC6D7
:10EF50001C103EC883C79500AA8A328593F7F7072D
:10EF6000A384F5002E89328497D0FFFFE780009DAF
:10EF700093170501C187635AF006AA89228597D0A5
:10EF8000FFFFE780A09B2A8A4E85032B040097B0E1
:10EF9000FFFFE780009B39ED83574400814405441F
:10EFA000F11793B71700A303F10083457100DA87C7
:10EFB0002287D2864E86280097E0FFFFE780E05741
:10EFC000014781463000CA85568597B0FFFFE7802C
:10EFD000C0C7A1679387F70348083ECC230A810086
:10EFE00026CE97D0FFFFE780406C45611733FFFFC7
:10EFF0006700430DA2851306710097E0FFFFE780CD
:10F000006066AA84094455D1528597E0FFFFE780E6
:10F0100060D40D4459D90546D28526859700000055
:10F02000E78060EA2A8451B71733FFFFE702E3075E
:10F03000835507000346270041112A842E8532C6D6
:10F040002EC497E0FFFFE780E0D001C93246A24519
:10F05000228597000000E78000E741011733FFFF9A
:10F060006700E3061733FFFFE702A30183C795009C
:10F070004111AA8A93F7F707A384F5003285AE8978
:10F08000328497D0FFFFE780608B93170501C1871B
:10F090006357F00AC1452A8A228597C0FFFFE7809F
:10F0A00080702A8D228597D0FFFFE78020892A89EA
:10F0B000228597D0FFFFE7804086930705F893F7F6
:10F0C000F70F1307E007AA8B637BF706228597D01B
:10F0D000FFFFE78080842A8C228597D0FFFFE7809E
:10F0E000C083AA8C5285032B040097B0FFFFE780F2
:10F0F000408539E983574400231101008144F11709
:10F1000093B71700A300F10005440347110083568D
:10F110002100938784005685DA8822885286CE851E
:10F1200097F0FFFFE78020A7A167E90748003EC4EA
:10F130002302810026C697D0FFFFE78000574101D8
:10F140001733FFFF670063F713061100A28597E0EE
:10F15000FFFFE7802051AA8409E52311010009443B
:10F160006DB7930521006A8597F0FFFFE780A0F057
:10F170002A8441FD835521009356C9001316490185
:10F1800085486688E2875E87858A51822685970052
:10F190000000E78060BF2A848DBF1733FFFFE702BE
:10F1A00043EE83C7950041112A8B93F7F707A38499
:10F1B000F5003285AE89328497C0FFFFE780007882
:10F1C00093170501C1876352F00A2A8A228597C0E6
:10F1D000FFFFE780A076AA8A228597C0FFFFE7801D
:10F1E000E0752A89228597C0FFFFE78000739307A7
:10F1F00005F893F7F70F1307E0072A8C6377F706F4
:10F20000228597C0FFFFE7804071AA8C228597C0B6
:10F21000FFFFE78080702A8D5285832B040097A022
:10F22000FFFFE780007239E58357440085440144BD
:10F23000F11793B71700A301F100034731009307BB
:10F2400084005A85DE882688D6865286CE8597F039
:10F25000FFFFE78040948D4748003EC423029100A1
:10F2600022C697D0FFFFE780404441011733FFFFDC
:10F270006700A3E4A2851306310097E0FFFFE78053
:10F28000603E2A84894455D99356C9001316490112
:10F2900085486A88E6876287858A5182D685970085
:10F2A0000000E78060AEAA8449BF1733FFFFE70282
:10F2B00023DE2A8981440144617A916A177BFF1F0A
:10F2C000130BCBAC97B0FFFFE780006863C7A400C7
:10F2D00022851733FFFF6700E3DE83270900939938
:10F2E0001400CE9703D50700330745014207418339
:10F2F0006364570305C103270B0019C785453E8585
:10F3000097400000E78060E9832709000504CE9755
:10F310002390070085047DB797000000E78060A276
:10F32000832709000504CE972390070065D5814502
:10F3300097F0FFFFE780C0BEF1BF1733FFFFE70282
:10F3400023D583C7950041112A8A93F7F707A38431
:10F35000F50032852E89328497C0FFFFE780005E7A
:10F3600093170501C187635AF004AA89832A040010
:10F3700097A0FFFFE780E05C31E5835744008544B8
:10F380000144F11793B71700A301F10003483100BE
:10F39000D68752850147CE862686CA8597D0FFFF3D
:10F3A000E780806AA167F50748003EC42302910008
:10F3B00022C697D0FFFFE780402F41011733FFFFA0
:10F3C000670043D0A2851306310097E0FFFFE78076
:10F3D00060292A8489445DD99777FF1F9387079B0B
:10F3E0009C4381CF044997B0FFFFE780E055AA8591
:10F3F000268597400000E78040DA13050401970056
:10F400000000E780C0EA228597800000E780003393
:10F410008144ADBF1733FFFFE702A3C683C7950042
:10F420004111AA8A93F7F707A384F5003285AE89C4
:10F4300032842311010097C0FFFFE780205093170B
:10F440000501C1876354F0062A8AC145228597C009
:10F45000FFFFE7804035AA8B5285032B040097A05D
:10F46000FFFFE780004E21E98357440085440144B3
:10F47000F11793B71700A300F100034811000357D9
:10F480002100DA875685D2862686CE8597D0FFFF63
:10F49000E780805BA1679387270248003EC4230270
:10F4A000910022C697D0FFFFE7802020410117334B
:10F4B000FFFF670083C0A2851306110097E0FFFFDE
:10F4C000E780401A2A8489444DD99777FF1F938794
:10F4D000E78B98433E8901CF044997B0FFFFE7804F
:10F4E000A046AA85268597400000E78000CB13053B
:10F4F000040197000000E78080DB97B0FFFFE78002
:10F50000A04495443DD9930521005E8597F0FFFF07
:10F51000E78060B6AA8435F11C4803572100228594
:10F520002390E70097800000E780402183270900AF
:10F53000A9D70355210097400000E780A0BD35BF43
:10F540001733FFFFE702E3B383C795004111AA8A8F
:10F5500093F7F707A384F5003285AE89328497C00C
:10F56000FFFFE780A03D93170501C1876351F006B7
:10F570002A8A228597C0FFFFE780403C2A8952856E
:10F58000032B040097A0FFFFE780A03B31E58357E2
:10F59000440085440144F11793B71700A301F1001B
:10F5A00003483100DA8756854A87D2862686CE857B
:10F5B00097D0FFFFE7804049A167F90748003EC4A4
:10F5C0002302910022C697D0FFFFE780000E410181
:10F5D0001733FFFF670063AEA2851306310097E083
:10F5E000FFFFE78020082A8489445DD99167CA9784
:10F5F000C2071167C1831307F7EF8544E362F7FA87
:10F600009767FF1F938787789843BE8B01CF044984
:10F6100097B0FFFFE7804033AA852685974000001A
:10F62000E780A0B71305040197000000E78020C819
:10F6300097B0FFFFE780403195443DD11C482285BB
:10F6400081442390270197800000E780200F83A743
:10F650000B00B9D74A8597400000E780A0AB89B777
:10F660001733FFFFE70263A42A844105B2849700A1
:10F670000000E780C0C311C5228597800000E780A5
:10F68000E00B81460146A685228597800000E78031
:10F69000C04E1C4C89C7DC4799C32285829717331B
:10F6A000FFFF6700C3A29767FF1F9387274F9C4305
:10F6B000014599C31385070182809767FF1F9387D0
:10F6C000E74D884382801733FFFFE702039E9317BD
:10F6D000C600DD8DC2054111C1812A8432C697C0A2
:10F6E000FFFFE780E0173246228511829375F60FFF
:10F6F00097C0FFFFE780C01441011733FFFF670089
:10F70000039D1733FFFFE702A39879713C083ED2AF
:10F71000B7070C003ED43C083ED683C79500AE84A4
:10F720002A8993F7F707A384F500A165938535042B
:10F73000481097A0FFFFE780E02BC165FD1501444D
:10F74000176AFF1F130A0A66930A400EAE892E8BB2
:10F750002EC697B0FFFFE7802022420593170401D1
:10F760004181C183B24563E9A702C167FD17638781
:10F77000F500481097C0FFFFE780800E501001474A
:10F780008146A6854A8597A0FFFFE780004C45612A
:10F790001733FFFF670003933307540383270A0BD4
:10F7A000BA9703D6C701630A3601638A3501481048
:10F7B00097000000E78060F1DA85050451BFB2854B
:10F7C000EDBF1733FFFFE702C38B79717C083EC89A
:10F7D000B70711003ECA7C083ECC83C79500AA89B2
:10F7E000328593F7F707A384F5002E8997C0FFFFB2
:10F7F000E780C01485676378F504A165AA8489054C
:10F80000080897A0FFFFE780E01E268597400000CC
:10F81000E78060ED133415000A04A285080897C03C
:10F82000FFFFE780E001A685080897C0FFFFE7809B
:10F83000200325CC014781461008CA854E8597A034
:10F84000FFFFE780804045611733FFFF6700E386D5
:10F85000B30754030327CA0ABA9703D70700631CE8
:10F86000970003D62700638065050808970000000D
:10F87000E780A0E5DE8505042EC697B0FFFFE78090
:10F88000A0104205931704014181C183B245E3E111
:10F89000A7FCC167FD17E38FF5F8080897C0FFFFC5
:10F8A000E78000FC41BFB285F9B7C165FD15014491
:10F8B000176AFF1F130A0A4F930A80022E8BAE8B22
:10F8C00065BF1723FFFFE702437E184183471700F8
:10F8D00083460700A207D58FD207D1832390F50076
:10F8E00083472700034717008D45A207D98F9183CF
:10F8F0002310F60097C0FFFFE780A0E91723FFFF62
:10F900006700E37C1723FFFFE7028378C1640144AB
:10F910001769FF1F1309094993098002FD1497B065
:10F92000FFFFE78060066347A40001451723FFFF40
:10F9300067004379330534038327C90A3E9583570B
:10F940000500E38597FE0504D9BF1723FFFFE702F3
:10F9500023742A8AAE89B284B68A97400000E78071
:10F9600080D819E591473E851723FFFF670083750F
:10F970002A894E8597C00000E780E08E2A84638E36
:10F980000A048D476DD103570500C547E31D47FDA8
:10F990000347F9018546AD47E317D7FC8347450088
:10F9A00081CF4146A6855D0597F00000E780C09EA7
:10F9B000814755D9AD4745BF130965012302E500CD
:10F9C000CA85268597100000E780606231C1A5478F
:10F9D000E38B0AF82302040079B705C183570500B9
:10F9E000E39247F94146A685190597F00000E780A4
:10F9F000A09A81472DD99947BDB74E859700000041
:10FA0000E78080F02A84954739DD130955004DBF02
:10FA10004146A68523104401231134011305190022
:10FA200097F00000E780A099228597800000E7808A
:10FA3000A0EA81470DBF1723FFFFE7020367797133
:10FA40007C003ECCB7070A003ECE7C003ED083C788
:10FA50009500B2842E8493F7F707A384F50013066C
:10FA6000A1002A892C00268597000000E780A0E5E8
:10FA7000A16528088D0597A0FFFFE780A0F79040BB
:10FA80008355A10003558100854697000000E7805B
:10FA900000ECAA84AA85280897C0FFFFE78040DA17
:10FAA0000356A10083558100280897000000E780D5
:10FAB000C0C1300801478146A2854A8597A0FFFF53
:10FAC000E780A018854748103ED42302910202D651
:10FAD00097D0FFFFE78060BD45611723FFFF6700F8
:10FAE000035F1723FFFFE702435C79717C003ECC84
:10FAF000B7070A003ECE7C003ED083C79500B28493
:10FB00002E8493F7F707A384F5001306A1002A8932
:10FB10002C00268597000000E780E0DAA165280820
:10FB20008D0597A0FFFFE780E0EC90408355A10092
:10FB300003558100814697000000E78040E1AA84D8
:10FB4000AA85280897C0FFFFE78080CF0356A10051
:10FB500083558100280897000000E78000B730082F
:10FB600001478146A2854A8597A0FFFFE780E00D07
:10FB700048102302910202D402D697D0FFFFE780FB
:10FB8000C0B245611723FFFF670063541723FFFFCF
:10FB9000E702A35197000000E78060DB1723FFFF17
:10FBA0006700E3529767FF1F938787FF8843828030
:10FBB0001723FFFFE702634F835725004111AE84EF
:10FBC0002A842307B10017F5FFFF130525466C00B3
:10FBD0002316F10097A0FFFFE780204991C42285FA
:10FBE00097800000E780E0D6FD572310F40013064D
:10FBF00020028145130554009720FFFFE780E04D68
:10FC000041011723FFFF6700834C1723FFFFE70223
:10FC1000234879717C003ECCB7070A003ECE7C00B9
:10FC20003ED083C79500AA89AE8493F7F707328543
:10FC3000A384F5001306A1002C0097000000E780C4
:10FC400080C803558100114497400000E780A0A9B7
:10FC500015C50355A100014497B00000E780A060DE
:10FC600011CD035705008357810045446318F70001
:10FC7000854597000000E780E0F301442169930582
:10FC80003900280897A0FFFFE780C0D6A285280882
:10FC900097C0FFFFE780C0BA0356A10083558100DB
:10FCA000280897000000E78040A2300801478146FD
:10FCB000A6854E8597A0FFFFE78020F948104AD41B
:10FCC0002302810202D697D0FFFFE780009E4561A4
:10FCD0001723FFFF6700033F1723FFFFE702433BA4
:10FCE0009767FF1F938787EB2A8488432E8915C562
:10FCF000035745038357C4016311F7022326050206
:10FD000023180502410597D00000E780209C630678
:10FD1000090097800000E78060DB81449769FF1F3E
:10FD200093894908130A800297B0FFFFE780C0C596
:10FD300063C4A4049767FF1F938707EF9C4399C789
:10FD40000355C40197200000E780C0BD6307090088
:10FD5000228597800000E780C0A01306400E8145F1
:10FD600022859720FFFFE7804037FD57231EF400D0
:10FD70001723FFFF670003353385440383A7C90AB0
:10FD80003E95035705008357C4016317F700CA85E2
:10FD900097000000E78000E2850479B71723FFFF92
:10FDA000E702032F83C795004111AA8993F7F7074C
:10FDB000A384F5003285AE8497C0FFFFE78000B8CA
:10FDC00085676378F5042A8997400000E780A09151
:10FDD000014401CD83D70400314463882701854560
:10FDE00097000000E78080EF01444E85A2864A8696
:10FDF000A68597D0FFFFE780A09CA1679387170493
:10FE000048003EC42302810002C697D0FFFFE7806E
:10FE1000C08941011723FFFF6700C32A1723FFFF93
:10FE2000E70203279767FF1F938747D7804329C4BB
:10FE3000014597C00000E780002181470148C16467
:10FE40001CDC232E0403232004041769FF1F13095D
:10FE500069F501449309400EFD1497B0FFFFE78058
:10FE6000A0B1634FA400814517F5FFFF1305857FFF
:10FE700097A0FFFFE780601F1723FFFF6700832421
:10FE8000330534038327090B3E958357C5016387E8
:10FE90009700854597000000E78040E4050475BFA2
:10FEA0009357050113D78700A380F5009317050129
:10FEB000C183A1832380E5002381F500A381A500F0
:10FEC00082801723FFFFE702431E2300050083C73C
:10FED0001500A300F50083C725002301F50083C7A3
:10FEE0003500A301F50083C745002302F50083C751
:10FEF0005500A302F50083C7650093059500A30391
:10FF000005002303F5002304050032859700000057
:10FF1000E78040F91723FFFF6700631B1723FFFFEC
:10FF2000E70203174111E9540DCD85CD93F9C5FFC3
:10FF30002E842A89AA84338AA900B7EA04006318A8
:10FF40009A020D88854411CCB7E704009C5F829724
:10FF50002AC622866C003305390197E00000E7804D
:10FF60000046268541011723FFFF6700A31583A7DD
:10FF70008A039104829793170501C183A183A38EFD
:10FF8000F4FE93570501238FF4FEA183238EA4FE74
:10FF9000A38FF4FE6DB763E6D5021723FFFFE702D8
:10FFA000C310B28741113686BE8536C697E0000081
:10FFB000E780E040B246410136851723FFFF670026
:10FFC0000311814636858280838705001387F500FB
:10FFD0003D05FD8793F77708834607007D15860664
:10FFE000B58FA300F5006307B7007D17834717009F
:10FFF0009D83DDB782801723FFFFE702030BB7E77E
:020000040001F9
:10000000040083A7070932872A863A858297133529
:1000100015001723FFFF6700830B15C181478DC1B2
:100020001723FFFFE7026308414697E00000E780DF
:10003000003985473E851723FFFF67004309814745
:100040003E8582801DCD1723FFFFE7020306414650
:1000500081452A849720FFFFE7802008414681459B
:10006000130504039720FFFFE78020070147C167BE
:100070002322040438C87CC805451723FFFF670006
:1000800003050145828081473DCDB5CD1723FFFF94
:10009000E702A301B2842E891306800581452A84D4
:1000A0009720FFFFE7806003CA8524C42685970058
:1000B0000000E780C0F64146814522859720FFFF7A
:1000C000E780A0013044A285228597000000E780E8
:1000D000C0F293040401A285268597000000E78002
:1000E000E0EEA6851305040297000000E78000EE0D
:1000F000228597000000E78020F585473E8517237D
:10010000FFFF6700C3FC3E8582801723FFFFE702E5
:1001100023F84111E9540DCD85CD93F9C5FF2E8407
:100120002A89AA84338AA900B7EA040063984403A1
:100130000D88814411CCB7E704009C5F82972AC6E2
:1001400022866C003305390197E00000E780202704
:10015000268541011723FFFF6700C3F683A78A03A3
:100160009104829793170501C183A183A38EF4FEA6
:1001700093570501238FF4FEA183238EA4FEA38F42
:10018000F4FE6DB765CD1723FFFFE70263F0B2847D
:1001900011E605451723FFFF6700C3F22A842E8965
:1001A0000145EDD93C487848B3E6E700E5D69386AB
:1001B000F7FFB3B7F6007D17032A4404BA9734C893
:1001C0007CC863050A06C14913050A03B38949417E
:1001D0002295637D3601B2862E86A68597000000A3
:1001E000E780A0DB7C40BE9464C065B7CE862E86D7
:1001F000CE8597000000E78040DAC114D2944E9972
:1002000023220404A2879306040103C7070003C640
:1002100007038507318FA38FE7FEE398F6FE30448E
:10022000A285228597000000E78020DD2699C1493C
:100230003306994063EC9900A9DCA686A6851305D0
:10024000040397000000E78040D579BF8147B306DB
:10025000F4003307F6000347070083C5060085074F
:100260002D8F2380E600E39437FF3044A28522855A
:1002700097000000E78060D8C1145DBF014582800F
:100280000DC11723FFFFE70243E2130680058145F6
:100290009720FFFFE78060E405451723FFFF670015
:1002A00003E301458280814749C5C1C51723FFFF8C
:1002B000E702A3DFFC4141462E84AA846399C70468
:1002C00013860501A2878146C14503C7070003C500
:1002D00007038507298F3305D600034505008506EA
:1002E000298FA38FE7FEE392B6FE3044A2852685D0
:1002F00097000000E78060D0228597000000E7802B
:1003000060F885473E851723FFFF670043DC1385B0
:1003100007031D8E814522959720FFFFE780E0DBD4
:100320007C40130700F813060402A2972388E70213
:1003300051BF3E8582801723FFFFE70203D76D710F
:100340002E84B284AA859010280036899700000078
:10035000E780A0D309EDD55725A050400C402800D8
:1003600097000000E78040E27DD5FD142104F5F4FC
:100370002C004A8597000000E78020F3814761DD6B
:100380003E8551611723FFFF670063D41723FFFFEA
:10039000E702A3D141112EC432C62C0005469700B6
:1003A0000000E78080F941011723FFFF670023D297
:1003B0001723FFFFE70263CF01112A842EC602C86C
:1003C00002CA02CC02CE97E00000E780402BB24682
:1003D0002A86A285080897000000E78060FB137555
:1003E000F50F05611723FFFF670063CE1723FFFF9B
:1003F000E702A3CB7971B2872A8421462308B10092
:1004000013051101BE853AC436C697E00000E780A7
:1004100000FBB24693059101368597000000E78006
:1004200060A82285141035460C0897000000E7806C
:1004300020F62A84224701E921460C103A8597E0EC
:100440000000E780C0F7228545611723FFFF6700A2
:1004500003C81723FFFFE70243C57171AE84AA8565
:100460000A85328497000000E78060BB11C90A86C4
:10047000A685228597000000E78020B8814711E11A
:10048000C5473E854D611723FFFF670043C417230F
:10049000FFFFE70283BE1D712A8AB289BE843546FA
:1004A0008547130511012E8CB68A3A8BC28C468D76
:1004B0002308F10097E00000E78060F010100C08BE
:1004C0005285231F010097000000E780C0F82A84AE
:1004D0003DEDA1476313FD089307900591E0E547C3
:1004E0003546E2851305110113990A012308F1002D
:1004F0001359090197E00000E78060EC1357890069
:1005000093978A00D98F90080C085285231FF10019
:1005100097000000E78020F42A8415E9A1E493877E
:10052000FA0091831379F9003EC66313090041492B
:10053000668B8144C14B854DB247639F970C6A8699
:100540008C0033855C0197E00000E78040E722855E
:1005500025611723FFFF670003B693079004C9F0D6
:10056000A547BDBF834701050947C14B2308F100DB
:1005700083471105A58FA308F100938724008144C8
:1005800063E1FB04014714083386E6008C08B38658
:10059000E400BA95DA9683C6060083C50500050710
:1005A000AD8E2300D600E390E7FE4147639CE7044D
:1005B00090080C08528597000000E780C0E925D11B
:1005C00081A0B3069B00BA871008B305F600900817
:1005D0003E9603C506000346060085078506298E5C
:1005E0002380C500E39277FF998F90080C0852850D
:1005F000BE9497000000E78000E68947014749D193
:100600002A84B1B790083E96034606001408BE96A9
:100610002380C600850759BFB247850463879714B6
:1006200081471808B306F70098083E973386F9000B
:1006300003470700034606008507318F2380E60045
:10064000E39177FF90080C08528597000000E7803F
:1006500080E05DF53546E285130511012308B101FF
:1006600097E00000E780A0D513970401418393979A
:1006700084002183D98F10180C085285231FF100A4
:1006800097000000E78020DD25FD814710183387A3
:10069000F9003E960347070003460600B306FB0039
:1006A0008507318F2380E600E39277FF65A818085D
:1006B000B306F70098083E973386F9000347070012
:1006C000034606008507318F2380E600E3E127FF1C
:1006D000CA87639E770990080C085285970000002E
:1006E000E78060D711FD81479800B306F7009008B6
:1006F00018103E973E9603470700034606008507FD
:10070000318F2380E600E39177FF3546E2851305BC
:1007100011012308B10197E00000E78040CA139758
:1007200004014183939784002183D98F10180C080A
:100730005285231FF10097000000E780C0D1E3112C
:1007400005EC814710183387F9003E9603470700F0
:1007500003460600B306FB008507318F2380E600C1
:10076000E3E227FFC109410BC1BB814785B794086C
:10077000BE9683C6060018083E972300D70085075B
:1007800089BF638006321723FFFFE702038F597189
:100790002A84BE89B28B85473546130511022E8BFC
:1007A000468C4289BA8A368A2300F10297E000001B
:1007B000E780E0C010180C10228523170102970073
:1007C0000000E78040C963180512A147631FFC06BB
:1007D0009307900563930900E5473546DA851305CD
:1007E000110293140A012300F102C18097E0000076
:1007F000E780E0BC93178A0013D78400D98F900854
:100800000C1022852317F10297000000E780A0C496
:100810007DE1639209049307FA00BD88918391E01A
:10082000C144C207C183DE8C814A3EC6414DB247F6
:1008300063E2FA0E6286B3854B01881097E00000F0
:10084000E78080B54DC93D557DA093079004E396A0
:1008500009F8A54759B7834701050947C14C23004B
:10086000F10283471105B3C7F900A300F102938792
:100870002900814963E1FC04814618103306D70042
:100880008C083387D900B69556970347070083C570
:10089000050085062D8F2300E600E390D7FE414733
:1008A0006390E70690080C10228597000000E7800F
:1008B00080BA35D189A0B3863A01BA871010B30542
:1008C000F60090083E9603C506000346060085071D
:1008D0008506298E2380C500E39297FF3387EC407D
:1008E00090080C102285BA9997000000E780A0B606
:1008F0008947014741D165611713FFFF6700A37B5B
:1009000090083E96034606001410BE962380C6004B
:10091000850779B7B247850A93990A01939D8A00A2
:1009200093D909016391570F85473546DA85130539
:1009300011022300F10293D9890097E00000E780BB
:1009400000A8B3ED3D0190000C1022852317B103E0
:1009500097000000E78020B059FD8147A68963EA2F
:10096000970626860C084A8597E00000E78020A5B8
:1009700081471810B306F700100898083E973E9676
:1009800003470700034606008507318F2380E600F2
:10099000E3E197FE639FA90590080C10228597005C
:1009A0000000E78040AB21F981479810B306F700BB
:1009B000900818183E973E96034707000346060026
:1009C0008507318F2380E600E391A7FF4109C10C21
:1009D000B9BD18089000B306F7003E963387FC00B7
:1009E00003470700034606008507318F2380E60092
:1009F000B5B798084E97034707001C10CE97238081
:100A0000E700850941BF85473546DA8513051102A0
:100A10002300F10293D9890097E00000E780209A33
:100A2000B3ED3D0190000C1022852317B103970010
:100A30000000E78040A2E31005EC81471808900011
:100A4000B306F7003E963387FC00034707000346D2
:100A500006008507318F2380E600E391A7FF41461A
:100A60000C084A8597E00000E780609581471810E0
:100A7000B306F700100898083E973E960347070014
:100A8000034606008507318F2380E600E391A7FF28
:100A900090080C10228597000000E780C09B1DD5B0
:100AA00099BD7D5582801713FFFFE7020360011196
:100AB0002A842E8593055100328902C002C202C4E5
:100AC00002C69304740097F0FFFFE780A03D1D4627
:100AD000A6851305910097E00000E780408E10087E
:100AE0008A854A8597000000E780E09619ED930714
:100AF0001400180883C6070003460700850705078A
:100B0000B18EA38FD7FEE397F4FE05611713FFFFA5
:100B10006700E35B1713FFFFE70283572E848C41C6
:100B20004111AA89838715003289914463D3070054
:100B3000A1449757FF1F9387A75D9C43A1C7C1CAD4
:100B40008D472310F10083C725004A852301F1005A
:100B500083C73500A301F10083C745002302F100DC
:100B600083C75500A302F10083C765009305910078
:100B7000A30301002303F1002304010097F0FFFF0A
:100B8000E78040320C404A860A8597F0FFFFE780F5
:100B900080330328040083564400A6881D0881473B
:100BA0000147E51642868A854E8597000000E7805A
:100BB000408E2A8919E5A685228597B0FFFFE78038
:100BC000E0C14A8541011713FFFF6700A34F4A8622
:100BD0000A8597F0FFFFE780002F6DB71713FFFF1F
:100BE000E702034B2E848C414111AA8983871500AB
:100BF0003289914463D30700A1449757FF1F93871D
:100C000027519C43A1C7C1C68D472310F10083C75C
:100C100025004A852301F10083C73500A301F100B7
:100C200083C745002302F10083C75500A302F100EA
:100C300083C7650093059100A30301002303F1001E
:100C40002304010097F0FFFFE780C0250C404A868F
:100C50000A8597F0FFFFE7800027835644000328AA
:100C600004008A85858EC2061D08C1822312D40025
:100C7000A68881470147E51642864E859700000009
:100C8000E78060B041011713FFFF6700A3434A8666
:100C90000A8597F0FFFFE78000234DBF1713FFFF82
:100CA000E702A340B335B000011185052A89131569
:100CB000F601336515012308B1009305110136844F
:100CC0003AC632C03EC442C297F0FFFFE780801DA3
:100CD000A2471248425593D68700230BF100930593
:100CE000910193578800A30AD100A30BF100230CB4
:100CF000010197F0FFFFE780E01A32470246032820
:100D00000400B337E000835644009207914411C2B7
:100D1000A1444A85A68842860C0897F0FFFFE78029
:100D200040772A8919E5A685228597B0FFFFE780DD
:100D3000E0AA4A8505611713FFFF670043391713BF
:100D4000FFFFE702E33401113EC68647B335B0002A
:100D50008505AA891315F6015D8D2308B100930559
:100D6000110136843A89B28442C446C297F0FFFF2B
:100D7000E780401322489248164593578800A30AFB
:100D8000F1009305910193D78800230B0101A30B78
:100D9000F100230C110197F0FFFFE780A01032470C
:100DA000104083564400B337E0009207032809003F
:100DB000914891C0A1480C084E8597000000E7803B
:100DC000809CAA8401E9835544004A8597B0FFFFBF
:100DD000E780C0A0268505611713FFFF6700832EFB
:100DE000AA959307F00F17170100130727A363179E
:100DF000B50013C5F7FF1375F50F8280050583460F
:100E0000F5FFB58FBA9783C70700D5B703574500DD
:100E100014419307F00F17160100130626A036970A
:100E200042074183139506014181631BE500AD8FA5
:100E3000B29703C50700130515F31335150082801B
:100E4000850603C5F6FFA98FB29783C70700D9BFF0
:100E50001713FFFFE7026325B28736842E86BA8612
:100E6000AA853E85BA8497F0FFFFE7806052634F02
:100E70000500228597E00000E78060802A86A6862C
:100E8000A285268597F0FFFFE78080501713FFFFAC
:100E90006700E3231713FFFFE702831F5D712A8BAF
:100EA000AE8A171501001305E5942C00B284368A2A
:100EB000BA893E8997F0FFFFE780C04F2A845DE141
:100EC00034104146DA85280097F0FFFFE780404C58
:100ED0002A8449E98547A303F100A6C2930771005C
:100EE0002408BEC4A68685470D462C18281002DCAF
:100EF00002DED6C0BEC697F0FFFFE78000442A841A
:100F000035E183477102A6860D4693F7F707230064
:100F1000FA00C1473EDE2C188947281026DCA303BF
:100F2000F10097F0FFFFE78040412A8405ED41463C
:100F3000A6854E8597D00000E78060488D47A6863D
:100F40000D462C182810A303F10097F0FFFFE7804F
:100F5000C03E2A8401E94146A6854A8597D0000013
:100F6000E780E045228561611713FFFF6700831565
:100F70001713FFFFE702631397F70000938707EF4C
:100F8000984383C7470079712A89AE8417150100F9
:100F90001305C5860C083AC42306F10097F0FFFF3D
:100FA000E78040412A8405ED14104146CA850808AF
:100FB00097F0FFFFE780C03D2A8415E1140815462D
:100FC0002C00081097F0FFFFE780803C2A8401E99D
:100FD00021462C08268597D00000E780403E2285D8
:100FE00045611713FFFF6700830E1713FFFFE7022A
:100FF000C30B97F70000938767E79C477971AA8432
:101000002E84170501001305E57F0C083EC697F0F6
:10101000FFFFE780203A0DE914104146A685080835
:1010200097F0FFFFE780C03605E1140811466C0019
:10103000081097F0FFFFE780A03519E58347F1011D
:1010400093F7F7032300F40045611713FFFF6700D0
:1010500003081713FFFFE70243053688A1488147BD
:101060000147E54697F0FFFFE780A0421713FFFF17
:101070006700E3051713FFFFE70223033688A14843
:1010800081470147E54697F0FFFFE780C06F1713E0
:10109000FFFF6700C3031713FFFFE70203010111FE
:1010A0002A842E850C0832C697F0FFFFE780803037
:1010B00009ED324797060100938646731008C14533
:1010C000228597000000E780E0D805611713FFFF35
:1010D0006700E3FF1713FFFFE70223FD4111C1473C
:1010E0002EC032C48A8509463EC23EC697F0FFFF35
:1010F000E780A02441011713FFFF670043FD17138A
:10110000FFFFE70283FA4111AE8613061009AA8594
:101110000A8502C002C202C402C697F0FFFFE78040
:10112000202741011713FFFF670063FA1713FFFF22
:10113000E702A3F73287970601009386266D2E8675
:101140009305000297000000E780C0D01713FFFF4F
:101150006700E3F71713FFFFE70223F57971C14733
:101160002ACC2ED032D42C080D4628003ECE3ED2BA
:101170003ED602C402C602C802CA97F0FFFFE7804B
:10118000C01B45611713FFFF670063F41713FFFFD0
:10119000E702A3F10111AA842E84170501001305AB
:1011A00065678A8597F0FFFFE780C02015E5140882
:1011B0004146A6850A8597F0FFFFE780601D09ED8F
:1011C0008347E1010347F101A207D98FCA07C98309
:1011D0006177D98F2310F40005611713FFFF6700B3
:1011E00003EF15CD1713FFFFE70223EC9757FF1FFF
:1011F0009387879F90439755FF1F9385259F17558A
:10120000FF1F1305659A97D00000E78000C51755AA
:10121000FF1F130565991713FFFF670043EB175571
:10122000FF1F1305659882808DCD1713FFFFE7021E
:10123000C3E79757FF1F9387279B944301112E8481
:101240000A869755FF1F9385659A97D00000E7801F
:1012500040C60A850294014505611713FFFF670028
:1012600003E77D5582801713FFFFE70203E497D061
:101270000000E78080D19757FF1F23A7A79617F597
:10128000FFFF1305E5C997B00000E780C07417138E
:10129000FFFF6700C3E31757FF1F13072797931735
:1012A000150008433E95FD572310F5008280171363
:1012B000FFFFE70283DF2A84084009E51713FFFFD9
:1012C0006700E3E01C4158401CC06313E5005CC0AC
:1012D0008347550023200500F99BA302F50097A042
:1012E000FFFFE780207CC9BF1713FFFFE70243DA47
:1012F0009757FF1F9387879398432A8411CB83477F
:10130000350093F7070289C7035505008945029701
:101310001305440197B00000E780403B835504006B
:101320000355E40097300000E780A00C485819C529
:1013300097A0FFFFE7800077232A040213058403A8
:1013400097000000E780E0F68144B1499790FFFFE5
:10135000E780C06D63CBA4028347340023200404DC
:1013600093F727FCA301F40000489790FFFFE78064
:10137000E06C13161500814522859710FFFFE7806A
:10138000C0D51713FFFF6700E3D3B38734030329E6
:10139000040385043E994A8597000000E78060F1C8
:1013A0002304090065B78347350093F7070299E3E3
:1013B000014582808357E500E39CB7FEC167FD17B6
:1013C0006316F60005458280054599A81713FFFFAF
:1013D000E702A3CD93170601C187B2842A8401498D
:1013E0006359F002835705009DCB01456367F60002
:1013F000034584003E953325A6001375F50F0DA017
:101400001C4813171900BA9783D70700E38E97FA81
:1014100005099790FFFFE7806062E343A9FE01455D
:101420001713FFFF6700A3CA1713FFFFE70243C6A6
:10143000AE89AA849790FFFFE78000562A8497D050
:10144000FFFFE780A02EAA860147130684019705B7
:101450000000938585E41745FF1F1305657B979072
:10146000FFFFE780801C2A8925C98C441304C5002E
:1014700022859E0593F5050897A0FFFFE780403C75
:10148000CC4083877400E18163DD070493E50508A0
:10149000228597A0FFFFE780A03A0D469385440080
:1014A000228597A0FFFFE780C03683D50400228500
:1014B00097A0FFFFE780E03D83D52400228597A019
:1014C000FFFFE780003D03D6490083A50900228580
:1014D00097A0FFFFE780E0334A851713FFFF6700FF
:1014E00063BE93F5F5076DB71713FFFFE702E3BB84
:1014F00001112A84328532C697A0FFFFE780E027DA
:101500009780FFFFE7806034835704001757FF1F61
:10151000130747893246231BF100930700F8A30DF8
:10152000F1001C471843231AA1008983858BB30758
:10153000F740B28548083ECE231C0100230D010070
:1015400097000000E78080EE05611713FFFF67003A
:1015500003B81713FFFFE702A3B3004101453DC4E1
:101560009304C40026853289AE8997A0FFFFE780E7
:10157000C02495452A8A2685035B040197A0FFFFB6
:10158000E7802021268597A0FFFFE780603E8D45FC
:10159000AA8A268597A0FFFFE780A01F268597A02F
:1015A000FFFFE780E03C5C48420A135A0A01D297E9
:1015B0005CC423186401814763983A0146054D8154
:1015C000330625419337160013F5F70F1713FFFF66
:1015D000670043AF1713FFFFE702A3AA89692A8BAD
:1015E000AE8B328AB68A81440144314CFD19979002
:1015F000FFFFE780A04363CDA4009790FFFFE78043
:10160000E045018D33B5AA001713FFFF6700E3AA79
:101610003389840383270B003E9963170A008347AD
:10162000890085043E94E1B703560A00DE854A85A9
:1016300033F6C90097000000E780E0F16DD1054561
:10164000E1B71713FFFFE70243A601112A847C00CC
:101650000355E5003ECAB70707003ECC7C003ECEEE
:1016600097200000E78020082A898545480897A030
:10167000FFFFE78020399945480897A0FFFFE780E2
:10168000E015AA844A8597200000E780A0082380FF
:10169000A4009747FF1F9387E7709C43416613069A
:1016A00006F09396870113D78701558F93D687004D
:1016B000F18E558FA207B706FF00F58FD98F11461F
:1016C0002C00138514003EC497D00000E78020CF83
:1016D0005008A38204008945228597000000E78016
:1016E000E0E019C9AA851305840397A0FFFFE780EE
:1016F000E0313C4085073CC005611713FFFF6700E0
:10170000039D1713FFFFE702439A9790FFFFE780BF
:10171000E0342A8405049790FFFFE78020333305E7
:10172000A402F14791453305F50297200000E780B8
:1017300020BA11E565551713FFFF670043999747D6
:10174000FF1F23ADA74C9790FFFFE78020312A842D
:1017500005049790FFFFE780602F3305A4028945B9
:10176000060597200000E780A0B669D59747FF1FC0
:1017700023AEA7489790FFFFE780402E2A840504F8
:101780009790FFFFE780802C3304A4029747FF1F48
:10179000239087489790FFFFE780402C2A849790FA
:1017A000FFFFE780A02A930714003385A70297471D
:1017B000FF1F2390A74697070100938767C9174724
:1017C000FF1F232BF7440145BDB71713FFFFE702A7
:1017D000238CAA842E8901449749FF1F9389895C31
:1017E000130A80069790FFFFE78040266347A40016
:1017F00001451713FFFF6700E38C3305440383A7FC
:1018000009024A86A6853E9597000000E780E0B968
:1018100019E10504C1BF0545E9BF1713FFFFE70242
:101820004386AA8A2E8BB28B368C3A8A8144014435
:101830008149974CFF1F938CEC56130D80069790AF
:10184000FFFFE780A02063C9A40011E085494E8511
:101850001713FFFF670063863389A40383A70C0275
:101860005E86D6853E994A8597000000E780E0B302
:101870001DC19790FFFFE780601E0544636D450121
:10188000D2866286DA851305090397000000E78097
:10189000A0D411C1854985045DB71703FFFFE70296
:1018A000237FC16441112A8901449749FF1F93890D
:1018B000694F130A8006FD1436C632C42EC29790B3
:1018C000FFFFE780A01892452246B2466348A40075
:1018D000014541011703FFFF6700C37E3305440341
:1018E00083A709023E9509C683473500C18B9DC772
:1018F00091C68347350093F707028DC363069900AD
:101900008357E500639C27010357050001CB63E77C
:10191000E50083478500BA97E3CDF5FA050469BF72
:101920001703FFFFE702C376C1642A890144974980
:10193000FF1F93892947130A8006FD149790FFFF24
:10194000E780C0106346A4001703FFFF670083779A
:101950003305440383A709023E958357E500638A54
:101960009700630499006396270197000000E780C1
:10197000E0970504E1B71703FFFFE70203708969E9
:101980002A8AAE8A328BB68B8144174CFF1F130C08
:101990006C41930C8006314DFD199790FFFFE78055
:1019A000E00A63C6A4001703FFFF6700C370338912
:1019B000940383270C028355CA015A863E994A85AF
:1019C00097000000E780609E31C1814D15A03384EF
:1019D000AD038327090303D60B00D68533F6C90070
:1019E0003E94228597000000E780E0B609E9850D66
:1019F0009790FFFFE7808003E3CBADFC01A8228531
:101A000097000000E780E08A23040400850471B792
:101A10001703FFFFE702E3664169AA8A014A174BF1
:101A2000FF1F130B2B387D19C14B054C9790FFFFFF
:101A3000E780C0016346AA001703FFFF6700E36762
:101A400093098006B3073A0383290B02BE9983D713
:101A5000E900638E270163842A01639A570103A476
:101A6000890301E84E8597000000E780C0BD050AA4
:101A700075BF83570401639977099304C4002685D1
:101A800097A0FFFFE78060D385452A8D2685835C7C
:101A9000040197A0FFFFE780C0CF268597A0FFFF36
:101AA000E780A0E762056185635905048D452685B9
:101AB00097A0FFFFE780E0CD8945268597A0FFFF2F
:101AC000E78020CD8945268597A0FFFFE78060CC81
:101AD0008545268597A0FFFFE780E0CC834705007A
:101AE000094793F7F707639AE7009945268597A07A
:101AF000FFFFE78040CBA30285014848337D2D01DD
:101B0000231894016A9548C40040A1BF1703FFFF42
:101B1000E702A35937E404008327041D82979747FF
:101B2000FF1F83C727151725FF1F1305659CA300FB
:101B3000F5008327441C82978327841C8146130663
:101B4000F00F8145014582971703FFFF6700235877
:101B50001747FF1F1307070218439745FF1F83C549
:101B600065119747FF1F9387670F834687030346D7
:101B700097036397D5009747FF1F238DC70E828079
:101B800083C587010347A7036317B6009747FF1F65
:101B90002382E70E828003C687016317C700974739
:101BA000FF1F2389D70C828083C687011307500249
:101BB0006319D700930760021747FF1F230CF70A2A
:101BC000828083C68701130660026315D6009307DF
:101BD0007002DDB783C7870155BF9747FF1F938703
:101BE000E707D44B0947638DE6081703FFFFE702B9
:101BF000C34B1749FF1F1309A9033E8483470900FC
:101C0000918B9DCFB7E4040083A7041D829783A71F
:101C1000441C1745FF1F13052502829783A7841CC8
:101C200081461746FF1F03462603814501458297DB
:101C300021C583470900ED9B1747FF1F230AF7FEC5
:101C40008347040093F7F70F85CB91471747FF1F92
:101C50002320F70297000000E78080EB9700000048
:101C6000E78040EFB7E70400BC4F41469145174578
:101C7000FF1F034525FF82971703FFFF67002345DA
:101C800082801703FFFFE70243428D47411163063D
:101C9000F504C5476308F50285476310F5029747C9
:101CA000FF1F238BA7FCB7E70400BC4B9305001074
:101CB0001745FF1F034505FB829741011703FFFFEF
:101CC0006700E34085471747FF1F2307F7FAB7E789
:101CD0000400BC4B93050020E1BF9747FF1F93878B
:101CE000E7F7D44B1147638DE600B7E7040083A7FD
:101CF000071D8297B7E70400BC4B930500044DBF56
:101D000005491747FF1F232527F783C7070032C65A
:101D10002E8493F7F70FD5D3B7E4040083A7041DEF
:101D20007D141374F40F8297E37689FCB2459947CA
:101D300003C61500E3F0C7FCFC4409061745FF1F66
:101D40001305C5F38297BC48930500081745FF1F8C
:101D5000034545F1829779BF1703FFFFE702E3349C
:101D60001747FF1F130787EF4047184B1C40974644
:101D7000FF1F23ABF6EE6316E4001747FF1F232770
:101D8000F7EE130584FE9790FFFFE78000AA035546
:101D900064FF9780FFFFE780807297A0FFFFE780D6
:101DA00060D01703FFFF670083321703FFFFE702CE
:101DB000C32F9747FF1F938767EAD84BDC4789C734
:101DC00097000000E78080F985471747FF1F232110
:101DD000F7EA9747FF1F9387E7D99C4393050002D3
:101DE0001745FF1F034505E883C787031747FF1FF4
:101DF0002302F7E8B7E70400BC4B82971703FFFF05
:101E00006700E32C9747FF1F23ACA7E482801703EA
:101E1000FFFFE702E32737E404007C4CA1451745A8
:101E2000FF1F034525E482977C48A1451745FF1F06
:101E3000034545E39744FF1F938444E28297DC44C3
:101E400089EB97000000E78080D91703FFFF670048
:101E5000632703D567FF9780FFFFE7804066AA8965
:101E60006DD1D84891476310F7027C4C91451745D6
:101E7000FF1F034525DF82977C4891451745FF1FCB
:101E8000034545DE829703A9490103D40901894727
:101E9000B7E904001747FF1F232CF7DC83A7091DB0
:101EA00021044204829783C784011715FF1F13057D
:101EB000256461191717FF1FA30CF76283A7491C3C
:101EC000418082979747FF1F238807DA83A7C91CA1
:101ED000814609469375F40F4A85829711E9974721
:101EE000FF1F83C7A7E989C79710FF1FE78020CD91
:101EF000B7E70400BC4F2146A1451745FF1F034526
:101F000065D6829799B71703FFFFE702031A93F785
:101F1000052001112E8481CF97000000E78020E981
:101F20001345042005611703FFFF6700431A93F769
:101F30000510A9CF9744FF1F938444D2DC48970033
:101F40000000E78020C11747FF1F1307A7C21843EF
:101F500083C78401034787036318F700DC4489C7FC
:101F600097000000E78080DF85471747FF1F232188
:101F7000F7D0B7E70400BC4B930500021745FF1FDD
:101F8000034545CE82971345041069BF93F70508B2
:101F9000BDC79747FF1F83C777CEE91719469745F7
:101FA000FF1F9385C5CD1305D10093F4F70F174993
:101FB000FF1F0349A9CC97C00000E78040409397DA
:101FC0000401C1831747FF1F1307C7CB231DF1006F
:101FD000231CF1009747FF1F938747C83ACE3ACAA0
:101FE000D8432306010009CBDC439315890154082B
:101FF0000D46E185680082971345040825B793F7DD
:102000002500A5C39747FF1F938747C5D84B89472E
:102010006306F7029747FF1F83C787C113F727009F
:1020200011EF918B99CFB7E70400BC4F1306000A5C
:1020300089451745FF1F0345E5C2829713452400D4
:10204000D5B59747FF1F9387E7B29C4383C78703A4
:102050001747FF1F2300F7C297000000E78060DBEF
:10206000F1BF93F7050281CB97000000E78060DAAB
:102070001345040245BD93F7850081CB970000000E
:10208000E780E0D21345840071BD93F7150081CB42
:1020900097000000E780A0B41345140061B593F7E2
:1020A000450081CB97000000E78060B313454400F2
:1020B00095BD93F7050495C39747FF1F83C707BADC
:1020C00091CB97000000E780A0A491471747FF1F1E
:1020D0002320F7BA13450404B1B593F70501014570
:1020E000E38207E49747FF1F938747B7D84B914791
:1020F0006310F7049747FF1F938787B39C4313D759
:1021000027008583D98F858B91E7B7E7040083A7E4
:10211000071D8297B7E70400FC4F91451745FF1F45
:10212000034545B4829785471747FF1F2322F7B41D
:1021300013450401C5BB9747FF1F2381A7C48280B5
:102140001703FFFFE70263F69747FF1F23AE07B0B1
:102150009747FF1F23AC07B085471744FF1F1304A1
:1021600064A11747FF1F2325F7B01C4083C78703CF
:102170001747FF1F2300F7B09790FFFFE7804093BA
:1021800029C59717FF1F23A9A7361C401705000074
:102190001305A5D783C787031747FF1F230CF7AC89
:1021A0001717FF1FA306F7349747FF1FA38807AA37
:1021B000B7E7040083A7070882979747FF1F238389
:1021C000A7AA1703FFFF670083F0B7C7898E93871D
:1021D00067ED1717FF1F2321F73245BF1747FF1F72
:1021E0000347C7A7795555E79747FF1F938707A769
:1021F00003C7170005079746FF1FA381E6A603C77D
:1022000017008D463377D7029746FF1FA388E6A4B1
:1022100083C617001747FF1F1307C795184393F688
:10222000F60FA9EE834787031747FF1F2304F7A480
:1022300085471747FF1F2303F7A29747FF1F938781
:10224000279F9C430145998BA9E71703FFFFE702EE
:10225000C3E537E404007C48C1451745FF1F03452B
:1022600065A082973C4885451745FF1F0345859F1C
:10227000829701451703FFFF670063E583C71700D7
:1022800085466395F6008347970379BF8347A70385
:1022900061BF82809747FF1F83C7479CA1CF170369
:1022A000FFFFE70283E037E404009747FF1F23871F
:1022B000079A7C4885451745FF1F0345A59A8297D5
:1022C0007C4C91451745FF1F0345C59982977C4873
:1022D00091451745FF1F0345E59882973C48C14546
:1022E0001745FF1F03450598829701451703FFFF18
:1022F0006700E3DD795582801703FFFFE702E3DA29
:102300002A84035565FF9780FFFFE780401B9747AE
:10231000FF1F9387A794D847BE841DEF9790FFFFB8
:10232000E78080779C48232004009DEB9747FF1FA0
:1023300023AE87929747FF1F23A88792B7E7040031
:10234000BC4B89451745FF1F0345C5918297014541
:102350001703FFFF6700A3D7630A8700184375BF01
:1023600080C39747FF1F23A38790C9BF7955CDB777
:102370001703FFFFE70263D39747FF1F938747A029
:1023800088432326050023240500510597A000005B
:10239000E780C0331703FFFF670063D31703FFFF16
:1023A000E702A3D01744FF1F1304849D1C40411172
:1023B00099CF9C472302B5002AC61CC19700000094
:1023C000E78040FB1C409C4B99C3324582974101FA
:1023D0001703FFFF6700A3CF1703FFFFE702E3CC5C
:1023E0004111444D328532842EC69790FFFFE7801D
:1023F000C0522AC422859790FFFFE780205403A88B
:102400004400630C0800B24583574400184022463C
:1024100083D54500AA862685029841011703FFFF50
:102420006700E3CA1703FFFFE70223C8404D1DC83A
:1024300008C097050000938565031305440197A024
:102440000000E78040169747FF1F938767939C43E0
:10245000014589E79747FF1F23A487921703FFFFD2
:102460006700E3C67D55DDBF1703FFFFE702E3C347
:10247000011168009305F00F02C602C802CA02CC1F
:1024800002CE97000000E780A0F105611703FFFF6F
:102490006700E3C39747FF1F9387878E9C43D84706
:1024A000A1679D076319F7021703FFFFE702E3BF68
:1024B000011132859790FFFFE7802046230AA10093
:1024C0008145680097000000E78080ED05611703F3
:1024D000FFFF6700C3BF82809747FF1F9387478A2C
:1024E0009C43D847A167938777036319F7021703C3
:1024F000FFFFE70283BB011132859790FFFFE78062
:10250000C041230AA1008145680097000000E780D0
:1025100020E905611703FFFF670063BB82809747CF
:10252000FF1F9387E7859C43D84795476316F704B9
:102530001703FFFFE70263B70111328532849790DA
:10254000FFFFE780803D230AA10022859790FFFFCF
:10255000E780C03E83574400231BA10081453ECC49
:102560001C4068003ECE97000000E78060E30561F4
:102570001703FFFF6700A3B58280930785FF8DC314
:102580008327C5FF91CFDC4B81CF1703FFFFE70205
:10259000C3B1032585FF82971703FFFF670023B3AD
:1025A00082801703FFFFE70243B02A8432859790A9
:1025B000FFFFE7808036BD4763EBA70018449377A1
:1025C000F5000345B70041995D8DA305A7001703EA
:1025D000FFFF6700C3AF1703FFFFE70203AD011161
:1025E0007C003ECAB70707003ECC7C003ECE5C4D67
:1025F000A9C72A8413858700AE8497A00000E780CE
:10260000E0FCA1652A899D0548089770FFFFE780D7
:10261000603E9305803EB345B902480893F5F50F37
:102620009790FFFFE780C021014781465008A685AB
:1026300022859770FFFFE780406105611703FFFF68
:102640006700E3A81703FFFFE70223A69700000037
:10265000E780A0F81703FFFF670063A71703FFFFDA
:10266000E702A3A401117C00AE843ECAA165B707AE
:1026700007002A843ECC48087C00938575033ECE33
:102680009770FFFFE78000371C44480883C5B700F8
:10269000BD899790FFFFE780A01A50080147814647
:1026A000A68522859770FFFFE780205A05611703F2
:1026B000FFFF6700C3A11703FFFFE702039F2A8400
:1026C000AE8497000000E78000EEA6852285970083
:1026D0000000E780E0F81703FFFF6700439F170340
:1026E000FFFFE702839C97000000E78060F7170375
:1026F000FFFF6700C39D1703FFFFE702039B03294A
:10270000C5014111630809022A843285B284979079
:10271000FFFFE78080202AC626859790FFFFE7808D
:10272000E021832749002A8691C7DC4781C7B2454B
:102730002285829741011703FFFF67004399170322
:10274000FFFFE7028396444D91CC2A84328597900F
:10275000FFFFE780A01EDC40AA8589C79C4799C37C
:10276000228582971703FFFF670063961703FFFF19
:10277000E7020392032AC5014111630D0A062E895F
:10278000AA849545328532849770FFFFE7808026C2
:10279000854522859790FFFFE7804004AA89CA8576
:1027A00022859790FFFFE780A00B83274A008DCBFF
:1027B000DC439DC722859790FFFFE780A000832719
:1027C0004A00104083564400DC437115A307A10062
:1027D000B2961307F1004E86CA852685829701C5F9
:1027E0002380090001A88345F10022859790FFFF0F
:1027F000E780C0FE41011703FFFF6700A38C1703AA
:10280000FFFFE702838A65711C083EC2B70780019B
:102810003EC41C0832893EC62A84AE84970000005C
:10282000E780A0ED4A859790FFFFE780201183574E
:10283000A1008DC3AA855000228597000000E78083
:1028400020F3014781465000A68522859770FFFF3F
:10285000E780A03F59611703FFFF67004387170315
:10286000FFFFE702E38265711C088329C5013EC2B0
:10287000B70780013EC41C082A84AE8432893EC654
:1028800097000000E780E0EB638A09024A85979091
:10289000FFFFE780A00A8357A100AA8585C35000E7
:1028A000228597000000E780A0EC01478146500098
:1028B000A68522859770FFFFE780203959611703AD
:1028C000FFFF6700238017F3FEFFE702037E6571B9
:1028D0001C083EC2B70780013EC42A841C0832850A
:1028E0003EC6AE849790FFFFE78040058357A10066
:1028F0008DC3AA855000228597000000E78040E73D
:10290000014781465000A68522859770FFFFE7802A
:10291000C033596117F3FEFF6700637B17F3FEFFB7
:10292000E702A378444D81EC8347450093B7170035
:10293000B307F0403E8517F3FEFF67004379184563
:10294000FD576DDB97070000938747032A845CCB14
:10295000970500009385A5C21385840097A0000009
:10296000E78060C480C003474400814761F71737A0
:10297000FF1F232997407DBF17F3FEFFE702437136
:102980008329C50141110329850081476387090A0D
:102990000324090191452A8A22859770FFFFE78069
:1029A0006005854522859790FFFFE78020E38945F4
:1029B000AA8A22859790FFFFE78040E2AA84977059
:1029C000FFFFE780400A83A749002A8B8DCB9C43F9
:1029D0009DC722859790FFFFE780C0DE83A749004F
:1029E000A306A1001040835644009C431307D10066
:1029F000B296D6851306E1005285829709CD83579A
:102A00000B002380F400A183A380F40023800A003C
:102A1000A306010039A88357E10022852380F40032
:102A20008345D100A183A380F4009790FFFFE78046
:102A3000E0DA8347D100B337F0000347B9009207CB
:102A400001453D9BD98FA305F900410117F3FEFF16
:102A50006700436717F3FEFFE702236541110DEDA1
:102A60009737FF1F93870732804315C80440130927
:102A700084009DC95C4099C79C4B89C726852EC69A
:102A80008297B2459307803EB385F5024A8597A0A9
:102A90000000E78060C121A0404DAA8469F841018F
:102AA00017F3FEFF6700A3624A8597A00000E78046
:102AB000E0C15C40EDD7DC4BFDD326858297C5B7DE
:102AC00017F3FEFFE702635E2A8432859790FFFFCB
:102AD000E780A0E4AA85228597000000E780C0F780
:102AE00017F3FEFF6700A35E17F3FEFFE702E35B49
:102AF0002A84AE8497000000E780C0FCA68522856A
:102B000097000000E78060AD17F3FEFF6700235CCD
:102B100008413355B5000589828017F3FEFFE702AF
:102B2000C3581734FF1F1304E4271C5C011123173B
:102B300001008D83858BA303F1008327040B2318E9
:102B400001002319010003D7C7013ECA3C0023142A
:102B5000E1007D572315E1000357C4023ECC02CEAD
:102B60002316E1009770FFFFE78020CE8357E10135
:102B7000231EA10093F707E093E71710231FF1002E
:102B80009737FF1F83C7A72495C305470145638A6D
:102B9000E7008347840393E727001737FF1F230FBE
:102BA000F722056117F3FEFF67006352814717F7AD
:102BB00000001307E7E585461306710085454808C0
:102BC00097900000E780408F69FD83478403F59B61
:102BD0001737FF1F2304F72085471737FF1F2308E8
:102BE000F71EC1B717F3FEFFE7022349973DFF1F0A
:102BF000938D4D1B03A6CD0639712A8981478144E7
